:020000021000EC
:10F00000F0FF002039F5010061F5010063F5010012
:10F0100065F5010067F5010069F5010000000000D9
:10F020000000000000000000000000006BF501007F
:10F030006DF50100000000006FF5010061BC0300E8
:10F040000152020073F50100F55302006152020003
:10F05000AD52020051640200A555020073F5010093
:10F0600073F50100A5BC030073F5010073F5010001
:10F0700073F50100115F020073F5010073F50100E3
:10F08000A1BC0300CD2A020073F5010073F5010055
:10F09000D52B0200B9D70300511C020073F5010003
:10F0A00073F5010073F5010073F50100B16602000C
:10F0B00073F5010073F5010000000000000000007E
:10F0C00073F5010073F5010073F5010073F501009C
:10F0D00073F50100DD60020073F50100000000001F
:10F0E0000000000000000000000000000000000020
:10F0F0000000000000000000000000000000000010
:10F1000000000000000000000000000000000000FF
:10F1100000000000000000000000000000000000EF
:10F4000010B5054C237833B9044B13B10448AFF35E
:10F4100000800123237010BD202E0020000000007A
:10F420009806060008B5034B1BB103490348AFF328
:10F43000008008BD00000000242E00209806060071
:10F44000154B002B08BF134B9D46A3F5803A0021B6
:10F450008B460F461348144A121A00F063F80F4BFC
:10F46000002B00D098470E4B002B00D0984700206F
:10F47000002104000D000D48002802D00C48AFF315
:10F48000008000F02BF82000290025F031FF00F06B
:10F4900011F800BF00000800F0FF0020000000008D
:10F4A00000000000202E0020C4C200200000000048
:10F4B0000000000008B5074B044613B10021AFF36C
:10F4C0000080054B1868836A03B19847204600F016
:10F4D00031F800BF00000000107C050070B50D4D34
:10F4E0000D4C641BA4100026A64209D10B4D0C4CF8
:10F4F00038F082FB641BA4100026A64205D170BD23
:10F5000055F8043B98470136EEE755F8043B984719
:10F510000136F2E7042E0020042E0020042E0020E5
:10F52000082E002002440346934200D1704703F89E
:10F53000011BF9E7FEE700BF0649074A074B9B1A84
:10F5400003DD043BC858D050FBDC06F0B5FEFFF7E6
:10F5500077FF0000A4060600402C0020202E00208B
:10F56000FEE7FEE7FEE7FEE7FEE7FEE7FEE7FEE773
:10F57000FEE7FEE71FB501238DF80030054B8DF83F
:10F58000080001916846D3E90012904705B05DF884
:10F5900004FB00BF20AE002061DF704748DF7047EA
:10F5A00010B50388012B11D8094A02EB03124388D6
:10F5B0005189CC1A032C09D4C3F57F43FD330B4486
:10F5C0005381002303804380184610BD0420FCE7CC
:10F5D00020B3002010B5124A0B6802EB00104268FD
:10F5E00073B15888033003EB800302F580524FF665
:10F5F000FF749A4202D91868013004D1002009E052
:10F6000002F10803F1E79888A04204D0188810B1ED
:10F610000B60012010BD5888033003EB8003E8E73E
:10F6200020B3002073B5436804460D4613B31E4A49
:10F6300011688B421ED3526893421BD813F003000B
:10F6400018D11A4A21891289914213D121689A68E6
:10F6500091420FD1164A5268934201D80A2004E021
:10F6600002F580529342F9D22880B0FA80F0400926
:10F6700002B070BD00232B801E46019601A9288888
:10F68000FFF7A8FF30B92B8801339BB22B80002BEA
:10F69000F3D0EDE7019B226899689142EED1636057
:10F6A000024B1B892381E3E70C2E0020E4AF0020EE
:10F6B00020B30020033083B240F2FD32934230B5D4
:10F6C0000ED909200BE0228965892A441A4492B296
:10F6D000B2F5806F08D2088062891344638130BD1F
:10F6E000024C20780028EED00720F8E720B3002055
:10F6F00010B50A494A788C78531CDBB29C4208BF8B
:10F7000000230C789C421FBF0370486802EB420242
:10F7100000EBC20008BF002010BD00BF9CB200205B
:10F72000AADF7047A9DF7047A7DF704785DF704702
:10F730007FDF70477EDF7047084A30B500230C2416
:10F7400004FB03F18D5A854202D10A44508830BD32
:10F750000133082BF4D14FF6FF70F8E74EAF0020CD
:10F760006EDF7047012804D0043804288CBF0020C5
:10F77000012070478378013B072B07D8DFE803F0AF
:10F7800007060606060704091423038070470123B1
:10F79000FBE743689B8809339B08F6E770B5054D86
:10F7A0000646002455F8043B304601349847052CA2
:10F7B000F8D170BD947D0500114BF0B500221426E0
:10F7C0001D4606FB02F4E75A874212D12344142651
:10F7D00000249A788A420AD001342246072A0BD89C
:10F7E00006FB02F3EF5A874208D1EB18F1D1184615
:10F7F000F0BD0132082AE4D10023F8E70132EDE739
:10F80000BCB40020F8B5074D074E074600243378F6
:10F81000A34200DCF8BD55F8043B38469847013454
:10F82000F5E700BFC0AF002071B100207DDF704759
:10F8300079DF70476DDF704758B1CB0801F00701E1
:10F84000C25C012303FA01F10A4214BF18460020EA
:10F85000704701207047000070B50A4E34680546B5
:10F8600054B1706860B1FF2D08D02946FFF7E4FF5E
:10F8700030B1F36803FB0544204670BD0024FBE76C
:10F880000446F9E7ACB4002030B5072185B0FFF796
:10F8900093FF044600283AD04568002D39D1007CFA
:10F8A000FFF7DAFF0721CDE902558DF80A1040B3C2
:10F8B000E368039003EB83031B019BB29B0802A840
:10F8C000ADF80830FFF756FF9DF80A00FFF74AFF32
:10F8D000D8B1114B1B789B0715D5BDF808500DF119
:10F8E00006012846FFF7E6FE48B9BDF80630A380BA
:10F8F000E5800A4B185C092803D005B030BD092803
:10F90000F7D90320F9E70220F3E70846F5E70520D9
:10F91000F3E70020F1E700BFE1AF00202C7C0500F9
:10F9200038B54FF6FF73984218BF01300D4614BF2B
:10F9300084B20024FF2C03D94FF6FF74204638BD53
:10F9400021462846FFF778FF0028F7D10134A4B2FA
:10F95000F0E7000038B5074C051E04F1080318BF96
:10F960001C4623682BB11A6822605B6828469847BA
:10F97000F7E738BDF8AE002040DF70473FDF704743
:10F980000023435082B043580193019B02B070475B
:10F990002DE9F0470D789DF820609DF824A00446DD
:10F9A0000F469946002D60D1D0F8243192F800809E
:10F9B0009BB14FF49271FFF7E3FF012363613B704A
:10F9C000B04550D1D4F80431002B4CD04FF48271A3
:10F9D0002046FFF7D5FF00251DE0D0F81C31FBB114
:10F9E0004FF48E71FFF7CCFFD0F824311BB14FF4E8
:10F9F00092712046DFE713789E4207D919F8033049
:10FA0000C0F81C35137801331370D9E70123BAF11C
:10FA1000000F03D0C3612846BDE8F0874361CFE7FC
:10FA2000D0F80831002BCBD04FF48471FFF7A8FF3A
:10FA3000D0F82431002BDAD113789E42C0D9D0F807
:10FA4000181509F8031013780133DBB21370721E16
:10FA5000934205D10223C0F8003201232362AFE7AD
:10FA60009E42FAD1ACE70125D5E74FF49271FFF73A
:10FA700087FF4FF48E71FFF783FF4FF48471FFF718
:10FA80007FFF9FE72DE9F3470C4605464FF482714F
:10FA900020461F469046FFF773FF4FF49271FFF721
:10FAA0006FFF4FF48E71FFF76BFF4FF48471FFF718
:10FAB00067FF0023012F85F8263085F8233008BF23
:10FAC00002224FF001030CBFC4F80022C4F8003238
:10FAD000236223602E6846BB05F1260A05F123093F
:10FAE000CDE900764346524649462046FFF750FF8F
:10FAF0000028F5D195F82330EBB1D4F8C434C4F81C
:10FB0000C434C3B113F0010F14BF4FF402400320FB
:10FB100048F2012213F0020F18BF104613F0040F31
:10FB200048F2022318BF184606E040F28623AB6075
:10FB3000AB68C4F80433002002B0BDE8F0872DE9BB
:10FB4000F3470C4605464FF4827120461F46164681
:10FB50009DF82880FFF714FF4FF49271FFF710FF14
:10FB60004FF48E71FFF70CFF4FF48471FFF708FF1D
:10FB70000023C4F8003285F8263085F823300123AD
:10FB80002362A36095F82620974232D9B35CC4F86B
:10FB90001C3595F82630013385F826302B687BBB61
:10FBA00005F1260A05F12309CDE9007833465246CE
:10FBB00049462046FFF7ECFE0028F5D195F82330A2
:10FBC00023B3D4F8C434C4F8C434FBB113F0010F28
:10FBD00014BF4FF40240032048F2012213F0020F39
:10FBE00018BF104613F0040F48F2022318BF18463E
:10FBF0000DE0B8F1000F01D0E361CFE76361CDE71D
:10FC000040F28623AB60AB68C4F80433002002B036
:10FC1000BDE8F0870023435082B043580193019B15
:10FC200002B0704708B502464FF492710068FFF7C2
:10FC3000F1FF4FF484711068FFF7ECFF13680122A5
:10FC40001A6008BD10B5CB7D0A464FF4847123B904
:10FC5000FFF7E0FFD0F8183510BDFFF7DBFF537E4C
:10FC6000D168D0F81805C854537E0133DBB25376FF
:10FC7000F2E70A4610B54FF48E71FFF7CBFF938A77
:10FC800091689BB2C95C938A01339BB29382C0F89E
:10FC90001C1510BD2DE9F04793F9005090B00024D9
:10FCA000013D6E46AD002746A446A0465FF0000E1B
:10FCB00003E05FEA080EBEEB050EB8EB0E0952F842
:10FCC00009A051F80E90A9FB0A9A14EB090457EB0E
:10FCD0000A075CF1000C1EF1040EAE4501DCC645BE
:10FCE000EBDD46F808403C4667465FF0000C18F133
:10FCF0000408A845DADDB8EB450FDADD46F8084020
:10FD0000D3F8B0303146984710B0BDE8F0871346BD
:10FD10000A46FFF7BFBFF0B5154689B01C46074637
:10FD20000E461A4629466846FFF7F1FF23466A4603
:10FD300039463846FFF7AEFF23462A4669466846ED
:10FD4000FFF7A8FF23466A4631463046FFF7A2FF79
:10FD500009B0F0BD00EB81010023884200D3704759
:10FD600051F8042D43EA52030B60D307F5E710B5B1
:10FD7000013A52B2130601D5002010BD50F82240BE
:10FD800051F822309C4205D802F1FF32F2D24FF0F6
:10FD9000FF30F2E70120F0E710B500235CB2A24289
:10FDA00000DC10BD51F8234040F823400133F5E753
:10FDB000013910B549B2041D0A06CBB204D4013989
:10FDC00054F82120002AF7D001335BB273B103F15C
:10FDD0008042013A50F82220002022B9013B00EB7A
:10FDE000431318B210BD52080130F6E71846F9E780
:10FDF000002310B51C465AB2914200DC10BD40F8F9
:10FE000023400133F7E7000000000000000000007D
:10FE1000C3F10803DB0070B50133002403A500BF64
:10FE20005B1920C940CAAD1B20C0184720C940CA71
:10FE3000B54120C020C940CAB54120C020C940CA30
:10FE4000B54120C020C940CAB54120C020C940CA20
:10FE5000B54120C020C940CAB54120C020C940CA10
:10FE6000B54120C06441B4FA84F0400970BD00BFC0
:10FE7000C3F10803DB0070B50133002403A500BF04
:10FE80005B1920C940CAAD1920C0184720C940CA13
:10FE9000754120C020C940CA754120C020C940CA50
:10FEA000754120C020C940CA754120C020C940CA40
:10FEB000754120C020C940CA754120C020C940CA30
:10FEC000754120C06441204670BD00BFF0B50822D6
:10FED00089B00C460646FFF75FFFCB6A03930B6BB6
:10FEE00004934B6B05938B6B0693CB6B07930027A7
:10FEF00008236A4669466846CDE901770097FFF70F
:10FF0000B7FF082305466A4631463046FFF7B0FF83
:10FF1000236B0393636B0493A36B0593E36B05441B
:10FF2000CDE906376A46082369466846FFF7A0FF11
:10FF3000082305446A4631463046FFF799FF236A95
:10FF40000093636A0193A36A0293A36B0693E36B26
:10FF50000793054408236A4631463046CDE90477C5
:10FF60000397FFF785FF636A0093A36AA26B01936F
:10FF7000E36A02930492636BE26B0393CDE905237A
:10FF8000236A0793054408236A4631463046FFF743
:10FF90006FFFE36A0093236B0193636B0293236A01
:10FFA0000693A36A0793054408236A463146304600
:10FFB000CDE904770397FFF72BFF236B0093636B67
:10FFC0000193A36B0293E36B0393636A0693E36A63
:10FFD00007932D1A08236A4631463046CDE9047747
:10FFE000FFF716FF636B0093A36B0193E36B029320
:10FFF000236A0393636A0493A36ACDE90537236BED
:020000022000DC
:1000000007932D1A08236A4631463046FFF700FF52
:10001000A36B0093E36BCDE90137636A0393A36A93
:100020000493E36ACDE90537636B07932D1A082320
:100030006A4631463046FFF7EBFE2D1A0D4C0FD4C1
:1000400035B9082231462046FFF791FE01280FD02E
:100050000823224631463046FFF7DAFE2D1AEFE735
:100060000823224631463046FFF702FF2D18F7D409
:1000700009B0F0BD447C05002DE9F04391B00F4676
:100080001C220021804609A8FFF74CFA01251C22FA
:10009000002101A80895FFF745FA394608AA11F989
:1000A000046B009533461046FFF7E2FE314608A880
:1000B000FFF77EFE013804B2012C07DC32466946A8
:1000C0004046FFF769FE11B0BDE8F0833A46684646
:1000D0006946FFF71CFE10AB601103EB80001FFAAE
:1000E00084F909F01F0350F8202C05FA03F313429A
:1000F00005D03B46424669466846FFF7CBFD09F10D
:10010000FF3424B2D8E770B5036813F00105064642
:10011000144605D013460A460146FFF7A9FE0546D8
:1001200021463046FFF716FE45B104F18042013A00
:1001300056F8223043F0004346F8223070BD70B5C7
:100140009DF910401E4623460546FFF761FE38B173
:100150002346324629462846BDE87040FFF788BE50
:1001600070BD2DE9F0438BB01446129D15F9046B58
:1001700000961F46804689462B460246214602A825
:10018000FFF7DDFF02A9129A0846FFF7C0FD129B98
:1001900002AA41464046FFF77DFD129B02AA214676
:1001A0002046FFF777FD2B464A46394638460096EB
:1001B000FFF7C5FF129A394602A8FFF7A8FD02A96A
:1001C0002B46424608460096FFF7B9FF02A92B4688
:1001D000224608460096FFF7B2FF2B4642462146CC
:1001E00020460096FFF7ABFF129B22464946484641
:1001F000FFF750FD2B4602AA414620460096FFF726
:100200009EFF129B224639463846FFF743FD2B4698
:100210004A46394638460096FFF791FF324602A912
:100220002046FFF7B9FD0BB0BDE8F08370B59DF92E
:1002300010401E4623460546FFF71AFE30B92246F7
:1002400029463046FFF793FD012807D02346324662
:1002500029462846BDE87040FFF7DABD70BD2DE99C
:10026000F0439BB01646229C14F9045B0095984617
:100270000746894623460246314612A8FFF75FFF2C
:1002800012A9229A0846FFF742FD229B12AA39467C
:100290003846FFF7FFFC229B12AA31463046FFF793
:1002A000F9FC23464A46414612A80095FFF7BEFFD7
:1002B00023464A46414640460095FFF740FF234605
:1002C0003A4631460AA80095FFF739FF229B0AAA51
:1002D00049464846FFF7DEFC2346324639460AA81F
:1002E0000095FFF7A3FF229A41463046FFF70FFD26
:1002F00023460AAA314630460095FFF720FF2346E1
:100300003246394602A80095FFF719FF229B02AA40
:1003100041464046FFF7BEFC23464A46414640461A
:100320000095FFF70CFF229A12A902A8FFF7EFFC35
:1003300002A923460AAA08460095FFF700FF2346B4
:100340003A4602A90AA80095FFF7F9FE0AA9229BDE
:1003500012AA0846FFF79EFC23464A460AA94846C9
:100360000095FFF7ECFE2A4602A93846FFF714FD78
:100370001BB0BDE8F0832DE9F04115468AB0044674
:1003800088461C22002103A8FFF7CCF82E1D95F902
:10039000007003232A46414620460293FFF7B7FC2C
:1003A000334602AA214620460097FFF7C8FE2B4697
:1003B000424621462046FFF76DFC0097334605F183
:1003C000840221462046FFF731FF0AB0BDE8F081E4
:1003D0000C4B1B78062B10D10B4B1B681A070CD14A
:1003E0000A4B186800F0F003302B08D000F0E00052
:1003F000A0F1400358425841704700207047012047
:10040000704700BFE00F00F0E40F00F0E80F00F0CD
:10041000094B1B78062B0CD1084B1B681A0708D117
:10042000074B186800F0F000A0F130035842584123
:1004300070470020704700BFE00F00F0E40F00F0AD
:10044000E80F00F010B9024B01221A60704700BF9C
:100450000050004010B50C494A6E042A044611D0E1
:100460000B6E1344032B02F101024A6688BF043B62
:10047000182202FB031318460021FFF753F82060EF
:10048000012010BD0020FCE7C0B3002010B50446D9
:1004900086B01422002101A8FFF744F86088ADF867
:1004A0000800FFF749F92378ADF80600092B0CD8AE
:1004B000DFE803F005051014161B1D0E1F2107238E
:1004C0008DF8043008238DF80C3001A8FFF79AF955
:1004D00006B010BD0D238DF80430F6E70E23FAE7C1
:1004E00007238DF804300523EDE70F23F3E71023EE
:1004F000F1E70523EFE706238DF80430A3680393A3
:10050000A388ADF80630E0E72DE9F041067904460E
:10051000407B174603360023834204DB51B93E601B
:100520000020BDE8F081226912F833200132164420
:100530000133F1E73B68B34229D3237833F0030852
:1005400027D10B7022794A708D1C2846A16837F09C
:1005500011FB2279617BA954AB180133627B4245C0
:10056000DDDD226912F8382003F8012B226902EB45
:10057000C801184612F83820496837F0FBFA22699A
:1005800012F838200346134408F10108E6E7042076
:10059000C7E70720C5E738B504461546084631B118
:1005A00062682B68934206D3216837F0E3FA6368E8
:1005B0002B60002038BD0420FCE708B5134644F248
:1005C0000102904203BF5A681988986800221AF005
:1005D00051FC000030B50B4B1B68012293F8501002
:1005E0000D338A4204DB405CB0FA80F0400930BD34
:1005F00013F8014B855CA54201D10132F1E70020DF
:10060000F5E700BF60AD002003681A78302A27D1D3
:100610005A1C02605A7802F0DF024F2A03D10233DB
:10062000036008207047582A03D10233036010206A
:100630007047422A04D0082013F8012F22B97047CE
:1006400002330360022070472E2A07D0A2F138013E
:10065000012903D9303A092AEED970470A20EBE77D
:100660000A20704770B5244B0022C3F80025234AA6
:10067000516831B12249C3F8081322490420C1F856
:100680008000D3F80C55D3F81445D3F80815D3F8E7
:1006900010054FF0FF36B542C3F8146518BF05F5D5
:1006A000E075C3F80C65C3F80865C3F810651EBF94
:1006B0004FF0A043022643F82560651C1FBF4FF092
:1006C000A04304F5E074022543F82450441C1FBFE6
:1006D00000F5E0704FF0A043022443F820404B1C8B
:1006E0001FBF4FF0A04301F5E071022043F8210045
:1006F0000023D376536070BD0020004020AE002060
:100700008402020000E100E070B58AB00C460146A8
:1007100068461E462DF0D2F80022214605A82DF08D
:10072000CDF868462CF07CFE044605A82CF078FE37
:10073000844205460DD0039832F0E0FC089832F070
:10074000DDFC002C01DB002D00DA56B9601B0AB07D
:1007500070BD002C07DA039832F0D0FC089832F014
:10076000CDFC0020F3E768462CF0FEFC05A82CF039
:10077000FBFCD6E7044A138A9BB223F0410343F003
:1007800040031382704700BF482E00200000000085
:100790002DE9F04F85B08A460390039C25782846C2
:1007A0002CF068FB0746C8B92D2D1AD1013401235E
:1007B00003940193DDF80CB0BAF1000F01D0CAF830
:1007C00000B003A8FFF720FF8046002835D1624D16
:1007D00000242046294605B0BDE8F08F013403947B
:1007E000DBE72B2D04BF013403940190E2E71846A8
:1007F00002932CF00DFBB0F10009029B20DBC845F1
:100800001EDD404636F038FC22462B4636F09EFC74
:1008100004460D46484636F02FFC22462B4636F05D
:10082000DFFA013604460D460396039E3378002B0B
:10083000DDD1B8F10A0F37D113E000240025F4E729
:10084000B8F10A0F30D12E2B0BD10FF20419D9E9D0
:10085000008901360396039E30783038C3B2092BE5
:1008600039D9039B1A7802F0DF02452A1CD15A1CA1
:1008700003925A782D2A01D02B2A05D12D3A5742BE
:1008800003F10203574103934FF000080A20039A33
:100890001378303BD9B2092936D9002F39D12F4FDF
:1008A0000026B8F1000F46D1039BBAF1000F01D02A
:1008B000CAF800309B458AD09BF800202E2A03D12D
:1008C0000BF1010B5B4582D0019B002B81D005F120
:1008D00000431D467DE736F0CFFB42464B4636F0DF
:1008E00035FC02460B462046294636F079FA0022AE
:1008F00004460D4640464946184B36F051FD013638
:10090000804689460396A6E7013200FB0838039229
:10091000BDE7124FC8F100080026B8F1000FC3D0A0
:100920002046294632463B4636F03AFD08F101089A
:1009300004460D46F1E72046294632463B4636F04E
:1009400005FC08F1FF3804460D46AAE7AFF3008026
:100950009A9999999999B93F0000F87F000024402D
:1009600070B586B014460E460022014601A82CF050
:10097000A5FF2546DDE901239A4204D3049832F00D
:10098000BDFB601B04E02DB9049832F0B7FB204694
:1009900006B070BD01A82CF04EFD013D06F8010B1C
:1009A000E8E710B586B00A46014601A82CF086FF9C
:1009B0000023DDE90112914203F1010401D2013368
:1009C0000AD1049832F09AFB202026F053FD14F14E
:1009D000FF340AD206B010BD01A82CF02CFD0A2865
:1009E000EFD026F047FD2346E3E70820EDE70000BF
:1009F00070B50D2023F066F80028264B46DB264C08
:100A00001871A17D01229A7000293DD1234DA18248
:100A100004334FF48E712846A360A275FFF7FAF8ED
:100A20002146AA60FFF725F9636893B92646A27D9F
:100A3000A38A9A420ED8A38A9BB2B3F5807F1BD0BB
:100A4000164BD3F81C21002AFBD00122DA600023C8
:100A5000A37570BDD5F81C3123B9A38A9BB2B3F539
:100A6000807FF7D1A38A9BB2B3F5807FE0D0314677
:100A70002846FFF7FEF8DAE70023A3750F210848A0
:100A8000BDE870402FF07CBA1121F8E700229A707F
:100A9000DFE700BF99B5002020AE00200020004015
:100AA0006A7E050030B58BB04FF4D823019305461C
:100AB00008B1002303602022002102A8FEF732FDC6
:100AC000002202A94FF4D82032F01AFCD0B1002441
:100AD000029B039A23F07F43033323F00303203365
:100AE00052B11C44032202A901A832F091FC002853
:100AF000EED120460BB030BD002DF3D02A68134450
:100B00002B60EFE70446F4E72DE9F04F202291B087
:100B100000244FF4D825824688460DEB020021467A
:100B2000CDE904540694FEF7FDFC012208A92846ED
:100B3000079532F0E5FBA8B905AB019306AB524629
:100B40004FF4EC21009304A8434632F0A3FE04982E
:100B5000013832F04DFC049032F0E0FE012011B07B
:100B6000BDE8F08F099B002B5DD0049E069BDDF84D
:100B70001C901E444E4523D0089B23F07F43203316
:100B80004B4401250D2702936A1E3E497A4302EB2E
:100B9000010B5846039232F023F8A8B1DBF800109D
:100BA000894508D8029B994205D2A6EB09030B445C
:100BB000039A34495350013540F6C4139D42E3D99A
:100BC00020230DEB030214E0584632F013F80028FE
:100BD000F1D0DBF800300C33B3FBF7F31D44EAE748
:100BE00012F8011B0AF804100134B4FBF8F108FBF9
:100BF000114413F1FF33F3D2069B089E2033069372
:100C0000079B26F07F46033603F1200905AB26F04B
:100C10000306019306AF009743465246494604A88F
:100C200032F038FE2EB9012208A907A832F0F0FBF5
:100C300081E7069B059AA8EB0300A8EB0405854213
:100C400028BF0546A24203D9121B954228BF15466C
:100C50000293ADB1B54228BF354649460AEB0400C0
:100C60002A4636F087FF029B2C442B440693B4FBA4
:100C7000F8F308FB134405AB761BA9440193CAE7BC
:100C800028466CE7682E002030B58BB04FF4D8248E
:100C90002022002102A80194FEF744FC002202A9B0
:100CA000204632F047FB70B1032202A901A8DDE91A
:100CB000015432F0ADFB0028F6D124F07F442335F7
:100CC0002C4424F00304C4F5EC200BB030BD00002C
:100CD000F0B40023124D0D271C4640F6C41607FB46
:100CE00003519A1CC87ACC72087B0C73C2F30B00B8
:100CF0004A79087122F00F02013342EA1022B3420E
:100D00004A71ECD147F6EB63064AEC54537823F072
:100D10000F035370044B01221A80F0BC31F0A8BFBE
:100D2000682E002053AD0020662E002037B5012329
:100D3000009300231A46054905462DF0ADFD0446F3
:100D4000284632F0DBF9204603B030BD8B7D05002C
:100D5000F8B50646437A807A000150EA13100C4633
:100D600019D031F07DFD07462DF07CFF451C38463B
:100D700032F0C4F9284631F0EDFB21462DF092F80F
:100D8000044638B1014630462EF009F8204632F0CC
:100D9000B5F9681CF8BD0125ECE7000038B5074C33
:100DA00025780023EDB202461946237030F05CFB33
:100DB00025700348BDE8384026F04ABB642E002069
:100DC00067F80500002370B50B6005460E4631F04C
:100DD0006DFC044670B129462DF0A0FE0546204664
:100DE0001DB932F08BF9284670BD2CF05FFD3060E4
:100DF0002046F6E70546F6E72DE9F843394F037933
:100E00001C2202FB03720646506820B132684FF480
:100E10000174C2F808431C2202FB0373DA7D52B14D
:100E20001A7E002A41D020B133684FF40172C3F812
:100E30000423112037E00120D875D9605A761A763C
:100E400035791C2303FB05739B7E1BB912B9304611
:100E5000FEF7E8FE4FF01C0808FB05783068D8F86C
:100E60000430002B35D14FF4A271FEF7D3FEC5EB51
:100E7000C50907EB89093068D0F82431D0F808217A
:100E8000D0F84441A2B90CB9002BF4D01C2202FBCB
:100E900005750022EA750BBB14BBA97E33680122DD
:100EA000A9B11A600020BDE8F88319610122C6E7E4
:100EB000002BEBD1002CE9D14946FEF7C3FE98F890
:100EC000193098F817209A42D5D82346DEE75A60A1
:100ED000E8E74FF40173C0F80433E3E70320E2E7E7
:100EE0000F20E0E720AE00200A490B4808B5FFF7C5
:100EF00083FF014610B109482FF042F8084906481F
:100F0000FFF77AFF014620B10648BDE808402FF000
:100F100037B808BD99B50020387C0500247E05004F
:100F20009AB50020477E050038B5002205462FF00F
:100F300066FB044650B100231A460146284623F0BA
:100F40003BFA2046BDE8384032F0D8B838BD000042
:100F5000F0B54FF080530220D3F85014D3F8542446
:100F6000284BC3F804032848C3F80403274B93F81D
:100F700000E093F801C09F78DE781D795C7998795C
:100F80004EEA0C033B4333432B4323430343204BA1
:100F90002AD083F800E083F801C09F701E715D7154
:100FA0009C71D8711D789C785A785E79586885EA6A
:100FB0000401514081F08801D970197971409E79FE
:100FC0007140DE797140197212020321597242EAAE
:100FD00005420C4B2243C3F8942500BA4422C3F8BF
:100FE0009005C3F8A025F0BD080A1970090C997086
:100FF000110A1A715971110C120E58709971DA7127
:10100000D0E700BF005000408000080094B20020EC
:101010007FB2002070B5EFF3108672B60D4A946867
:101020000123A4B993600C4B0C4DD3F880102940D8
:101030001160C3F88050D3F8841051604FF0FF3234
:10104000C3F88420047006B962B6002070BD037036
:10105000F9E700BF64B5002000E100E0FC06FFBC3A
:10106000437882781B01120202F4E06203F030033D
:101070001343027802F003021343C278120302F40E
:10108000805213430279120402F4E022134342799E
:10109000120502F4801213438279120602F0807264
:1010A0001343054AC2F81835C379017AC2F81415FA
:1010B000C2F81035704700BF0070004010B588B00E
:1010C00012788DF80C200021FF2202918DF80D205E
:1010D00001214FF6FF72104C01908DF81C10ADF8F5
:1010E0000E208DF8103022F077F970B12BF068FCEB
:1010F00058B914F1FF34F6D2084904202FF00AF849
:1011000001A822F079F908B010BD002CF4D02BF022
:1011100057FC0028F0D1F3E780841E00727D0500A3
:1011200038B50B4C0B4D2B785BB12BF049FC40B91B
:1011300014F1FF34F7D208490420BDE838402EF0FE
:10114000E9BF002CF7D02BF03BFC0028F3D138BDD1
:1011500080841E0084B50020147D0500F7B5354F4E
:10116000354C7E797601A31905465A7E002A5FD157
:10117000A2590AB101225A7695E80F0004EB060E37
:101180000EF1080C8CE80F0006F1180323445A797D
:1011900022F003025A719EF81A20FF2A1FBF012372
:1011A00093404FF0A042C2F80C352A6822B102F0F9
:1011B0006043B3F1005F06D1AB6853B103F0604305
:1011C000B3F1005F05D0344400236376102003B0F0
:1011D000F0BD3B682979C3F84425C3F848152A7B3C
:1011E000A968C3F834150020C3F83825C3F81801DE
:1011F000D3F818210192019AC3F850050122C3F8CF
:1012000040051A61A2597AB9D3F81821002AFBD0F7
:101210003444A27EFF2A05D0012393404FF0A04220
:10122000C2F808350020D2E74022C3F80423CEE7F5
:101230001120CCE7B42C002064AE0020F0B5154698
:1012400085B01C4E07460C46FFF76AFF0123FF2DB1
:1012500033702B4628BFFF231FB3FA1816490A60C4
:101260000CB3E218154900970A60154A0294002C45
:10127000A5EB0305DBB21560684614BF1A460022D1
:101280008DF80C208DF80430FFF768FF024660B13E
:10129000002404200B4934702EF03CFF204605B09A
:1012A000F0BD3A46DAE72246DCE7FFF739FF0120D6
:1012B000F5E700BF84B5002088B5002080B5002088
:1012C00078B50020017D050013B51A4B1B78044644
:1012D00063B3FFF725FF184B1B6800220120042190
:1012E000C3F80025C3F80005C3F80813C3F80821A4
:1012F000D3F80811009100991049E4B20870C3F8BE
:101300001C45D3F808010028FBD0C3F80821D3F806
:10131000080101900198D3F818050A70C3F8002558
:101320000722C0B2C3F8002502B010BD4FF0FF3055
:10133000FAE700BF7CB50020B42C002084B5002063
:1013400037B50B015BB249B2044643EA01008DF8A0
:1013500004001A4D50B20343120152B28DF8053009
:101360002B78114302438DF806108DF8072013B334
:1013700002AB03EB941302AA13F8040CC4F3011399
:10138000134413F8043C43EA002019F097FD2B782E
:101390008BB102AAC4F3810304F003041344144480
:1013A00013F8040C14F8043C43EA002003B0BDE831
:1013B000304019F083BD03B030BD00BF7CB50020C4
:1013C000C30914BF13020B0210F0400F70B506469C
:1013D00014BF10460846184314460D46FFF774FF25
:1013E000B1064CBF23022B0216F0100F14BF20468B
:1013F00028461843FFF768FF32074CBF23022B0231
:1014000016F0040F14BF204628461843FFF75CFF70
:10141000B3074CBF2002280216F0010F08BF2C466C
:101420002043BDE87040FFF74FBF000020292DE9A1
:10143000F0470BD9244A254E2139C9B2002314465E
:10144000DFB2B94205D814F801C0B6BB4008BDE808
:10145000F08712F8017B01333E44F1E7745CC82C3D
:101460001ED81EF80450DFF86C90194B4FF000089E
:101470005FFA88FA54450DD803EB0509994511D157
:1014800001316145EADB0232504320F07040073001
:101490000009DCE719F801AB08F101085344E7E75C
:1014A0000023E9E713F8018BB8FBF7F407FB14847A
:1014B000E4B2A242B8BF2246E0E700210A46DFF8C4
:1014C00014E00D27DDE700BF8B7E05006A7F050075
:1014D0008E810500C580050010B5074A002332F84B
:1014E000024B8C4203D1184100F0010010BD0133C2
:1014F000082BF4D10020F9E768AD0020F0B5224BAD
:101500009F7C1C4600221D46D6B2B7420ED895F8E5
:1015100078701D4C0022D6B2B74216D895F8DE502E
:101520000022D4B2A54220D800200DE0B4F814C0A7
:10153000844502F1010204F10A04E5D142F64D238B
:1015400001200B808870CE70F0BDB4F87AC0604581
:1015500002F1010204F10A04DDD142F64D230B80B1
:1015600002238B70CE700120EEE7B3F8E060B0424A
:1015700002F1010203F10A03D3D142F64D230B809D
:1015800003238B70CC70EEE7F0AF002010B50C4C4D
:10159000226886B0034682B104208DF804000868F2
:1015A000D989ADF80C10123333F8021C0290ADF853
:1015B0000E10049301A92046904706B010BD00BF4D
:1015C000F0AF00207FB54B89022B0FD1094A136879
:1015D00063B1097B0068029011F0010F14BF022172
:1015E00003218DF80410104601A9984707B05DF853
:1015F00004FB00BFF0AF002070B50D4D002435F89E
:10160000026B964210D10122A240D2B2D543EDB274
:10161000014410F8014B2BB11443884200F8014CEF
:10162000F7D170BD2C40F8E70134082CE7D1F8E77A
:1016300068AD002070B50023084C1A4641FA02F547
:10164000ED0706D504EB420600EB4305B688AE80F5
:1016500001330132082AF1D1036070BD64AD00206E
:1016600010B586B004460022684616F0A1FD20465B
:10167000009916F0CBFE204606B010BD38B5012308
:101680000B7004460D4631F045FA88B100220B4933
:1016900020462EF0B4FF10B12EF0B6F92870204687
:1016A000002207492EF0ABFFBDE838402EF05EB8AF
:1016B0002046BDE838402DF0D5BA00BFF47C0500C7
:1016C000F97C05002DE9F04F2DED028B8DB0436ABA
:1016D000059390ED048B1F02836A07671E0246671D
:1016E000B0EE480AF0EE680A0446069333F0A4FB15
:1016F00059EC108BB0EE480AF0EE680A33F08CFC1F
:1017000094ED067B404653EC172B49465BEC10AB3F
:101710008DED007B35F044FE0022614B35F016FD67
:101720000022604B35F05CFB35F0C0FFDDE90023A3
:101730000790A0675946504635F032FE0022584BBC
:1017400035F004FD0022574B35F04AFB35F0AEFF73
:10175000E0670546059835F08FFC29F00043CDE998
:1017600008010698CDF80880039335F085FCDDE983
:101770000223CDE90A01DDE9080135F0E7FCD04696
:101780002BF0004942468B464B468246DDE90A0172
:1017900035F0DCFC02460B465046594635F020FB3E
:1017A000DDE9002335F0D2FC00223E4B35F018FB7A
:1017B00035F07CFF42464B468346DDE9080135F0B3
:1017C000C5FCDDE90A2380468946DDE9020135F0E2
:1017D000BDFC02460B464046494635F001FBDDE9BB
:1017E000002335F0B3FC2F4B002235F0F9FA35F029
:1017F0005DFF94F820305BB1226863680BEBDB710E
:10180000A2EB6102226000EBD072A3EB6203636083
:101810002368059A5B44A36063680344E360079B05
:101820000BFB03F3013300FB053303EBD373D2014E
:10183000A2EB6303C4F88030079B58430130069B3A
:101840000BFB150505EBD575D80194F82130A0EBFD
:101850006505C4F884503BB90DB0BDEC028BBDE802
:10186000F08F3B44C4F88030D4F88030002BF8DB94
:10187000D4F880309F420BDDD4F88430002B0BDB92
:10188000D4F884309E42E7DC9B1BC4F88430F7E731
:10189000DB1BC4F88030EBE73344C4F88430EBE75B
:1018A000000070400000E03F1F4B204A1B6800BF53
:1018B00000BF00BF00BF00BF00BF00BF00BF93421A
:1018C0002FD000BF00BF00BF00BF00BF00BF00BFE0
:1018D00000BF00BF00BF00BF00BF00BF00BF00BF10
:1018E00000BF00BF00BF00BF00BF00BF00BF00BF00
:1018F00000BF00BF00BF00BF00BF00BF00BF00BFF0
:1019000000BF00BF00BF00BF00BF00BF00BF00BFDF
:1019100000BF00BF00BF00BF00BF00BF00BF00BFCF
:1019200000BF0138C3D17047A42C00200024F4006C
:1019300008B1FFF7B9BF7047084B5A6E013A5A66B3
:1019400022B907490A7822F002020A701A6E01329F
:10195000042A08BF00221A66704700BFC0B30020E7
:10196000E2AF002030B5044685B00D4610220021BC
:101970006846FDF7D7FD237A012B0AD0022B0ED043
:1019800063680193236829469B686846984705B0B9
:1019900030BD23690293A38AADF80C30F0E7012330
:1019A000A2898DF80030E389ADF80A20D31AADF88A
:1019B0000830E5E728DF704729DF704738B51C4B52
:1019C0005A6E19465AB31C6E182202FB04331A7A57
:1019D000012A07D0022A23D018460921BDE8384041
:1019E000FFF7C0BF1825D88A9A8A05FB0414D4E9EA
:1019F0000314121AB2F5806F4FEA80000144B4BF9D
:101A000092B24FF480622044FFF7D6FF11280BD129
:101A1000084A137823F0020343F00403137038BD1F
:101A20009889FFF7C7FFF1E70028F8D0D4E700BF97
:101A3000C0B30020E2AF0020054A137813F0060F70
:101A400004D143F002031370FFF7B8BF704700BF23
:101A5000E2AF00202DE9F3411F4B1B781746DA0750
:101A6000064688462BD51D4D1D4B9D4229D31D4B47
:101A70009D4226D239B330B341EA00039B0724D1FB
:101A80002B68984223D36A6800EB87039A421ED3DF
:101A9000FFB101A8FEF7DEFC78B1019B0024C3E989
:101AA0000054019B01221A72C3E903869F82FFF74B
:101AB000C3FF204602B0BDE8F0810720FAE701200D
:101AC000F8E70220F6E70320F4E70620F2E7052016
:101AD000F0E70420EEE700BFE2AF00200C2E00206C
:101AE0000C2E00201C2E002038B5074B074A5968E1
:101AF000948810684A880332032592B200EB840070
:101B00001D70FFF7A7FF38BDE4AF002064B40020CC
:101B100010B501220C460649FFF79CFF28B905497C
:101B200001EB041101238B7310BD0E20FCE700BFF5
:101B3000A87D050020B3002008B502220149FFF767
:101B400089FF08BDAC7D050008B5034B0349186843
:101B50000222FFF77FFF08BD64B40020B47D0500BA
:101B600073B51B4B1B78DB0705462BD5194E1A4B5B
:101B70009E4229D3194B9E4226D238B3C0F30B04A0
:101B8000D4B93368984219D3726800F580539A42E9
:101B900014D301A8FEF75EFC90B1019BC3E9006479
:101BA000019B02221A722D0B01229D811A82FFF7DE
:101BB00043FF204602B070BD0620FBE70520F9E791
:101BC0000720F7E70120F5E70220F3E70320F1E71C
:101BD000E2AF00200C2E00200C2E00201C2E002036
:101BE00010B50B4C0B4B628803EB02139A892AB990
:101BF0005868FFF7B5FF0423237010BD0523237039
:101C0000054B022218689A80FFF7AAFFF5E700BF8C
:101C1000E4AF002020B3002064B4002008B5074BD7
:101C2000191D5888FDF7D6FC18B1BDE80840FFF72C
:101C30005BBFBDE80840FFF7D3BF00BFE4AF0020A3
:101C400010DF7047002208B5114619F013F90000A3
:101C50002DE9F347254B1B681BB1984730B3FFF7BD
:101C6000F1FF234B1B7803F0FF07FBB1214D224E00
:101C70002C68DFF88C90B4FA84F46409B0463378A9
:101C8000A3B901A8FDF78AFC052812D00028E6D1E7
:101C9000019B0BB9FDF75EFE184B1B680BB1019859
:101CA00098474CB10124EAE7002CFBD002B0BDE814
:101CB000F087002CFAD13C46DFF848A098F80030B5
:101CC000002BF3D1B9F80030ADF80430DAF8003069
:101CD00001A91846FDF760FC0528E5D00028BED113
:101CE0002A6818469047002CE8D1C8E7D0AF0020FA
:101CF00061B400209CAD002062B400206CB40020D0
:101D000098AD00205CB5002010B5084B9A685AB118
:101D100050B9EFF3108172B6054A1C6814605C6814
:101D20005460986001B962B6002010BD64B500200F
:101D300000E100E02DE9F3411D4F7B6806460D46AA
:101D40009BB304292FD943697BB3437C0024012B27
:101D50000DF107000CBF8846A0468DF80740FFF73D
:101D600059F90DF10600FDF7C3FCD0B10123037052
:101D7000104B4660D3F80435C0E90484C0E902354D
:101D80009DF806307B709DF80700FFF7BDFF24B972
:101D9000094B4FF48012C3F80021204602B0BDE881
:101DA000F0810424EFE70724F7E70824F5E700BFF4
:101DB0009CB200200010014000E100E02DE9F34159
:101DC000CE0801F007044FF0010808FA04F4855D1D
:101DD000E4B22540074613D10DF107008DF80750F6
:101DE000FFF718F9BB5D9DF807001C4202BF1C43BA
:101DF000BC554546FFF788FF284602B0BDE8F08194
:101E00000025F9E72DE9F3478146002701261FFA4F
:101E100087F84FEAD80A08F0070406FA04F419F81C
:101E20000A50E4B2254008D00137B7F5807FEED1E3
:101E3000B846404602B0BDE8F0870DF107008DF8C6
:101E40000750FFF7E7F819F80A309DF807001C4221
:101E500002BF1C4309F80A400125FFF755FF002D7A
:101E6000E2D0E6E773B50546B8B1C1F3C70401F0A7
:101E7000070301269E40035D33420ED000230DF17F
:101E800007008DF80730FFF7C5F82B5D9DF80700B8
:101E900023EA06062E55FFF737FF02B070BD00009B
:101EA00038B50A4B1A687AB15D686DB1FF280BD05E
:101EB00084B221462846FDF7BFFC28B121462846BA
:101EC000BDE83840FFF7CEBF38BD00BFACB400203E
:101ED0002DE9F74F9846531E072B81460F461546AE
:101EE00000F2BB80FF2800F2B88001465E48FDF793
:101EF000A3FC0646002800F0B08039464846FDF7AE
:101F00005BFC044600283ED0C3689D4247D805D2FA
:101F10005FFA85F9E368207C994543D394F81090E3
:101F2000B9F1FF0F40F09780504B1A689B46002A8A
:101F300041D14FF6FF732380A3700023C4E901331E
:101F4000E360238A03F4784343F0FF0323821120E4
:101F500084E0237C1844C0B2FFF7A2FFE3685FFA75
:101F60008AF083420AF1010AF3D84FF6FF73238007
:101F7000A3700023C4E90133E360238A03F47843A8
:101F800043F0FF032382FF214FF6FF70FDF714FC9F
:101F900004460028DBD0A0F800908770BEE74FF021
:101FA000000ADBE74844C0B209F10109FFF778FFF6
:101FB0005FFA89F9AEE75B68002BBAD00023DBF843
:101FC00008205FFA83FA924502D34FF0FF0912E02E
:101FD000DBF8040060B351460193FFF7EFFE019B6D
:101FE00030B3B9F1FF0F08BFD146AAEB090A0AF1D5
:101FF000010AAA4521D1B9F1FF0F84F8109098D0B9
:10200000E560207CFDF728FC58B305EB85052D0124
:10201000ADB2AD0888F80270C8F80400A8F8005006
:1020200026B1082F02D1AD00063D8580002015E0C5
:10203000B9F1FF0F0CD14FF0FF090133BFE748465C
:10204000019309F10109FFF72BFF019B5FFA89F961
:10205000D145F4D3EFE70026D2E7072003B0BDE86F
:10206000F08F0320FAE700BF78B30020ACB4002063
:1020700038B504460025E368AB420ED84FF6FF732F
:102080002380A3700023C4E90133E360238A03F4AF
:10209000784343F0FF03238238BD207C2844C0B23C
:1020A000FFF7FEFE0135E6E737B5FDF785FB054690
:1020B000A0B144682CB10A4B01941B789B0706D44D
:1020C00003242846FFF7D4FF204603B030BD01A803
:1020D000FDF766FA04460028F3D0F1E70524F3E79C
:1020E000E1AF0020FF2810B5044609D80146054895
:1020F000FFF7B8FE21460448BDE81040FFF7B2BE26
:1021000010BD00BF78B3002098B3002013B50DF1C7
:1021100006010446FDF786FA70B1BDF80620084BAB
:1021200003EB02139A894AB1A17A39B1013A00202E
:102130009A81A07202B010BD0A20FBE70620F9E7E1
:1021400020B3002037B50D460DF106010446FDF71A
:1021500069FA88B1BDF80620084B616803EB0213E9
:1021600000209A8901329A81296063680C336B6080
:102170000123A37203B030BD0A20FBE720B3002087
:102180002DE9F043DFF88480D8F874E0BEF1030F46
:102190000F46944635D81C4E756CC1F108039D421C
:1021A0002FD8D8F8704074441C2304F003048146EF
:1021B00003FB0484B9E80F000FC499E807000EF18F
:1021C000010384E80700C8F87430C7B1336C2B44AE
:1021D00003F0070306EBC303002206F138040CEBFF
:1021E000C20103C9A34202F1010283E8030014BF44
:1021F0000833054B9742F2D1736C1F44776401207A
:1022000000E00020BDE8F083A8AE0020A4B20020CA
:102210002DE9F0411C46184B1B789B0706460F46DC
:10222000154627D5DFF85880A3880BB10A201FE098
:1022300098F800302BB92146A088FDF7CBF920B9DA
:102240002060A3880133A380EEE723681EB199883C
:1022500032889142EFD11FB119883A889142EAD170
:102260009B682B6023686B60044B1B892B810020CB
:10227000BDE8F0810220FBE7E1AF0020E4AF0020E1
:1022800020B3002030B587B04CF2070305460C465A
:10229000ADF8043003AA0F4B01A90020FFF7B8FFE7
:1022A00010B1002007B030BD01A903A8FFF74AFF15
:1022B0000028F6D10723A370019B5A882280029A36
:1022C00062609B8803F580432B8003A8FFF71EFF05
:1022D0000120E7E7D4AF00201FB50023A0F5804020
:1022E000A1F58041CDE90233ADF80400ADF8061048
:1022F00002AB0DF1060101A8FFF78AFF002818BF05
:10230000052005B05DF804FB2DE9F04102230B80A8
:10231000164B00251C6800F5805E2F4608304FF6EE
:10232000FF7870450AD305B11C6002B11770BDE893
:10233000F08101270EE0344601250BE006680136E6
:10234000F1D086884645F4D00688002EF1D0866804
:10235000A642F0D8468806F1030C00EB8C00B1F8D9
:1023600000C00CF1030C66440E80DAE76CB100206B
:1023700070B5064D0646002455F8043B0BB13046B7
:1023800098470134082CF7D170BD00BF84AE0020FF
:102390002DE9F047AA4C266F1C2707FB06F586B0EF
:1023A000635D013B8046052B00F22A81DFE813F0D4
:1023B0000600640064001D011D017E0130B1A14AC8
:1023C000137823F00103137001201FE025442B79BB
:1023D000032B15D8DFE803F002072C34FFF7B4FB1A
:1023E00001232B7109E0984D2B78022B40F03C82A1
:1023F0006868FFF7A1FB00232B70002800F0F08035
:10240000904A137823F0010313700E201C237343AA
:10241000E218E35C0290023B012B00F232818B4B0D
:10242000907D196C5A6C0144121A19645A6428E19F
:10243000874F3868FFF794FB0223BB800023D0E767
:10244000834FDFF804823868FFF776FB814BD7F8BB
:1024500000E05B88B7F804C01B0108EB0302516879
:10246000A2F808C0C2F804E00222BA800022396053
:1024700008F803202A71C0E707FB0647724BB7F83C
:1024800012A04FEA0A1A03EB0A029946118960B1B9
:10249000FB8803F103088844C3F57F435189A2F800
:1024A0000880FD330B4453818EE7536803EB8108AA
:1024B0003B7C062B00F29780DFE803F02D733C4D48
:1024C0001F84040041F61D501C2303FB0643D14426
:1024D000DB88B9F80810DA1C0A44A9F80820C3F50B
:1024E0007F43B9F80A20FD331344A9F80A3041F6B6
:1024F0001D53984200F0C38088E75748574900238E
:1025000043601C2303FB06439B690360FDF78AF8C5
:10251000002800F04C81291D012221444046FFF78C
:1025200099FA1C2303FB064302221A74002857D091
:102530000E20C9E705F10C010122214408F1080031
:10254000FFF788FA1C2303FB06439A7D002A14BF79
:1025500003220122E9E73D4B5A6C002A00F08C81EE
:10256000196C1C2505FB0645481C00F0070003EB11
:10257000C1071864A88A53F83110013A5A6408EB6D
:102580008000BA88FFF766FAAB8ABA881344AB8238
:10259000AB7D013BDBB2AB75002BC7D101232B74A4
:1025A000C4E705F108010122214408F10400FFF706
:1025B00051FA1C237343E25C032A0CBF0522062256
:1025C0002344B2E7254B1988234B5868FFF7A0FA3C
:1025D0001C2303FB064306221A7400287FF474AF01
:1025E00006B0BDE8F0870F206EE700287FF4ECAE60
:1025F00007FB06473B79012B32D01BB1022B3ED0A3
:102600000F2003E7CDE90200FB6801930DF1020101
:1026100001A8FDF707F880B10298BDF80210838881
:10262000FB8003883B81FFF773FA1C2303FB0643FF
:1026300002221A710028D3D059E70A20F5E700BF1B
:10264000A4B20020E1AF002020B30020A8AE0020FB
:1026500064B40020E4AF00203C2E002070B50020C0
:10266000864FA81D3B4601AA41462044FFF7D0FDF6
:10267000B8B9B9880298FFF74BFA0A28DAD10023D3
:1026800002931C2303FB06F2A25C013A052A00F226
:10269000B580DFE812F08E009200A000CB00D500DC
:1026A000E1000A28C7E90088E9D020E700287FF484
:1026B0008BAE734BDA7AAAB1D8721A78013A062A2D
:1026C0009ED801A151F822F0792702007327020059
:1026D000892702008F2702000126020095270200A9
:1026E000A52702001A78072AE7D801A151F822F09D
:1026F00011270200BB260200BB2602002D27020084
:10270000412702005F2702005F27020029270200FD
:102710001A8901321A8100225A80DA72594A1278D3
:10272000B2FA82F252099A72012207E056495868B9
:102730008A884088033202448A8002221A70BCE7E9
:102740005D88504A504902EB051208685568506090
:102750008888108102228A800D600622EEE7072217
:10276000ECE7484900229A728A8942B9897B31B1E3
:102770005A80FFF753FA5DE79A7A002AF1D10022D6
:102780001A705A805A607AE7FFF7AEF952E7FFF7FE
:1027900027FA4FE75A883B4B03EB02135868FFF7C1
:1027A000CBF947E700225A60FFF7CEF942E70A204B
:1027B0002CE600238DF8043020E003FB06430122C1
:1027C0008DF804201A89ADF810209A88ADF81220EF
:1027D000DB68039312E003FB064302228DF804201A
:1027E0001A89ADF810209A88ADF81220DA681B7C9F
:1027F00003929A1F534253418DF8143001A8FFF7FA
:10280000B7FD206F1C22002102FB0040FCF78AFE6E
:10281000636F1BB3226F013202F00302013B226798
:102820006367DBB10020FFF7B3FDD9E603FB064386
:1028300003228DF80420DA88ADF810201A89C5E744
:1028400003FB06430422DB88ADF8103000238DF82B
:102850000420ADF81230D1E70523ABE70B4A13781B
:1028600023F004031370BBE6084A137843F0020315
:1028700023F00103137002E71368FFDE90B5002018
:10288000E4AF002020B3002064B40020E1AF0020BA
:102890000846FFF77DBD0000054A137813F00400D9
:1028A00004D143F004031370FFF772BD704700BFFB
:1028B000E1AF0020F0B51C463D4B1B789E0789B068
:1028C00007460D466FD509884FF6FF7399426CD0C5
:1028D0006B88002B69D06968B5F808C000239C4557
:1028E00003D8BAB9164604310AE051F8330080071C
:1028F00057D10133F3E731F83200304486B2013268
:102900009445F8D80DF102013046FCF7D3FE28B10A
:1029100009B0F0BD13885688ADF8023000238DF859
:102920001430BDF80230ADF816300323ADF818307E
:10293000204B8DF804401A6829898DF81A1001324D
:102940001A602B88ADF80C30032C6B88ADF808307A
:1029500004BF04238DF81430049208BF3B686A68F2
:1029600008BF0793002401A8ADF80A60ADF80E4037
:10297000FFF706FC50B9BDF802200F4B03EB021322
:1029800058890338801B58810820C1E7049B3B60AD
:102990000A4B7C601B89BC723B81FFF77DFF2046A0
:1029A000B6E70320B4E70220B2E70420B0E700BF97
:1029B000E1AF00206CB1002020B30020E4AF002084
:1029C00030B58BB0FF28044601921D4645D88B7860
:1029D0001846FCF7C7FE00283FD04A6802920A88D2
:1029E000ADF80C20A4F58042ADF81C20A3F5804280
:1029F000ADF81E2002AA08920122ADF82420194643
:102A000004AA2046FFF768FC0528019A0ED102238C
:102A100052B907A904A8FFF74DFF07281FD010D807
:102A2000B0B103200BB030BD01AAF2E732B10E4BBA
:102A30001B789B0702D501A8FCF7B2FD03230022F7
:102A4000E7E708280DD00E280CBF11200320E9E786
:102A5000002DE7D0049B2B60E4E70720E2E7862007
:102A6000E0E71120DEE700BFE1AF002073B5154EAF
:102A7000736805461BB343690BB3002404740DF15E
:102A800007008DF80740FEF7C5FA0DF10600FCF7C8
:102A90002FFE90B1022303709DF8063045607370DD
:102AA0009DF80700FFF730F924B9074B4FF4801267
:102AB000C3F80021204602B070BD0424F0E70824CA
:102AC000F8E700BF9CB2002000E100E02DE9F843E8
:102AD0002649274B0025C1F84051C1F84451C1F89F
:102AE0004851C1F84C51C1F80051C1F804511B685C
:102AF000002B39D0D1F804451E49DFF88C800968D5
:102B0000641A24F07F442F461A68A24217D8A41AE8
:102B100015441A7CDE6982B1D8F800901F74D3E99D
:102B20000521B9F1000F06D01046C84728B1FFF7BC
:102B300089F83346E8E708469047002EF9D10E4A57
:102B40000E4B11781B788B4205D10133DBB2022B7F
:102B500008BF002313701278094B43F82250094B29
:102B60004FF48012C3F80021BDE8F8830010014043
:102B700060B500207CB4002079B4002078B4002037
:102B800070B4002000E100E0CCAF00200D4B0E49F6
:102B90004FF4003210B5C3F8802001244FF4803385
:102BA000C1F848332F20C1F808334C60FEF77CFE93
:102BB000064B8C602F2000211960FEF775FE044B38
:102BC000197010BD00E100E0001001407CB400204D
:102BD00059B400202DE9F04FB64AB7491378097867
:102BE000B64D85B09942D5F80080019500F09580EA
:102BF0000133DBB2022B08BF002313701278B04BF5
:102C000053F82260019A08EB060323F07F43136018
:102C10000127AC4BAC4A18680290AC48117890F888
:102C200000904FF0000CE2465078884278D1BCF119
:102C3000000F02D0A54981F80090002F40F0BB8022
:102C40001F6802997F1A18BF012700201968029196
:102C50009E49039191F800E000244FF001080028FC
:102C600040F0AD8092F80190D2F804C092F802A032
:102C70001178494540F0C1801B68029A9A4201D1FF
:102C8000002F44D0002B00F01281D3F80090904C1C
:102C9000019BD4F8046519688E4F751A3B7825F0AE
:102CA0007F450335A3B94FF48033C4F84433C4F8E7
:102CB0000433894B4FF400324FF00108C3F88021F0
:102CC0002F201A60C4F80080FEF7EEFD87F8008020
:102CD000A9452CBF4944491921F07F41C4F840154A
:102CE000D4F804359B1B23F07F43891B033321F069
:102CF0007F418B420BD9D4F80435C4F840352F20DE
:102D0000FEF7D2FD744B4FF40032C3F80021039A52
:102D10000023137005B0BDE8F08F0026374678E732
:102D200001EB4104506892F802B000EBC40E01318F
:102D300010F834401868C9B28B4508BF0021022C36
:102D400004D0032C7FF470AF002410E0DEF804B050
:102D500004468646002C3FF467AFA34500F0C080D0
:102D6000A646E469F6E780F810A0C06901240028AF
:102D7000F9D1002C3FF458AF186055E7D4F80C9007
:102D8000C4F800E0761A8C44E1691960B9F1000FCB
:102D900007D008EB0C0121F07F41C4E90119E06183
:102DA00020461C68002C3FF451AF2168B142E5D9A0
:102DB0008E1B26604AE7002084468646F1E70146DE
:102DC000C069019DD1F804A02E68444DD1F8089047
:102DD000AAEB060C2CF07F4CAC4535D80CEB090661
:102DE0000E60D3F800C081F81080C1E90144CC61C5
:102DF000BCF1000F33D1196031E701EB410B013118
:102E0000C9B2514514BF117014701CF83B10012950
:102E10000CEBCB067FF42CAF716891F810B0BBF1CE
:102E2000000F7FF425AFD6F808C0C1F804C0F568DC
:102E30008D603569CD6076698E61BEF1000F0CBF83
:102E400066465E464E60BCE7A6EB0A0626F07F4665
:102E50004E4502D2A9EB0606C2E70C60C1E7D1F8E5
:102E60000090DCF80060B1451FD8A6EB0906CCF84D
:102E70000060C1F81CC0BEE7A9EB0A09D6F81CA087
:102E8000B446BAF1000F0AD05646D6F800A0CA459B
:102E9000F2D3AAEB090AC6F800A0B2466646C1F80A
:102EA0000090C1F81CA0F161D9E66646EDE7FFF796
:102EB0006DFE2CE778B4002079B400207CB40020AB
:102EC00070B4002060B500209CB2002058B40020EF
:102ED0000010014059B4002000E100E0FEFF7F0037
:102EE00074450FD1D0F81CB0C3F800B0BBF1000F8F
:102EF00008D10A4D0120A86001984FF0010CC0F8DC
:102F000000B0E1462068E469CEF81C40002C3FF494
:102F10008BAE25682844206086E600BF0010014083
:102F200037B5074B054693E803006C46002384E859
:102F300003001A4621462846FFF742FD03B030BD84
:102F4000147C0500FDF7A2BA10B54FF6FF730446D6
:102F50009C42084609D1FEF755FFB0F5807F044634
:102F600001D14FF6FF74204610BDFF2CF9D8214641
:102F7000FEF724FF0028F6D1F3E710B5044601F070
:102F8000EFFC2046BDE8104000F02EBF1FB50378CF
:102F900093B90279072A0FD1448803932046CDE9DB
:102FA00001338DF80420FCF7C7FBADF8060001A83B
:102FB000ADF80840FFF7E1FF04B010BD1FB50023D6
:102FC000CDE901330393ADF80600022301A88DF883
:102FD00004308DF80810FFF7D0FF05B05DF804FB52
:102FE00086DF704738B504884CB9821C00F10A05A9
:102FF00012F8013B1BB99542FAD100200AE00B8878
:10300000A342FAD108220231023034F0A5FDB0FA11
:1030100080F0400938BD08B570B171B103780A7805
:10302000534013F0FE0F08D106220131013034F075
:1030300093FDB0FA80F0400908BD0020FCE710B510
:10304000044600F0BDFF2046BDE8104000F04ABF36
:1030500043DF70476FDF7047024B0022C3E9002255
:10306000704700BFD4AF0020F0B5FF2887B00446FA
:103070000E4615461F4629D80846FCF773FB28B3B1
:1030800003AA2046FFF728F918B10524204607B007
:10309000F0BD01A903A8FFF755F804460028F4D1B4
:1030A000019BAE705A882A805FB13B6892009A42B9
:1030B0000AD30299686834F05DFD03A8FFF726F88B
:1030C000E4E7029B6B60F8E70424DFE70724DDE711
:1030D0002DE9F041CEB020AE502380460CADB82291
:1030E0000021304601930395FCF71CFA0DF197037C
:1030F00005930DF1AE0306930DF1C503079337ABAE
:1031000008930DF1F30309930DF585730A931C4F92
:1031100004960DF221130B930024444507D1E2B22B
:10312000002104A8FFF796FF4EB0BDE8F0815022C1
:1031300000212846FCF7F6F901AB02AA072137F86F
:10314000020BFFF791FF20F002000528ECD06B7C0A
:10315000032B12D817230DF1310203FB04630DF189
:10316000450152F8040B43F8040B8A42F9D1118847
:10317000198092789A700134CFE743F20220D3E7A6
:103180008AB400202DE9F04110220546A6B00021A6
:103190002D48FCF7C7F935B929462846FCF7E0FA6F
:1031A00026B0BDE8F0816A0028492748DFF89C80F6
:1031B00004AE34F0DFFC382200213046FCF7B2F9CF
:1031C00000245023CDE9013412AF0397502200218F
:1031D0003846FCF7A7F901AB02AA072138F8020B21
:1031E000FFF742FF20F002000528D9D09DF85930A2
:1031F000032B26D8C4EBC402B318DDF85910B15024
:103200000134BDF85D209A80A5429DF85F209A7137
:10321000DCD10DF1170313930DF11E0314930DF17F
:10322000250315930BAB16930DF1330317930DF193
:103230003A0318930DF1410312961993E9B23846F7
:10324000ACE743F20220ABE79AB400208AB4002036
:103250002DE9F043037889B00546002B3FD1017971
:1032600007293CD104AA4088FFF7FEFEB8BBFFF750
:10327000F3FE02A90DF10600FFF704F878B36E889B
:10328000BDF80670BE42F4D0059C631C184611348C
:1032900013F8012B12B9A342FAD1EAE7DDF80C804A
:1032A000102208F1010134F057FC08F111018146A8
:1032B0002046FFF7B0FEB9F1000F01D00028D8D0AA
:1032C0003046FCF739FA0023ADF81A0006A88DF84D
:1032D0001830ADF81C60ADF81E70FFF7B0FE09B0F5
:1032E000BDE8F083CA1F012A73B5064654D80025ED
:1032F000CDE900558DF80210FCF75EFA044600286F
:103300004CD0437CDB074BD4007CFCF7A5FA10B90A
:10331000032002B070BDE368019003EB83031B013F
:103320009BB29B086846ADF80030FCF723FA626850
:1033300004F1080369463046FFF742FB637C03F063
:103340000603062B01BF174A136803F1FF3313600E
:1033500030B9637C23F0070343F001036374D8E7BB
:1033600011280BD10F4A136801331360637C23F0DB
:10337000060343F0040363740020CAE7862809D1DA
:10338000084A136801331360637C23F0060343F09B
:103390000203E3E70728BBD10720BAE70520B8E717
:1033A0002846B6E774B100202DE9FF4105461022FA
:1033B00000216846FCF7B6F868882979ADF8020064
:1033C0008DF80410FCF7F8F92B78454E092B5ED8E0
:1033D000DFE803F00505684D4D6C7173757D0028BD
:1033E0003FD0437CDC073CD5FEF742FE2B78581ECD
:1033F00043424341002468468DF800408DF8083070
:10340000FCF7CCF933684BB3364E002537464FF006
:10341000140808FB05735B7C5A0703D49B0759D536
:10342000002C57D0B1783088FFF75CFF002851D0CE
:1034300014235D437B1986289B788DF804307A5BD2
:1034400016BF0290082309236846ADF802200CBF7E
:103450008DF800308DF80030FCF7A0F904B0BDE81D
:10346000F08101238DF80030AB68029316E080B143
:103470008268AB689A420CD1437CD90709D532687F
:1034800023F00503013243F0040332604374002447
:10349000B8E702238DF80030EB6803936846FCF729
:1034A0007DF9F4E703238DF80030F7E704238DF866
:1034B0000030EB68D9E70523F5E70623F7E7072394
:1034C00068468DF800300124FCF768F99AE7EB684C
:1034D0000293DCE70135082D06F1140699D1BDE70A
:1034E00074B10020BCB4002070B500238CB02D490D
:1034F0002C4E4FF6FF70CDE90033FCF711FA4FF672
:10350000FF750446AC420BD0A4F58043ADF81430EF
:1035100002AA6B46002105A8FEF77AFE0A2822D0EF
:10352000214B1A781846E2B94FF6FF718C4218D039
:103530001E4E367801251D70B607A4F580439BB258
:103540001DD58B422CD005218DF8141005A81146ED
:103550008DF81850ADF81A30FEF712FE60B1FFF783
:103560009BF90CB070BD2046FEF7BCFD20463146ED
:10357000FCF7D6F90446C5E70D4B1D70F1E70223B1
:103580000022092102708DF8141005A8FF21ADF862
:1035900016408DF81810CDE90723FFF705FFE0E787
:1035A0000423EDE798B3002031B30020E1AF002001
:1035B00032B30020F0B5426805783D4C85B0B2FAD0
:1035C00082F149090391691E0346042924D8DFE8E2
:1035D00001F0030330496A009989DE8901F58041D1
:1035E00089B243F6FE77B94204D906F5804080B22D
:1035F000B84211D8012DADF802108DF8046013D136
:10360000002A14BF032100218DF8001003929B684B
:1036100002936846FFF7C8FE23781BB1002323708E
:10362000FFF762FF05B0F0BD002A14BF042101219D
:10363000EAE79989DD8901F5804189B243F6FE7692
:10364000B14204D905F5804080B2B042E4D8002AE6
:103650000CBF02220522ADF802108DF804508DF83F
:103660000020D4E7988900F5804080B243F6FE71CF
:103670008842D1D8DB89002BCED1FF23ADF80200E0
:103680008DF804305AB906238DF80030FEF72AFD74
:10369000084A002323701370FFF726FFB9E70723BA
:1036A0008DF80030F4E708238DF80030B1E700BF53
:1036B00032B3002031B30020F8B50D490D4DFCF7B1
:1036C0002FF94FF6FF760446A5F12007B44201D149
:1036D0002046F8BDFF2CFBD821462846FCF7ACF865
:1036E0000028F5D020463946FCF71AF90446EDE7E4
:1036F00078B3002098B3002073B5104B104C93E8BA
:1037000003006D46002385E803001A4629462088F9
:10371000FFF756F94FF6FF762388B34201D0112800
:1037200001D102B070BD1846FFF7C6FF00231A464C
:1037300029462080FFF744F9EEE700BF1C7C050016
:10374000BCAF00201FB50378012B044615D10179C9
:10375000012912D1002302AA4088FFF785FC60B935
:1037600002238DF800306388ADF80230039B684671
:103770001B788DF8043000F0B5FD054B1A884FF624
:10378000FF739A4201D0FFF7B7FF04B010BD00BF2E
:10379000BCAF002070B504468AB0142200216846F0
:1037A000FBF7C0FE6588ADF804502846FBF7C4FF60
:1037B0002378ADF80200092B15D8DFE803F00516D1
:1037C0003048525E8614A1A507238DF80030237976
:1037D0008DF808309DF80A3043F001038DF80A3067
:1037E0006846FCF70FF80AB070BD07238DF800306B
:1037F00023798DF808309DF80A30444AA168039176
:1038000043F001038DF80A301368002BE8D0994289
:10381000E6D1002313603E4A03931580E0E70823B6
:103820008DF8003023798DF80830E3680493374B26
:10383000A1681A680391002AD2D09142D0D13549AB
:1038400000221A600B680392013B0B60C8E7072354
:103850008DF8003023798DF8083001238DF8093078
:10386000BEE708238DF8003023798DF80830012356
:103870008DF80930A3680493B2E7274D09238DF82A
:1038800000302B78002BABD04FF6FF70FFF714FF02
:103890004FF6FF7398420646A2D12049FCF740F844
:1038A000B04204469CD1142200210DEB0200297085
:1038B000FBF738FE0B238DF81430ADF81840ADF847
:1038C000164005A8FBF79EFF8AE70A238DF8003013
:1038D000114BA4681A780294002A81D01422002186
:1038E0000DEB02001970FBF71DFE0C238DF8143050
:1038F0004FF6FF73ADF81830ADF816300794E0E7D7
:1039000005238DF800306BE70623FAE774B3002037
:1039100068B10020B8AF0020BEAF002098B30020EF
:103920002DE9F047474B1B788AB00546002B00F085
:103930008780454B454F93E803003C7803AE86E80B
:103940000300BCB94FF6FF70FFF7B6FE0123ADF8D8
:10395000143001AB06930423029305AA02AB06219F
:1039600080460194ADF81640FFF77EFB07284AD148
:1039700001233B70364B1C689846002C5AD1354ABF
:10398000354F12883B68AA4241D1002B3FD0142208
:1039900021460DEB0200FBF7C5FD072328468DF8F5
:1039A0001430FBF7C9FE0623ADF8160005A8ADF8E4
:1039B00018508DF81C30FBF725FF20460AB0BDE8F3
:1039C000F087CDF804A0019B4046A34224BFC14626
:1039D0001C46FFF771FEBDF814309B00029305AA48
:1039E00002AB06218046FFF73FFB0028EBD00528FD
:1039F000E7D04FF6FF7398451CD1164BA3F8009003
:103A0000154B1C60B4E74FF6FF79A246EDE7013392
:103A10003B6000220E4B31462846FEF7D1FF0028BE
:103A2000CCD00023C8F800303B68112803F1FF33E5
:103A30003B6001D11120C1E7862818BF0320BDE7F4
:103A40000820BBE770B10020247C050073B3002080
:103A500074B3002068B10020B8AF002063DF704766
:103A6000A6DF7047A2DF70472DE9F04391B098467A
:103A700011238DF8043013788DF805300024164694
:103A800001254FF0000365F34203074689461C22D7
:103A9000214609A88DF80630FBF744FDB3788DF870
:103AA0000930C3F30302A24214BF1A2212228DF876
:103AB000242001AA0E9203AB72788DF8082004939B
:103AC000224602AB65F34202059308238DF80A20D3
:103AD000CDE9064404AAADF81C3009A9434638884C
:103AE0008DF80E50ADF80C900894FFF7BBFF11B0A5
:103AF000BDE8F083A0DF7047044A012311688340CA
:103B00000B401ABF1218507E1846704764AD002053
:103B100070B4094D134601262A6806FA01F41442CE
:103B200007D001F1190402463146281970BCFDF78F
:103B300063BD70BC704700BF64AD00201FB500239B
:103B4000CDE9013303938DF80A201A46074BADF8EF
:103B5000081006241978ADF806008DF80440FFF728
:103B6000D7FF01A8FFF709FA04B010BDAF2C002061
:103B700010B4084A012314688B40234006D00A443D
:103B80005DF8044B0146507EFDF7A6BC18465DF873
:103B9000044B704764AD002010B50A4B19780446F9
:103BA000FFF7E6FF58B1084B00205A88A24201D126
:103BB000C0B210BD0130082803F10C03F5D1FF207D
:103BC000F7E700BF4CAF00204EAF00202DE9F843CF
:103BD0000546FBF7B1FD234B07460022142098460B
:103BE00000FB02F1CC5AAC422AD10B4400263446E9
:103BF0004FF014095BB199782846FEF755FA10B1D9
:103C0000052818BF032401363246072A1DD9A4B956
:103C1000FF2D24D8144928464FF6FF75FFF794F975
:103C2000FFF762FCAF4208D03846FFF7B5FFFF2828
:103C300003D00C2343430D4AD5522046BDE8F883F8
:103C40000132082ACCD10023D0E709FB02F338F86F
:103C50000310A94201D14344CCE70132D5E7072440
:103C6000EBE700BFBCB4002098B300204EAF0020AB
:103C70002DE9F0411F46154B9DF818400E46904621
:103C800019780546FFF744FFB8F1000F17D0104B25
:103C90003A4619782846FFF73BFF0E4B2246197823
:103CA0002846FFF735FF44B12846FFF775FFFF2888
:103CB00003D00C234343084AD652BDE8F081002CC0
:103CC000FBD03046BDE8F041FFF780BFAF2C0020AD
:103CD000B12C0020B02C00204EAF002008B5FFF71B
:103CE0005BFFFF281DBF0C234343034A4FF6FF70C1
:103CF00018BFD05A08BD00BF4EAF00202DE9F043D9
:103D000085B00546FFF7EAFF4FF6FF739842074676
:103D100041D001224FF0030901AB0821384602F1DE
:103D20000108FEF7D5F81FFA88F8064648BB029945
:103D30000A46032342F8049B06312846FBF7F0FCB1
:103D4000044660B908213846FFF7CCFA0446112C26
:103D50003FD01AD80CB30C2C2FD107231EE00C280F
:103D60000DD0052800D1344608213846FEF79CF9CD
:103D7000002818BF03244246002ECDD1E7E70126D4
:103D8000F2E70728E9D00446E1E7862C13D043F296
:103D900002039C4211D100221CE0012328468DF829
:103DA0000430ADF80850FFF799FFADF8060001A800
:103DB000FFF7C8F8EFE70823F0E7092328468DF856
:103DC0000430FFF78BFFADF80850ADF80600039400
:103DD000EDE70122034B28461978FFF799FE05B05D
:103DE000BDE8F083DEAF00200378072B02D14088C6
:103DF000FFF784BF704700002DE9F0434FF6FF75D1
:103E0000A84285B0044668D0FFF768FFA84227D1D2
:103E100000260327B0464FF001093B463246414693
:103E20002046FBF77FFC042805464DD0082847D0E4
:103E30000B282DD117F002031FD1B8F1000F20D1AC
:103E40001EBB032320468DF80430FFF747FFADF873
:103E50000840ADF8060001A8FFF774F8002237E02B
:103E6000002301AA0821FFF7FFF80028D0D1029B08
:103E700003F106089E881F68CDE701274FF000096F
:103E8000CBE703271E469846F8E703274646F5E7A3
:103E9000B9F1000FD5D0112819D043F2020398428E
:103EA000DCD008B90223CDE7092320468DF8043081
:103EB000FFF714FFADF80840ADF806000395CAE718
:103EC000B9F1000FEED1BCE7B9F1000FB9D0012272
:103ED000034B20461978FFF71BFE05B0BDE8F083C1
:103EE000DDAF002037B50578012D044614D1408898
:103EF000FFF782FF6088FFF7F1FE00236A4629463C
:103F0000FFF7B2F840B9019B1B782BB1034B6088D7
:103F100019782A46FFF7FCFD03B030BDDFAF002063
:103F2000F0B587B004460E461746FFF7D7FE4FF6AA
:103F3000FF739842054624D01E4B20461978FFF7A0
:103F400017FE80B30023CDE90033029304238DF8DC
:103F50000030194BADF802401978ADF804602046E6
:103F60008DF80670FFF704FE68B12846FFF72EFEB5
:103F7000124B204600221978FFF7CAFD6846FEF76B
:103F8000FCFF07B0F0BD07212846FEF78DF8052895
:103F9000EED10923049003A88DF80C30ADF80E4043
:103FA000FEF7EBFFE4E73A4631462046FFF7C6FD51
:103FB000E7E700BFB12C0020B02C0020AF2C002080
:103FC00010B5027886B004461AB1012A09D006B0AD
:103FD00010BD0E4B1B78002BF9D0C088FFF7F6FD03
:103FE000F5E70B4B40881978FFF792FD142200216A
:103FF00001A8FBF797FA6088ADF80600FFF76EFEA0
:10400000ADF8080001A8FBF7FDFBE0E770B1002068
:10401000A0AD002070B5044686B01422002101A88E
:10402000FBF780FA23786088ADF80600013B0B2B84
:1040300000F29080DFE803F02106233A4E585C68D6
:10404000747A7C8C2679444B321C19784FF0010528
:1040500018BF01228DF80450FFF75AFD731B5A4216
:104060005A413E4B60881978FFF752FD6088FFF790
:1040700035FEADF80800002D42D106B070BD022318
:104080008DF804302379002B14BF012302238DF80F
:104090000C30314B01221978FFF73AFD2F4B227972
:1040A00019786088FFF734FD0125DFE703238DF8D9
:1040B00004302A4B1978FFF75BFD002814BF012359
:1040C00002238DF80C30A3798DF81030A388ADF859
:1040D0000E30E9E7204B1978FFF74AFD0028CCD1D4
:1040E00002238DF80430DFE703238DF80430EAE77C
:1040F0000723A2888DF80430ADF808208DF80C3025
:1041000001A8FBF77FFBB8E708238DF80430A388EC
:10411000ADF8083007238DF80C30A3680593EFE75E
:1041200006238DF8043063680393BDE70523D8E7C1
:1041300003238DF80430094B1978FFF719FD002887
:1041400014BF012302238DF80C3041F20113BEE7A6
:104150000423C6E7002589E730B30020A0AD002086
:104160001FB50D294FF0000301930393ADF806002E
:10417000029108D10B2301A88DF80430FFF74AFF04
:1041800005B05DF804FB86290CBF0A230923F2E77A
:1041900030B508490A680023012505FA03F42242D4
:1041A000D8B202D122430A6030BD0133182BF4D1BA
:1041B0001846F9E764AD002010B50378182B0446C3
:1041C00002D1FFF7E5FF207010BD000010B5024BD3
:1041D000197DFDF72FFA10BD64AD00202DE9F04FD9
:1041E0003D4D89B02878FFF787FC60B103A8FFF741
:1041F000EDFFDFF8E8A0DFF8E8B00DF110090027C7
:10420000039B9F4202D309B0BDE8F08F39F8024BFF
:1042100029782046FFF7ACFC064678B39AF80010E0
:104220002046FFF7A5FC804640BBBBF800304FF6A8
:10423000FF7219462046FBF777FA43F203029042D9
:1042400029D10133ABF80030EFE7052320468DF884
:104250000030FFF743FDADF802006846ADF80440BA
:10426000FEF770FEB046324629782046FFF750FC34
:1042700042469AF800102046FFF74AFC0137BFE794
:104280002046FFF72BFDFEF74BFE0026EBE720460E
:10429000FFF7B2FDE7E70828F2D012D80028D4D003
:1042A0000628EDD00923029020468DF80030ADF8A5
:1042B0000440FFF713FDADF802006846FEF742FE2A
:1042C000D1E743F202039842CDD043F20143984232
:1042D000DDD01128E6D1C6E7DFAF0020E0AF002037
:1042E0008CB500201FB5044640882378ADF8060041
:1042F000012B10D05AB21AB1022B15D004B010BD48
:1043000001A88DF80420FEF71DFE6088FBF714FA63
:10431000FFF772FDF2E78DF8043001A8A388ADF82D
:104320000830FEF70FFEE9E72379002BE6D0FBF714
:1043300003FA4FF6FF739842E0D0044B012219783C
:10434000FFF7E6FBFFF74AFFD8E700BFDFAF00202B
:1043500038B5074C0146207DFDF7BEF830B1A07D91
:10436000FDF7BAF8002814BF0220012038BD00BFB5
:1043700064AD00202DE9F0478CB089461646804692
:10438000FFF7E6FF20228246002104A8FBF7CAF8C7
:10439000BAF1000F46D0B9F1000F17D099F80050CC
:1043A00015F001054FF6FF7415D04046FFF796FC57
:1043B000A042074639D14048FDF724FDB0F5807F83
:1043C00001D0B84275D10025032470E04D46852602
:1043D0004FF6FF775FE02E4627465CE04A463146BF
:1043E0004046FBF7A5F90446B9F1000F5DD000285F
:1043F0005DD199F8003013F0010F14BF01210221A3
:104400004046FEF7DBFDB6F1850218BF012200240D
:104410000095012339464046FFF72AFC20460CB0A0
:10442000BDE8F08743F20204F8E7002502AB012261
:1044300007213846FDF74CFD0446002837D12146B8
:1044400050220398FBF76EF8039B83F800A0039CAF
:10445000079604F13403049304F118030893631CD2
:1044600009934046154B0B93FFF796FBFF280CD0A2
:10447000134A0C2101FB002050F8042FC4F811202E
:104480008288A4F815208279E2753846FBF7FCF99A
:10449000044660B90646BAF1020F04AB9ED1002271
:1044A00031464046FBF744F90446002CABD00022CD
:1044B000AEE707460125B9E778B3002033B3002003
:1044C0004EAF0020F0B585B00446FFF741FF324FF4
:1044D000012806463D7831D12046FFF7FFFB4FF615
:1044E000FF7398422AD0204632462946FFF710FB38
:1044F0000023CDE90133039301A80C238DF8043088
:10450000ADF80640FFF786FD244B1B78E3B1397800
:104510002046FFF72DFBB8B9214B22491A682046E7
:10452000FFF728FF8628054632D011280FD070B13A
:1045300029462046FFF714FE05B0F0BD00222946AB
:104540002046FFF7E5FADFE700221146E7E7A5F18D
:1045500011035E425E410022134B20461978FFF79B
:10456000D7FA124B324619782046FFF7D1FA104B92
:10457000002219782046FFF7CBFA0E4B002219785B
:104580002046FFF7C5FA002DD6D0112DD4D0CFE7A5
:1045900000260122E0E700BFAE2C00205FB400201F
:1045A0001CB300205AB40020AD2C0020AC2C0020FD
:1045B000AB2C0020AA2C0020F0B587B0074601A83C
:1045C000FFF704FE02AD0024019B9C4201D307B01B
:1045D000F0BD35F8026B39463046FFF7C9FA10B125
:1045E0003046FFF76FFF0134EEE700002DE9F04F92
:1045F000054687B0904699460F4639B9A14B1B78BE
:10460000F3B90524204607B0BDE8F08FFFF7A0FE00
:104610000138C0B2012800F22D8100212846FBF7A5
:1046200089F80446862C00F0B080112C00F09980A7
:10463000002C00F09680B9F1000F00F0BF80B9E0C7
:10464000FFF786FE012800F09E80022840F01281CC
:104650008D490B78284613F001048B4614BF4FF0A8
:10466000010A4FF0020AFFF739FB4FF6FF73984239
:10467000064659463AD03B4602AA0721FEF7F4FC0B
:104680000446F0B9039B93F84420D10740F1C7805A
:10469000B8F1000F40F0D68003F1340202F11201AC
:1046A0002846FBF743F84FF0000A04460023009326
:1046B000BAEB030318BF0123B4FA84F2520931465E
:1046C00045E00528F2D1BDE004AB012207213046C8
:1046D000FDF7FEFB0446002840F0C1803046FBF7A2
:1046E000D3F80446002800F0B280B8E0002C41D096
:1046F0006648FDF787FBB0F5807F834637D0B04230
:1047000036D004AB01220721FDF7E2FB044650B985
:104710005846FBF7B9F8044628B95B492846FBF729
:1047200009F8044638B107215846FDF7BDFC10B121
:10473000052818BF03244FF6FF73BBEB030318BF14
:104740000123B4FA84F20093520901235946284602
:10475000FFF78EFA002C7FF465AF51462846FEF72E
:104760002DFCA4F111035E425E4100220FE0B3462E
:104770000324E0E72846FAF7DDFF0097044601230B
:10478000B0FA80F29AE7404948E700260122404B00
:1047900028461978FFF7BCF93E4B3246197828466F
:1047A000FFF7B6F9B9F1000F08D0002C3FF42AAF9B
:1047B000112C17D021462846FFF7D2FC0D2C3FF4D0
:1047C00021AF06D8002C3FF41DAF082C18BF0324DE
:1047D00018E7862C14D043F202039C423FF412AF38
:1047E000112C1AD12C4B3A4619782846FFF790F92C
:1047F0002A4B424619782846FFF78AF9002401E738
:10480000254B3A4619782846FFF782F9234B424652
:1048100019782846FFF77CF9F4E60324F2E6B8F1AC
:10482000000F0FD1598D03F1180200297FF436AF24
:1048300003F12C01343311F8010B00287FF42EAF63
:104840008B42F8D19BF80030DA073FF53DAF0E49B7
:104850002846FAF76FFF044600283FF427AF0721E8
:104860003046FDF721FC00283FF420AF052818BF93
:1048700003241BE743F20204B9F1000F3FF4C2AE78
:1048800098E700BF5FB400205AB4002078B300203E
:10489000AB2C0020AA2C0020A92C0020A82C002042
:1048A0002DE9F04786B00746FFF726F958B101A871
:1048B000FFF78CFCDFF84880DFF8489002AE002557
:1048C000019B9D4202D306B0BDE8F08736F8024B4B
:1048D00039462046FFF74CF980B198F80010204681
:1048E000FFF746F999F8001082462046FFF740F995
:1048F0000123014652462046FFF778FE0135DFE7E7
:10490000A82C0020A92C002010B50378062B0ED966
:10491000072B1BD10E4B1C782046FFF7EDF810B18A
:104920002046FFF749FE0B4B1878FFF7B9FF0A4BFB
:104930001C782046FFF7E0F810B12046FFF73CFE58
:10494000064BBDE810401878FFF7AABF10BD00BFA6
:10495000AD2C0020AB2C0020AC2C0020AA2C002079
:104960001FB503780446092B09D8DFE803F0050AD0
:1049700020202020202020204088FFF7A3FD04B025
:1049800010BD144B197819B3134B00791B7803F041
:104990000102904206D86179C3F34003994294BF63
:1049A00000210121012300226088FFF71FFE2378E8
:1049B0008DF80430043434F8023CADF8063094E845
:1049C000030004AB03E9030001A8FFF723FBD6E7CC
:1049D0000121E7E75FB400205AB4002037B5174B38
:1049E000174A5B881188174C174D994208D852888E
:1049F0009A4205D36369FBB900232B7003B030BD25
:104A00002B783BB16369002BF6D000228DF804208F
:104A100001A80FE00D490E480978D4E901230029C7
:104A20000CBF11461946FDF785F90028E4D0A369AB
:104A3000002BE1D09847DFE70122E7E7AEAF002087
:104A4000B8B3002010AF0020A4AE002088B400202E
:104A50002CAF00207BDF70477ADF704776DF70472E
:104A600075DF704737B5164B18884FF6FF739842BD
:104A700010D0144A144D1378297B0133DBB29942CC
:104A800013702C4608D31149FFF7EAFF10B1AB6948
:104A900003B1984703B030BD002313702B7C33B1B2
:104AA0003B21FFF7DBFF10B1AB6903B198476369A6
:104AB000002BEFD000228DF8042001A8E9E700BF09
:104AC0000CAF002088B4002010AF0020B8B3002045
:104AD00065DF70472DE9F74F0C9CBDF834B027888F
:104AE000002580468A4691462E46B8F80020B242FC
:104AF0000BDC35B12288013AD21B92B2FF2A39D899
:104B0000DA55002003B0BDE8F08FD8F8042052F841
:104B10002600019000220DF1030101A8FFF7D8FF44
:104B20000028EFD19DF803204A4521D12288002D8D
:104B300014BF0020022002EB09010144594519DC91
:104B40003DB9013292B2228003F802A022880132DC
:104B5000228022880DF103011A4401A8FFF7B8FF53
:104B60000028CFD121889DF803200A442280012506
:104B70000136BAE70C20C5E72DE9F341089CBDF8E2
:104B800024501746CDE9004502220646FFF7A2FF52
:104B900048B9102239463046CDE9084502B0BDE893
:104BA000F041FFF797BF02B0BDE8F0812DE9F04F6B
:104BB00000231688138090F82D3085B007460D46E7
:104BC00014465BB3082E01D80C2008E102A8FAF7BE
:104BD00031FE002840F0038113880822CA5423883C
:104BE00001339BB21B222380CA54238801339BB21A
:104BF000CA18DDF809102380E950BDF80D30938004
:104C000023889DF8082006339BB212F0FE0218BFDD
:104C100001222380EA54238801332380BB78FBB12F
:104C200023880433B342CFD802A8FAF701FE002844
:104C300040F0D58023880322EA54238801339BB2B5
:104C400019222380EA542388BDF8082001339BB23F
:104C5000E9182380EA54120A4A7023880233238019
:104C6000FA789AB12388D91CB142ADD80221E9540F
:104C7000238801339BB201212380E95423880B440C
:104C80009BB22380EA5423880B4423807A68AAB11C
:104C90002388D91CB14297D8022192F90020E95407
:104CA000238801339BB20A212380E95423880133EE
:104CB0009BB22380EA542388013323803B89002B55
:104CC00040F081803B8A53B1CDE900462B46072254
:104CD000032107F11000FFF74FFF00287FD13B8B26
:104CE00053B1CDE900462B461522142107F11800D7
:104CF000FFF742FF002872D13A6A002A72D1D7F832
:104D00002480B8F1000F30D0B8F804302188981C06
:104D10008A1C0244B2423FF657AFFE283FF654AF1A
:104D200003336B54238801339BB2FF222380EA5460
:104D3000238801339BB22380B8F80020EA54E91895
:104D4000120A4A702088023080B22080B8F804200D
:104D50005AB1D8F8081000294ED0284432F00AFF82
:104D60002388B8F804201344238097F82C30002BB4
:104D70007DD1387898B33B88012B3DD0228802F151
:104D8000020CB4453FF620AF012805D17B780233F1
:104D900013449E42FFF418AF023EB61AB6B202A9FF
:104DA00005EB0C00ADF80860FAF740FDB8B93B78A8
:104DB000022B40F09F80BDF80830B34240F2B5802E
:104DC000ADF808609FE0CDE900462B46062202219F
:104DD00007F10800FFF7D0FE00283FF473AF05B0DD
:104DE000BDE8F08FB4F800C00CF10603B3423FF603
:104DF000EBAE1188052901D80720F0E76FF4486E63
:104E000001EB0E039BB24FF27D3E7345F4D95388FC
:104E1000052BF1D96FF44860181880B27045EBD9B2
:104E20004FF6FF70814203D0834201D09942E3D80C
:104E3000052305F80C30238801339BB2122123800F
:104E4000E954238801339BB223801188E954E81880
:104E5000090A4170238802339BB223805288EA54A6
:104E6000E918120A4A7023880233238047E7BB6A95
:104E7000002BC1D04FF000094FF00C0A4FF0160B79
:104E800097F82C305FFA89F293427FF672AFB96AD5
:104E90000AFB02F201EB0208B8F80430981CFE2865
:104EA0003FF692AE208803332B54238801339BB204
:104EB000238005F803B0238801339BB223808A5AEC
:104EC000EA54E918120A4A702088023080B2208021
:104ED000B8F804205AB1D8F8081000298CD028441A
:104EE00032F048FE2388B8F804201344238009F1E7
:104EF0000109C5E7012B7FF463AF7B789E42FFF485
:104F00005FAFADF808300821BDF80830FE2B3FF642
:104F10005BAE22880133AB542288013292B22280E8
:104F2000A95422881344238059E70921ECE70000A3
:104F30002DE9F0430646B2F8009007460D4690462C
:104F40000FCE9FB06C460FC40FCE0FC40FCE0FC450
:104F500096E8070084E807003C2200210DEB0200E0
:104F6000CDE90C118DF82E108DF82D1000910E91B9
:104F7000FAF7D8FA3C2269460DEB020032F0ECFD5C
:104F8000002840F0C9807C6B002C34D1BB6B23B16E
:104F900004F12400002D3ED184B23B6B23B104F117
:104FA0001201002D62D18CB297F82E30002B00F048
:104FB000A980E11C002D7CD18CB297F82D300BB16B
:104FC0000934A4B2BB780BB10434A4B2FB780BB1A2
:104FD0000334A4B23878002800F08F80012840F014
:104FE00094807B78ADF83C300020BDF83C30023333
:104FF0001C44A4B281E065B1B9F1020F03D80C20C2
:105000001FB0BDE8F083022223782A7011226A7053
:10501000AB700324BAE74845F1D811222A55621C27
:1050200092B22221A954A21C03F1170115FA82F2AF
:1050300003F1270C0E4651F804EB42F804EB6145EE
:10504000F9D104F1120292B21121A95404F1130210
:1050500092B223211434A954073315FA84F453F877
:10506000042B44F8042BB342F9D195E74945C6D83F
:1050700011222A55621C92B21020A854274A1668A1
:10508000023415FA84F456B1107992F805C08445BB
:1050900040D900F1010C82F804C046F820405A1EA5
:1050A000013C0F3312F8010F04F8010F9342F9D1BC
:1050B00079E74945A3D8601C022280B22A551C26F4
:1050C0001444013B2E54A4B2032B25D8DFE803F08F
:1050D0000205071800232B5502E00123FBE72A55A0
:1050E0008CB2A9EB040929190FAA3846ADF83C90F7
:1050F000FFF75CFDBDF83C301C44A8F800407FE79A
:105100000323E8E7002DECD157E70FA90020FAF7B9
:105110008DFB6AE7042073E7072071E780B4002065
:10512000F0B590F82D3085B00C461546002B44D1D3
:1051300090F82E30002B40D1436B002B3DD0C3782C
:105140000BB15B0739D584B32B68072B33D9083BE8
:10515000B3F5803F28BF4FF6FF7304F10806ADF8A2
:1051600006300DF106023146FFF7E2FE0346F8B9BC
:10517000BDF80620083292B2ACB1110AA71C6170CA
:10518000F11B89B2052902902270CDF80B0012D9CB
:1051900002A8FAF74FFB50B9DDF80910C4F8021065
:1051A000BDF80D10E1802A6002E02646D9E70346EB
:1051B000184605B0F0BD0423FAE70723F8E713B556
:1051C00090F82D301446CBB190F82E30B3B1436B2C
:1051D000A3B9C3780BB15B0710D52368B3F5803F43
:1051E00028BF4FF6FF730DF10602ADF80630FFF74A
:1051F0009FFEBDF80630236002B010BD0720FBE71C
:1052000007B5144B1A686AB1002018601B68009338
:105210004FF08042009B0123C2F808330E4A5370BE
:10522000FAF798FB0D4B1A688AB100221A601B68C6
:105230000193019B4FF080430222C3F80823064BE1
:105240000120987003B05DF804EBFAF783BB03B05C
:105250005DF804FB00010040F0AE002004010040B6
:105260000E4BD3F8183182B0B3B10D4B0D4800226C
:105270001A601B680193019B0B4B997EFF291FBF8E
:1052800001228A404FF0A041C1F8082500225A7639
:105290001A711B6802B0184702B070470030004016
:1052A0001831004068AE002064AE002070B52D4C6F
:1052B00086B094F82130019394F820300093E3698C
:1052C00004F1260204F123014FF04020FAF760FBBD
:1052D0002346E0B994F82360A56906BB217B8A1EAA
:1052E000012A1CD8E0692269904218D16269E37BE7
:1052F000E261C5F34015032984F8203084F8215079
:1053000007D100954FF040212046FAF718FC06B06F
:1053100070BD4FF040212046FAF7B4FBF7E7124A80
:1053200007CA06AC04E90700C6B14FF04021D1F826
:10533000C424C1F8C42490070CD501228DF808209C
:10534000002283F824206A07E1D4D3E9002102A8CF
:105350009047DCE75107F3D50222EFE78DF80860AC
:10536000EEE700BF3CAE002048AE0020F7B5154682
:105370004FF0FF32C1F8082390F8242004460F466E
:1053800002F0FF0E2AB18368C1F80433112003B084
:10539000F0BD012680F82460836100F10C0C95E8D3
:1053A00007008CE80700AA7884F820206A68E26188
:1053B0006A78C7F888252A78B24212D012B91E1C22
:1053C00018BF012684F821600096AB786A683946D8
:1053D0002046FAF7B4FB2368002BD8D184F8243098
:1053E000D5E784F821E0AB786A6839462046FAF7B9
:1053F00049FBF0E730B54A4AD2F8043313F4007F92
:1054000085B015464AD0D2F82431002B46D04FF44F
:1054100092711046FAF7FEFB4FF40173C2F808339D
:10542000404B997E09B9012151603D4902228DF816
:105430000020D1F88024C1F880240392DA7D8DF811
:105440000820DA6801920022DA751A766846D3E9F4
:10545000001290473248D0F81C313BB1314A938A50
:10546000917D994247D91146FAF703FC2C4AD2F8AC
:1054700044318BB14FF4A2711046FAF7CBFB294BA4
:10548000997E09B101211160DA7D2AB10022DA7515
:10549000587ED968FAF76EF805B030BDD5F80433F8
:1054A0005B07D7D5D5F80831002BD3D01D4C1C484D
:1054B0002146FAF7C7FB637EE27D9A422346C9D1B3
:1054C000227E52B12369E168E3600023607EE275C9
:1054D00023766376FAF74EF8BCE7A27E0AB901227A
:1054E0006A600F4A4FF40171C2F808130022DA759E
:1054F000587ED968EEE74FF48E71FAF78BFB917DF9
:105500000029B3D000238DF8081091688DF8003081
:10551000019193756846D2E900139847A6E700BF4A
:105520000020004020AE0020800000F1A040D0F814
:10553000003723F44033C0F80037D0F8003743EA8F
:105540000141C0F8001770470E4B034493F9402007
:10555000072A02DD0021FFF7E7BFD3B2072B10D8DF
:10556000930003F1804303F5C043D3F8101521F0F5
:105570000101C3F81015012303FA02F2024BC3F82C
:1055800008237047B4AD00200060004000F1804067
:1055900000F5C040002382B0036003680193019BC3
:1055A00002B070472DE9F04F85B00024594D0194A9
:1055B0004FF48072012102F1804303F5C04390B2A1
:1055C0001B68012B06D1D5F804330B4202D0FFF73C
:1055D000DDFF0C430432B2F5907F4FEA4101EAD17E
:1055E0004D4B1B68012B0AD14FF4BE70FFF7CEFF65
:1055F0004FF0A04344F00044D3F81035019314F069
:10560000FF0F1AD0454F01260025344210D0AB00C1
:1056100003F1804303F5C043D3F81005D3F8101508
:1056200057F8253023B1C1F30141C0F30420984756
:105630000135082D4FEA4606E7D1002C63DA4FF01A
:10564000FF330022CDE90232344D354E0024A2460C
:1056500001274FF0A04816F9012B531C46D0D2B2B7
:1056600022F0C0094FEAD90104A8084402F0070358
:1056700010F808CC07FA03F31CEA030F36D005EB49
:10568000090C92099CF940C055F82CB0BBF1000FF1
:105690000AD1032A2AD10DF10C0E1EF801C04CEAE2
:1056A000030C0EF801C001E0032AF4D009F5E07103
:1056B00010F80C0C58F821101842C1F3014105D024
:1056C000022913D1032A0BD1114604E003290DD17D
:1056D000032A05D102214846FFF726FF0134E4B230
:1056E000BBF1000F02D011464846D8470AF1010A23
:1056F000BAF1080FAFD134B14FF0A043019AD3F8FB
:105700001035934202D105B0BDE8F08F0193039BA1
:1057100002939AE7006000407C610040B4AD002035
:1057200014AE00200028C3B2A8BF00F160424FEAC7
:10573000501010B5BABF0D4A03F00F0402F56142D4
:105740004FEA41114FEA8000C9B200F16040B4BF96
:10575000115582F8001300F5614003F01F02012388
:105760009340C0F88031036010BD00BF14ED00E02D
:105770002DE9F8430568EB175906674B41EAD51147
:1057800004464FF0FF3268068B4208BF82420AD3BC
:10579000624A002332F022F800F5006020F47F67AF
:1057A00027F00F072FB929465D48BDE8F8432AF0D6
:1057B00007BC207922F0C6FC40B9607922F0C2FC17
:1057C00020B95848BDE8F8432AF0FABBE279E17AFB
:1057D0000D201EF01BF8237B534A002B00F08A801B
:1057E000537843F01003514E5370F3781BB10023EC
:1057F000F370FAF737FF257900232846F37022F07B
:10580000A1FC20B14FF44071284615F0B9FF65792D
:10581000284622F097FC20B14FF49851284615F005
:10582000AFFF637A2579002B284614BF4FF00E098D
:105830004FF0000922F086FC00285FD03C4B05EBBE
:1058400045051D4495F801806479204622F07AFCD4
:10585000002856D0364B04EB44041C446378354C86
:10586000E27E002A50D15A1C0AD04FF0A0410122FA
:105870009A40C1F8082503F5E072032041F82200A0
:10588000B8F1FF3F2C4D1FBF4FF0A04108F5E0726B
:10589000002041F82200C5F82475C5F86C95002752
:1058A000C5F81485C5F80C35244B636028464FF4C1
:1058B0008E712760FAF7AEF94FF4A271FAF7AAF9E0
:1058C0001F4BC5F8043302210846FFF72BFF0423C2
:1058D000C5F80035B8F1FF3F4FF48073E7822776B3
:1058E000638315D01748FAF79DF90123A376FBF7D8
:1058F000FBFA0DE0537803F0EF0374E74FF0FF3845
:10590000A2E74FF0FF33AAE708210F482AF038FB3F
:105910000123F370BDE8F88347E8010048E801007F
:10592000247D0500397D05005CAD002099B500207F
:10593000BC7D050020AE0020002000400195030042
:1059400080000200387C05004F7D050010B50D4C2D
:1059500000226260A2602261E2600B4A106810F0CF
:10596000010002D10621FFF7DDFE084B1B7823B9A9
:105970004FF080430122C3F8182501232370002033
:1059800010BD00BFF0AE002000E100E061B40020D7
:10599000F8B50E46D11C48BF911D144641F387014E
:1059A0000546671EFAF724FA00214AB2A24201F125
:1059B000010100DBF8BDBB1A23F00300B25C03F069
:1059C0000303DB0002FA03F32A581A432A50ECE7D8
:1059D000F0B500254F1E6CB28C4205F1010500DBCD
:1059E000F0BD3B1B23F0030603F003039659DB00D5
:1059F00026FA03F30355EEE72DE9F041B3F902402F
:105A000014F11F0548BF04F13E050F4603F12406BB
:105A100045F34715904601462B4632463846FAF77D
:105A200027FAB8B9B4EB451F16DA6211012304F066
:105A30001F0403FA04F457F822301C4214BF012457
:105A400000242B46324639464046FAF711FA2046E2
:105A5000BDE8F0810124F4E70446F2E710B5002325
:105A60001A465CB2A14203DCB2FA82F0400910BDD2
:105A700050F8234001332243F3E700002DE9F04FB3
:105A80008A46234F8BB00646114650461446FAF715
:105A90008FF93B68FBB10425C0EB441014FB05FBF8
:105AA00000B205FB04654FF0FF38043D28FA00F80A
:105AB0004FF040093B6859463046984758B12B682B
:105AC00003EA08032B6021463046FFF7C7FF20B1E9
:105AD000B9F10109EED1002017E0234632465146C4
:105AE00002A8FAF795F92146019002A8FFF7B6FF40
:105AF000019B003318BF01235B00002814BF5842EC
:105B0000C3F10100C0B20128E2D10BB0BDE8F08FB3
:105B1000602E00202DE9F04FD1B0CDE905015B9D4D
:105B200095F9004048A8914622461F46FAF734F9F5
:105B3000A3000793069BA20013441946224638A8E7
:105B40000293FAF729F995F90060002F00F08C8094
:105B50003246394628A8FAF71FF90DF5807A324601
:105B600030AF48A95046FAF717F938A93846FAF77E
:105B700013F92B4628AA38A948A8FAF7CCF82B46DF
:105B800028AA38A948A8D5F8A460B0472B4628AA67
:105B900039465046FAF7BFF8BDF968310497023B21
:105BA0001BB2002B67DCD9F80030009503F0010828
:105BB0004FEA481840AADB4302EB080A03F001034E
:105BC00030AA90445B0140AA1A44039230AAD31829
:105BD0004146039A0493504605F10409FAF73FFB46
:105BE0004B4640AA48A908A80094FAF7A8FA08A9C1
:105BF00008462B464246FAF74DF808A908462B46B8
:105C0000069AFAF747F8214608A8FFF727FF002869
:105C10005DD008A8FAF7ECF808A92B46029A0846C6
:105C2000FAF738F808A92B4652460846FAF732F830
:105C3000DDE90301434652460095FAF792FA2B46F6
:105C400008AA30A940A8FAF766F8224640A90598A4
:105C5000FAF7A2F8059B079C234430A91846FAF7E7
:105C60009BF851B0BDE8F08F314628A8FAF7C0F88C
:105C70000123289371E71FFA83F85B1108F01F02D4
:105C800059F823300095012101FA02F21A42049BCF
:105C900013BF20270027202600260AEB070B1F44EE
:105CA0000AEB06030393049B039A1E4433463946CA
:105CB0005846FAF7D4FA08F1FF383B4600955A46A1
:105CC00031460398FAF74DFA0FFA88F369E710AFF7
:105CD000224608A938460DF1600BFAF75DF820AEB0
:105CE00049465846FAF758F830462146FAF780F800
:105CF000012328A82093FAF77BF822465946384614
:105D0000FAF735F828B9224620A908A8FAF744F886
:105D100082E73B68DA0709D421463846FAF71AF8D1
:105D2000224649463046FAF7EEF9E6E7189BDB07CC
:105D300007D421465846FAF70DF82246494628A8C6
:105D4000F1E7002823461CDD5A4639463846FAF763
:105D50005FF821463846F9F7FDFF224628A930466C
:105D6000FAF705F8002805DA23464A463146304658
:105D7000FAF77EF8234628AA31463046FAF748F863
:105D8000CEE73A4659465846FAF742F82146584671
:105D9000F9F7E0FF2246314628A8F9F7E8FF002886
:105DA00005DA28A923464A460846FAF761F828A9E1
:105DB000234632460846FAF72BF8BEE72DE9F047AE
:105DC00093F9006092B00446894610463146154664
:105DD0009846FFF743FE002840F09180424649462E
:105DE0000AA8F9F794FF43460AAA214602A8F9F740
:105DF00051FF0AA908464246F9F789FF43462A4659
:105E000049464846F9F746FF08F104074246294645
:105E10002846F9F77CFF3B462A4621462046009655
:105E2000FAF704FA3B462A46294628460096FAF72E
:105E3000FDF93B462A46214628460096FAF77FF9A7
:105E400043462A4621462046F9F724FF3B46224690
:105E5000214628460096FAF7E9F93B4600962A467D
:105E600021462046FAF7E2F92368DB074AD5334694
:105E70003A4621462046F9F7FBFF31468246204646
:105E8000F9F768FF06F18043013B54F8230040EA2C
:105E9000CA7044F82300424621462846F9F737FFE6
:105EA0003B4602AA294628460096FAF748F93B469F
:105EB00002AA294628460096FAF741F902A908469F
:105EC0003B462A460096FAF73AF9434602AA21468B
:105ED0002046F9F7DFFE0AAA3B4610462146009607
:105EE000FAF72DF9324629462046F9F755FF49467B
:105EF0002846F9F751FF0AA94846F9F74DFF12B0B5
:105F0000BDE8F08731462046F9F724FFC3E70000DB
:105F100073B500230DF102008DF80230FBF77AF81B
:105F2000264B1B7803F0FF04002B41D1244B1A6849
:105F3000002A3DD0234AD2F80813C90738D51C607F
:105F40001B68214D01930DF10300019BD2F80865F8
:105F50008DF80340FBF75EF86A6829681F2A98BF2E
:105F6000541CA142F6B26C6004D1202C14BF611CF9
:105F70000021296015499DF803008E542A68944237
:105F80003ABFC2F121021319A31AAA689A4238BF74
:105F9000AB60FBF7B9FE6B682A681F2B94BF013317
:105FA00000239A4201BF074A0123C2F80833536015
:105FB0009DF80200FBF7A8FE02B070BD61B400209E
:105FC00000D1004000D000404CB4002028B4002094
:105FD00030DF70472DE9F74F3B4F06468846B8F152
:105FE000000F03D1012003B0BDE8F08F4546202DFE
:105FF00028BF20255FFA85FB002400230DF1020055
:106000008DF80230FBF706F8304B1B7803F0FF09E0
:1060100093BB0DF103008DF80390FAF7FBFFD7E96E
:1060200000148C4204D3641AA54207D9052414E055
:106030002134641AA542F9D8C1F12104244BA542A8
:10604000194431D82A46304631F094FD3B682B4440
:10605000212B28BF00233B6000249DF80300FBF7A1
:1060600053FE1C4B00221A601B680193019B1A4BC4
:106070000122C3F804231A609DF80200FBF744FED6
:10608000B9F1000F08D059463046FFF7A1FF42F2A0
:10609000070398420446ADD0022CAED0002CA9D103
:1060A000A8EB05082E449AE72246304631F062FDFF
:1060B000074BA5EB040A52461946301931F05AFD38
:1060C000C7F800A0C8E700BF4CB4002061B40020AE
:1060D00028B4002000D1004000D0004017B4314A5D
:1060E000314B116889B90021304A106820BB00206B
:1060F0005A79D40740D408B9002949D01C68DA88F5
:10610000234603B05DF8044B184700211160126864
:10611000D9680092009A0029E5D0254AD2F84005B6
:10612000814204BFD88801EB8001C2F840155A793A
:1061300042F004025A71D7E7002010601268986894
:106140000192019A0028D2D0194AD2F83845A042CB
:1061500004BFDC8800EB8400C2F838055A7942F0AD
:10616000020214075A71C3D512F0010402BF64F38E
:10617000C3025A712046BBE702F00601062907D187
:1061800022F0060211075A7106D56FF3C3025A7145
:1061900003B05DF8044B7047054AD2F83805D2F8D1
:1061A0004015ABE714510240A4AD00200451024059
:1061B00000500240A5DF7047A4DF7047A3DF70479F
:1061C0002DE9F0470E4690B016F010058146924634
:1061D0009846189C0CD011238DF8083023788DF840
:1061E000093001224FF0000362F342038DF80A30B8
:1061F0001C22002109A8F9F795F98DF8246005B152
:1062000002AD42F64D23ADF80C3063789DF8641072
:106210008DF804300022A3788DF80530134661F321
:10622000C303DBB243F00303CDE906220E95012739
:1062300001AD8DF80630089203AE1A9BB9F8000044
:106240008DF80E7004AA09A9CDE90465ADF81CA06B
:10625000FDF708FC58BB42F60813ADF80C30637824
:106260008DF80430A3788DF80530034667F34203B8
:106270008DF806301A9A98F800308DF8003098F8AA
:106280000130CDF81A00ADF81E008DF8013032F85B
:10629000080B8DF80E70022304A9CDE90465ADF852
:1062A0001830ADF81C30CDF820D0FFF787FF10B0C4
:1062B000BDE8F087A1DF704708B5FAF7A9F810B17B
:1062C0004F4B504A1A60FAF783F828B14E4B4F4AA9
:1062D0001B68C3F342331360FAF79AF820B14C4AB3
:1062E000D36823F08073D360FAF772F840B14FF0AF
:1062F00080430022C3F80C21C3F81021C3F83825CD
:10630000FAF786F810B1434B03221A60FAF780F8C7
:1063100040B1414B05221A6001229A6700229A601F
:106320003F225A603D4B1B78062B50D13C4B1B68DB
:106330001B074CD13B4B1B6803F0F003502B46D19D
:106340004FF08052384BD2F80414C3F82015D2F81D
:106350000814C3F82415D2F80C14C3F82815D2F881
:106360001014C3F82C15D2F81414C3F83015D2F851
:106370001814C3F83415D2F81C14C3F84015D2F819
:106380002014C3F84415D2F82414C3F84815D2F8E1
:106390002814C3F84C15D2F82C14C3F85015D2F8B1
:1063A0003014C3F85415D2F83414C3F86015D2F879
:1063B0003814C3F86415D2F83C14C3F86815D2F841
:1063C0004014C3F86C15D2F84424C3F87025F9F7CB
:1063D000FFFF28B1154B164A1B6803F04F031360EB
:1063E000144AD2F8883043F47003C2F88830BFF3FF
:1063F0004F8FBFF36F8F104B104A1A6008BD00BF5C
:1064000074C007400DF0ADBA440200103C050040D6
:10641000F0ED00E0A005004010560040E00F00F055
:10642000E40F00F0E80F00F000C000405802001038
:10643000E40E004000ED00E0A42C00200090D0030A
:10644000002382B0036003680193019B02B0704790
:106450002DE9F341844BD3F8042162B3D3F8003320
:106460009F0728D5814D8248FFF7EAFF2B7803F07C
:10647000FF08F3B97F4F804E7B783C4603F0FF0264
:10648000002B00F0AF8073684046984701A88DF854
:106490000480FAF7BFFD7B689DF8040001337B6040
:1064A000FBF732FC754B0122DA601A60744B002254
:1064B0001A6001232B706C4BD3F81821D2B1D3F89A
:1064C0000023560616D5D3F824356E48DB08C3F3EF
:1064D000080113F4FF7F18BF0239FFF7B1FF624BC9
:1064E0004FF48052C3F808254A1EFE2A40F2A480C9
:1064F0000122DA615C4AD2F81031D3B1D2F800330C
:10650000DD0616D56048FFF79BFF1023C2F808335D
:106510005E4BC2F81035FF23C2F814350123D36156
:106520005B4B1C682CB15B4800231A4603210068B2
:10653000A0474D4AD2F84C3133B3D2F800331C0394
:1065400022D55548FFF77CFF4E48FFF779FF5348A7
:10655000FFF776FF4D4BC2F81035FF23C2F8143514
:106560000123D3614FF48863C2F804330D23C2F8CA
:106570000C34C2F80434464B1C682CB14548002347
:106580001A4619460068A047374AD2F828315BB14D
:10659000D2F80033580507D54048D2F80C34FFF73D
:1065A0004FFF0D23C2F80C342F4AD2F81C31B3B17F
:1065B000D2F80033190612D53948D2F80414FFF77F
:1065C0003FFFCB0707D5374B197821B10121C2F81E
:1065D000041400221A70244B0D22C3F8042402B0C4
:1065E000BDE8F0810DF103008DF80320FAF712FDEC
:1065F000BA68134683B93260A660636833B92A4B20
:106600001B7803F0FF025BB1F9F7B8F963689DF8F6
:1066100003000133636043E7B342EED01B68E9E750
:10662000224B1A601B680193019B4FF080430122AB
:10663000C3F804231A60E9E7144A1078502803D1FC
:10664000184901220A7054E711480468002C3FF4ED
:1066500051AF4FF6FF70C3F808050E480B460068AF
:106660000221A04746E700BF00500040DCAF0020F9
:1066700004510040F0AE002004AF002000B0014003
:106680005C2E0020185100401051004080B10020C5
:106690008CB2002090B200204C51004028510040A4
:1066A0001C51004060B4002061B400200001004093
:1066B00013B5284B2849D3F83C3413F0030345D1D4
:1066C0000A680132072A0A602CD9244A012414617D
:1066D0000DF107008DF80730FAF79CFC204B5A6843
:1066E000013A5A605A6822B91E4A127802B3F9F781
:1066F00043F99DF80700FBF707FBBFF35F8F1A4ACA
:1067000000231360BFF35F8F01211160174A1468E3
:106710001CB117481A460068A047164B00221A7091
:10672000FAF716FC0D4B0022C3F8402102B010BD51
:10673000114A4FF080411460D1F80C2402F001128C
:10674000B2F1011FF8D000225A70D2E700230B608B
:10675000E8E700BF005000405C2E002000B0014080
:10676000F0AE002061B40020FC5F00408CB200203D
:1067700090B20020DCAF002004000040D0E90123EB
:1067800093423FBF026842F82310836801333ABF47
:1067900083600020042070472DE9F04F87B00D463C
:1067A00093460190C8B1C2B103680393ABB14FF0F7
:1067B0000009C846019B9B68434503D8CBF800906D
:1067C000002022E0B8F1000F09D1012B0CBFC0233B
:1067D0008023039A52F8284044B90E2015E008F1AE
:1067E000010293420CBF40230023F2E76178227A32
:1067F000571869B9971D002D44D0DBF80020A2EB93
:106800000902BA42029205D2042007B0BDE8F08F17
:106810000737F0E72B702278AA4613430AF8023BA9
:10682000227A6A7062783ABBAE1D227AE1683046FD
:1068300031F0A0F9237A62781E442AB130466168AB
:1068400031F098F963781E44029BDB1B05932369A2
:10685000002BC2D005AA3146606998470028D4D1E0
:10686000059B16B11ABACAF800201F44B94405B1F5
:106870003D4408F101089DE743F00803EE1DAA71AD
:106880002B70D2E7AA462E46E1E710B5144661B157
:1068900013689BB14378027803F00F0343EA0213B5
:1068A00001F8013B2368013B236022464068FFF763
:1068B00073FF10B923680133236010BD0420FCE787
:1068C00070478DDF704777DF7047D0E91F32816FE7
:1068D0001A44D0F88430C0F880200B4490F821107E
:1068E000C0F88430C9B1016F002ABCBF5218C0F88B
:1068F0008020D0F880208A42A4BF521AC0F880209D
:10690000426F002BBCBF9B18C0F88430D0F8843095
:106910009342A4BF9B1AC0F884307047D0F88030EF
:10692000C0F88830D0F88430C0F88C3070470368E5
:10693000C91A436870B5D21AD0E91E6302FB03F48A
:10694000724301FB064501FB1322D0F88040D0F8CA
:1069500084302C441A44C0F88040C0F8842070BDB4
:106960002DE9F04F89B00E4600AF0023044607F131
:10697000140130467B6128F092F805465EB318BBDF
:10698000304629F06BFF8046786126F021F808F543
:10699000807383420CD9A949012029F0BBFB324600
:1069A000A749012029F0B6FB2437BD46BDE8F08F8A
:1069B00008F1070323F00703ADEB030D6D464246D4
:1069C000294630462AF06EF87E693EB99D4901207D
:1069D00029F0A0FBE8E70028F6D1E0E74FF0030834
:1069E000B6FBF8F303EB43039E4201D09649EEE772
:1069F000204621F0A7FB08B99449E8E7944BC7F873
:106A000008D004EB44041C446378924C217900299B
:106A100040F00B81904A0120C2F80415FF2BC2F808
:106A20002415C2F82015C2F81C05C2F82815C2F8B2
:106A300018154FF0C051C2F81415C2F810054FF0E8
:106A4000A04118BF03F5E070C1F85887C1F8FC8A6F
:106A500018BF41F820804FF01601C2F864154FF0BE
:106A6000FF01C2F8681508BF4FF0FF334FF0FF3148
:106A7000C2F860152520C2F87035C2F86C15774B46
:106A800023600221FEF74EFE012323710323B6FB90
:106A9000F3F39BB203EB430808F1010828F001026D
:106AA0009100ADEB010D6846FA606D4A3A604118FD
:106AB0004FF0000C796082F800C0E91C4FF0EE093D
:106AC000851C4FF0880A4FF08E0B63455FDC0C226B
:106AD00002FB030300227968994200F29E80267926
:106AE000012E40F0A28000F06043B3F1005F40F05F
:106AF000A280FB68C3F34E02574B0021C3F8502518
:106B0000C3F83815C3F80815C3F84005C3F80C6579
:106B10006579E28025F0090545F008056571C4E94D
:106B20000210C3F80065022323710D46002977D0B7
:106B30004FF6FE7208EA0202F8F7F4FC494B002215
:106B40001A601B68FB61FB69474B1A601B68BB61DD
:106B5000BB69414B2222C3F8042301221A603A6820
:106B60001278042AFBD94149002222250120C3F8CA
:106B700008530860C3F80025C3F808530860C3F839
:106B800000253B4B2021C3F88410227150E011F8FE
:106B9000026C11F8032C360246EA024611F8012C69
:106BA00005F10C0E164306F44012B2F5001F1ED07C
:106BB000B2F5401F20D0B2F5801F20D105F802BCED
:106BC00006F44002B2F5000F1CD0B2F5400F1ED003
:106BD000B2F5800F1ED105F801BC0235AE454FEA73
:106BE0000616E0D10CF1010C033175466DE76FF02C
:106BF000170205F8022CE3E705F8029CE0E705F828
:106C000002ACDDE76FF0170205F8012CE5E705F8A7
:106C1000019CE2E705F801ACDFE703F8012B5AE736
:106C2000014623682846984788E70820FBF70AF8BA
:106C3000D7F808D0B8E61020F8E700BF7293050037
:106C400099930500C5930500E59305001094050090
:106C5000BC7D0500A4AD002000500240C98D03009A
:106C6000F8B5002004510240145102400450024083
:106C700000E100E070B500221049054629F0BFFC94
:106C800028F074FD0E4B0F4906460322586829F080
:106C9000B6FC044630B10022B1B228F0ACF920466F
:106CA0002CF02CFA084B18682BF096FB00210446B8
:106CB000284613F0C5FA204670BD00BF428A050081
:106CC000482E00204F8A0500B8B5002010B5828AF2
:106CD000C2F30C0402F46043D20448BFC4F3851429
:106CE0000BB9204610BDB3F5005F02D1062060430A
:106CF000F8E71B0407D500220449006829F07FFC4F
:106D000028F034FDF3E70020ECE700BFD091050048
:106D100008B540B2FFF7D7FD40F2EA71BDE8084080
:106D200012F0F0BE38B5054608460C462BF034FF8D
:106D3000002808BF002422460F49284628F0D4F92D
:106D40000E4B4FF6FF72198884B18A4206D100209B
:106D500040F63551BDE8384012F0D4BE0022188804
:106D6000114613F0E3FA0828F2D1F0E78A42EED098
:106D7000188813F0D9FAF6E72B8A0500682D002051
:106D8000014B188812F0D2BE682D0020014B1888E4
:106D900012F0CCBE6A2D002008B5084B1A884FF6B9
:106DA000FF71914209D018881321FDF757FE4FF467
:106DB000F171BDE8084012F0A5BE08BD6A2D0020A3
:106DC00007B500230846072269460093CDF8033033
:106DD000F9F7C6FD0A4B1A884FF6FF7191420BD0A6
:106DE00018886A46012113F0CDFA40F6DF3112F01F
:106DF00089FE03B05DF804FB43F20200F5E700BF33
:106E0000682D002038B500220E49054629F0F7FB11
:106E10000446A8B90C4925F031FC0A49044602464B
:106E2000284628F061F92A460849204628F05CF9EE
:106E300000202BF087FB06490246204628F06DF91A
:106E4000204638BDE2890500E7890500018A050072
:106E5000218A0500F8B5044628B9244A136823F4AA
:106E600080431360F8BD224927F0AEFD0028F4D11D
:106E700020462BF0A3FE0546A0B11C4A136820460D
:106E800043F48043136029F07FFF53EC102B10EE86
:106E9000100A194616F074FB40F6E121BDE8F840EF
:106EA00012F030BE20462BF035FE0028DAD00F4A13
:106EB0001049136843F48043136020462A4629F0A2
:106EC0009EFB2AF0BDFC2A4606460F4620460A498C
:106ED00029F095FB2AF0B4FC02460B4630463946B1
:106EE00016F04EFB40F6E721D8E700BFBCB5002006
:106EF000BF8D0500C48D0500D08D0500084B1A68B4
:106F000018B142F400521A60704722F400521A601D
:106F1000044B1860044B01221A7012F089BB00BFA9
:106F2000BCB50020FCB50020FAB50020F0B583B058
:106F3000044600AF28B9014612F0B6FB0C37BD4637
:106F4000F0BD2BF087FF28B1204627F08BFE0421EF
:106F5000C0B2F1E77860391D204627F0A0FD054654
:106F6000F0B9204629F07AFC0646786025F030FD1D
:106F700006F58073834208D90D49012029F0CAF82B
:106F80000C49012029F0C6F8D8E7F31D23F00703C8
:106F9000ADEB030D6D4632462946204629F082FDB1
:106FA00079680029ECD0284612F0B0FBC6E700BF94
:106FB00072930500E895050008B5044B044958682C
:106FC00028F0A3FCBDE8084012F0D8BB482E0020F2
:106FD00028960500F0B583B0044600AF12F0CEFB52
:106FE000002C60D00023391D20467B6027F057FD20
:106FF000054610BB204629F031FC0646786025F096
:10700000E7FC06F5807383420CD93149012029F051
:1070100081F83049012029F07DF8002420460C3702
:10702000BD46F0BDF31D23F00703ADEB030D6D4628
:1070300032462946204629F035FD78680028E8D0F8
:107040002BF034FB044608B92349E3E7234B2449DA
:107050000246586828F048F820462CF04FF82046A1
:1070600026F024FC7A68294630F084FD204626F07C
:107070001DFC0546204627F0E9FC0146284612F093
:107080008DFB0023391D0A207B60F9F79BFE7B688E
:107090000446002BC2D0134A116819605168596028
:1070A00012891A81BAE720462BF000FB044620B96A
:1070B0000949012029F02EF8B0E7084B084902469B
:1070C000586828F011F820462CF018F8CEE700BFD9
:1070D00072930500E8950500FF950500482E0020F5
:1070E000289605007FB20020F0B583B0054600AFBA
:1070F00048B9384B3849586828F007FCFFF75CFF5F
:107100000C37BD46F0BD0023391D7B6027F0C7FC5E
:107110000646F0B9284629F0A1FB0446786025F020
:1071200057FC04F58073834208D92C49012028F0CC
:10713000F1FF2B49012028F0EDFFE1E7E31D23F0EB
:107140000703ADEB030D6E4622463146284629F073
:10715000A9FC78680028ECD013302BF0A7FA05467C
:1071600008B92049E6E71B4B1B490246586827F03F
:10717000BBFF284626F09AFB044628462BF0BEFFAC
:10718000194B224603F1100153F8040B42F8040B8B
:107190008B42F9D11B8813807D6831462A4604F161
:1071A000120030F0E7FC65742544FE23AB74002028
:1071B000FFF710FF3946054627F071FC28B1036838
:1071C0002360436863600389238128462BF096FF80
:1071D00096E700BF482E0020E09505007293050059
:1071E000E8950500FF950500FA880500F0B5ADF5B6
:1071F000037D064600AF50B9334B3449586828F038
:1072000084FBFFF7D9FE07F50377BD46F0BD0023E9
:10721000391D7B6027F043FC0446F0B9304629F065
:107220001DFB0546786025F0D3FB05F5807383428E
:1072300008D92749012028F06DFF2649012028F0B0
:1072400069FFE0E7EB1D23F00703ADEB030D6C4690
:107250002A462146304629F025FC7B68002BECD0DD
:107260004FF400721C4D3A600022AA601B4A1C4970
:107270001460DBB228465360FFF780FA38B9AB6878
:1072800093B13A4607F108012846FFF785FA40F620
:10729000CC0112F037FC0028B5D138682BF006FA83
:1072A000044618B90F49C9E70720F0E726F0FEFAAF
:1072B0003A6807F1080130F05DFC2046FFF714FF43
:1072C00020462BF01BFF9EE7482E0020E09505008E
:1072D000729305006A950500842D0020B0B500204A
:1072E000142D0020819505002DE9F043E1B00546FD
:1072F00000AF58B95E4B5F49586828F006FBFFF7AE
:107300005BFE07F5C277BD46BDE8F0830023391D5B
:107310007B6027F0C4FB0646F0B9284629F09EFAA8
:107320000446786025F054FB04F58073834208D945
:107330005149012028F0EEFE5049012028F0EAFED4
:10734000DFE7E31D23F00703ADEB030D6E46224696
:107350003146284629F0A6FB7B68102BECD107F1BB
:1073600008044FF480733C220021204607F14405B5
:107370004FF001083B604FF00209F8F7D3F840F2F4
:1073800001433C2200212846BE637B8187F8089098
:1073900087F8358087F83680F8F7C4F87E67384E6E
:1073A000384BBB67736938495B6887F846800022B1
:1073B0009A60736987F844905868FFF7DFF90028EE
:1073C0003AD1736931495868FFF7D8F9002833D1A9
:1073D0002F4B304A1B781370DFF8D0802E4AC8F844
:1073E0001440003318BF012388F801302B4B2C4C7C
:1073F0001B78DFF8BC901370003318BF0123A06026
:1074000031462046C9F8145089F80130FFF7B6F923
:1074100090B941462046FFF7B1F968B94946204680
:10742000FFF7ACF940B91F4B3A461860988007F156
:1074300080012046FFF7B0F940F6910112F062FB9F
:1074400000287FF45EAF38682BF030F9044608B9A5
:10745000154972E726F02AFA3A6807F1800130F000
:1074600089FB2046FFF740FE20462BF047FE48E709
:10747000482E0020E095050072930500AE950500AA
:107480003C2D00209A960500E82C0020BC2C002002
:107490002F2D00200CB600200DB600202E2D002030
:1074A000302D002080B4002081950500902D002013
:1074B0006C2D00202DE9F04182B0054600AF50B997
:1074C0004E4B4F49586828F020FAFFF775FD0837F2
:1074D000BD46BDE8F0812BF04AFC28B92A4649494F
:1074E000032028F017FEF2E70023391D28467B60B1
:1074F00027F0D5FA0446F0B9284629F0AFF9064638
:10750000786025F065FA06F58073834208D93E4914
:10751000012028F0FFFD3D49012028F0FBFDD6E7C2
:10752000F31D23F00703ADEB030D6C4632462146F5
:10753000284629F0B7FA7D68002DECD0072234499F
:10754000204630F009FB60B9073D07347D604FF0FD
:10755000030878681B302BF0A9F8064680B92D493E
:10756000DAE708222C49204630F0F6FA28B9083D1F
:1075700008347D604FF00408EBE74FF00008E8E7BF
:107580001E4B1F490246586827F0AEFD304626F0D4
:107590008DF9054630462BF0B1FD204B2A4603F10C
:1075A000180153F8040B42F8040B8B42F9D11B88E5
:1075B00013807E6885F819802146324605F11A004D
:1075C00030F0D8FAF3B203F108022E440133EB7520
:1075D000FE236A740020B376FFF7FCFC39460446AC
:1075E00027F05DFA28B103682B6043686B6003895C
:1075F0002B8120462BF082FD69E700BF482E00203A
:10760000E0950500FE9405007293050019950500AC
:10761000309505004195050038950500FA8805006C
:1076200010B504462BF0B8FA094B0A49002808BFE8
:1076300000242246186827F057FD201C18BF01209F
:1076400012F076FE40F2CC71BDE8104012F05ABA4A
:10765000482E00202B8A05002DE9F74F464B47495D
:1076600007460322586828F0CAFF064600283CD087
:1076700000224349DFF80881384628F0C0FF314630
:107680008146684625F0D2FC009CF4B1204628F0E3
:1076900089FE00224146054628F0B1FF0123002261
:1076A00049468246F9F730F810BBB5F80B3003F5C0
:1076B0000073A5F80B302C46504629462BF0F9FDF7
:1076C000684625F0A2FC002CDED000982BF016FDB9
:1076D0003946002C4CD001A825F0A8FC019D4DB9DD
:1076E0003246494620462BF0D7FD03B0BDE8F08F67
:1076F0000024E1E7B5F80B3003F50073A5F80B3073
:10770000284628F04FFE012229460746204627F04A
:1077100098FE1C498046284627F056F91A498246A9
:10772000284627F051F9BAF1000F00D170B1404658
:1077300028F038FE8346B0B1BAF1000F0FD0012215
:1077400039462AF0B0FC58462BF0D8FC40463A4661
:1077500029462BF0A1FD01A825F057FCBEE73946CC
:1077600028F029FFEFE73946404625F0CFFFEDE747
:10777000304627F0F7FBB3E7482E0020738B050057
:10778000CD8C05007A8B0500838B0500F8B5054686
:1077900008460C462BF0BEF90646D8B100222B490C
:1077A000204628F02CFF28F02FF900220646284911
:1077B000204628F024FF044698B12BF0A2F980B9A6
:1077C00020462BF09BFC224622490320BDE8F840CE
:1077D00028F0A0BC2CB122461F49032028F09AFCB7
:1077E000344628462BF0D8F940B33DB348F248015F
:1077F0001A4826F090FC074688B12246002127F05F
:107800000CFF2A461649384627F06EFC154B1649E0
:1078100018683A4627F068FC38462BF06FFC281CA5
:10782000314618BF012012F039F840F2DC6112F045
:1078300069F92046BDE8F8402BF060BC094B0A49C5
:10784000186828F062F80025E9E700BFE68D05001A
:107850008F8C0500ED8D0500218E0500B57D0200A1
:107860003A8E0500482E00203F8E05002DE9F84392
:1078700080460C462BF090F930B92F494246012042
:10788000BDE8F84328F046BC20462BF097F90546A2
:107890002046C5B129F078FA57EC106B0024324627
:1078A0003B46304639462FF0EBFE30B90022234BE1
:1078B000304639462FF0BCFEC8B121490120BDE851
:1078C000F84328F027BC2BF025F950B12A461D4972
:1078D000204628F094FE40B129F0B2FF06460F463C
:1078E000DDE714B122461849C9E7184F0026184DA4
:1078F000D5F804902AF09EFE16490246484627F025
:107900000CFC42461449686827F0EEFB0821134836
:1079100026F001FC054628B12146FFF737FF28462F
:107920002BF0ECFB32463B460D481CF02DFDBDE82C
:10793000F8432BF0E3BB00BF098B05000000244097
:107940005A8B0500628B0500378B050000409F4075
:10795000482E0020738B05006A8B050059760200C3
:107960006579020037B5144C00210846FFF70EFF79
:1079700003221249606828F042FE0022019010495B
:10798000606828F03CFE0D490546606827F0BDFFA1
:107990000B49606827F0B9FF019B33B12DB101237A
:1079A00001AA294600201CF0D7FD294601982BF09A
:1079B00080FC03B030BD00BF482E0020738B050053
:1079C0006A8B05001FB54FF08052D2F8A430D2F870
:1079D000A820D8B20290C3F307200190C2F3072178
:1079E000C3F3074000901B0ED2B241F0C001034820
:1079F00028F018FB05B05DF804FB00BF8F8B050075
:107A000038B52AF02DFE1E4D044628682AF0A2FD46
:107A10001C490246204627F080FB68682AF09AFD40
:107A200019490246204627F078FBA8682AF092FD03
:107A300016490246204627F070FBE8682AF08AFDC6
:107A400013490246204627F068FB28692AF082FD88
:107A500010490246204627F060FB68692AF07AFD4B
:107A60000D490246204627F058FB287E2AF06AFD81
:107A70000A490246204627F050FB204638BD00BF89
:107A8000C8B50020B7920500B0980500BA9205006D
:107A9000BE920500C2920500C6920500CA9205007A
:107AA0002DE9F04786B00D46014601A825F0BEFA43
:107AB000019838B9044601982BF020FB204606B007
:107AC000BDE8F08728F06EFC00229949064628F0B0
:107AD00096FD0746002800F0E180002294492846E0
:107AE00028F08DFD3946804602A825F09FFA012432
:107AF0000298002840F0A180414638462BF0D9FB7F
:107B000000228C49304628F07AFD0746E0B1002279
:107B10008849284628F073FD804638462BF062F9E4
:107B2000002800F0BD8040462BF05CF9002800F0F2
:107B3000B7804146384626F043F90028414638468A
:107B400008BF00242BF0B5FB00227B49304628F00B
:107B500056FD074610B300227649284628F04FFD0F
:107B6000804638462BF003F998B140462BF0FFF8D9
:107B700078B1384626F048FF8146404626F044FF5B
:107B8000814506D80123002241463846F8F7BCFD5E
:107B900000B10024414638462BF08BFB0022674998
:107BA000304628F02CFD074680B100226349284664
:107BB00028F025FD01468046384626F001F9414669
:107BC0000028384608BF00242BF073FB00225C49D4
:107BD000304628F014FD804670B12AF09BFF40B17A
:107BE000414605A825F022FADFF85491059F002FA1
:107BF00062D140462BF082FA00225249304628F0EA
:107C0000FEFC804670B12AF085FF40B1414605A8D0
:107C100025F00CFADFF830A1059F002F6CD140460B
:107C20002BF06CFA30462BF069FA01A825F0EDF93B
:107C3000002C3FF43DAF01243DE7B8F1000F10D018
:107C400028F0B0FB014603A818F004FC414604A844
:107C500025F0ECF94FF00009049838B9B9F1000F9C
:107C600000D1002402A825F0D0F941E728F09AFBC2
:107C7000014605A818F0EEFB9DF816209DF80E3081
:107C80009A4207D1BDF81420BDF80C309A4208BFC3
:107C90004FF0010904A825F0B8F9DDE701242FE72A
:107CA00038462AF0EFFD814640462AF0EBFDA9EB6D
:107CB00000035842584140E7B7F80B3003F5007312
:107CC000A7F80B3000224946284628F098FC824647
:107CD00080B10022394627F0B4FB002808BF0024F9
:107CE0002BF00CFA384651462BF0E3FA05A825F0A4
:107CF0008CF97BE70446F5E7B7F80B3003F5007322
:107D0000A7F80B3000225146284628F078FC81461F
:107D10000146384626F054F849460028384608BF40
:107D200000242BF0C6FA05A825F06FF974E700BF10
:107D30007A8B05007C950500E08A0500CD8C050056
:107D4000838B0500EB8A0500FC8A050073B50546A8
:107D50000E462AF0D6FE38B91549032028F0DAF984
:107D60000024204602B070BD30462AF0CAFE00282A
:107D7000F2D02AF05FFC04460028F2D0294601A880
:107D800025F054F901980028EBD028F00BFB0546AC
:107D900001463046FFF784FE18B12946204627F0F9
:107DA000E1F828462BF0AAF901A825F02EF9E9E719
:107DB000BA8A05002DE9F04F87B000AFC7E902018C
:107DC0001446002A6CD09149002024F057FC002270
:107DD000054638618E49204628F011FC8C49024640
:107DE000284627F09AF900228A493D69204628F062
:107DF00006FC88490246284627F08FF92AF01AFC2B
:107E000080462AF02DFC002282468349204628F035
:107E1000F6FB8146E8B102467F49386927F064F9EC
:107E2000002307F1140148467B6126F038FE044622
:107E3000002844D1484628F011FD0546786124F019
:107E4000C7FD05F5807383422ED97449012028F0BF
:107E500061F9B8F1000F07D0D8F8003023B14246DD
:107E60006F49386927F040F9504626F0EFFD20B100
:107E700052466C49386927F037F952464146484620
:107E80002BF00AFAFB68002B40F0B78007F11003D3
:107E900001220021B86823F0A3FE38692BF02EF9E7
:107EA0001C37BD46BDE8F08FEB1D23F00703ADEB9B
:107EB000030D6C462A462146484628F0F3FD7B69AF
:107EC000002BC6D0B8F1000FCED0BAF1000FC0D051
:107ED000002514E0092A09D1A91C2144701ED7F8F5
:107EE00010B02BF01AF95049024619E0911E0129F1
:107EF00027D89B4602239E4216DA013635447B6919
:107F0000AB42A6D96319665D5A78082AE2D1A91C4A
:107F10002144701ED7F810B02BF0FFF843490246F9
:107F2000584627F0FAF8E8E73BF8021F40487B6024
:107F300028F078F80146404627F040F87B68023385
:107F4000D9E7911F012908D8A81C204418F052FB3A
:107F50000146404627F032F8CFE7162A2BD0212AD7
:107F600032D1A81C204418F045FB122383463B6005
:107F7000BBF1000F1BD001225946504627F061FA91
:107F80003B6878605919701CC01A214425F0C7FA63
:107F90007A6803463AB130B101463860104625F0A0
:107FA000B5FBD7E90032194610462BF082F9584646
:107FB0002BF0A4F8A1E759881D4828F033F82AF0DF
:107FC00001FA04238346D2E7FF2A96D1D8789B781A
:107FD000D7F810B043EA00202AF0BCFA154902464F
:107FE000584627F09AF8291D2144F01ED7F810B002
:107FF00025F095FA1049024692E7D7E90301FFF709
:108000004FFD00287FF442AF47E700BFB08E050068
:10801000CD8C0500318A0500FA95050072930500A4
:108020007A8B0500838B05007C950500C08E0500CA
:1080300096BE0500FC8A0500EB8A05002DE9F0419B
:1080400086B000AF00238846391D04467B6026F0C9
:1080500026FD0546002C38D0E0B9204628F0FEFB6E
:108060000646786024F0B4FC06F58073834206D996
:108070004149012028F04EF8224640493BE0F31DDB
:1080800023F00703ADEB030D6D463246294620462B
:1080900028F008FD7B68002BEED040462AF07CFDDE
:1080A00028B1374B37491868424627F01DF8364B40
:1080B0001A6812F0400F1E460AD13449012028F0F8
:1080C00029F81837BD46BDE8F0810028E2D1D3E792
:1080D0002F4A12884FF6FF71914201D12D49EDE7E9
:1080E0001A6812F0800201D02B49E7E77C68102C57
:1080F00005DD2A491022012028F00CF8E1E7284B81
:1081000093F800C0274BA4B2BCF1000F25D19A7C94
:1081100072B3B3F8760188422CD09B8A7C80C7F872
:108120000AC0A7F80EC03B810123BB7207F108010A
:10813000BB1CC7E90435FBF793FC18B97B88A34245
:1081400018BF0C2040F6BB3111F0DCFC0028B8D180
:10815000336843F080033360B3E7B3F876018842B5
:1081600008D07C80C7F80A20FA81B3F84E31DAE7EC
:108170000720E7E70820E5E772930500368D050044
:10818000482E0020C68C0500BCB50020D08C050010
:108190006A2D0020E48C0500F38C05000B8D050092
:1081A000F9B50020F0AF00202DE9F04F9D4B91B0C4
:1081B0001B681B0700AF044607D59B49012027F029
:1081C000A9FF4437BD46BDE8F08F15F053FA2046AD
:1081D0002AF0A0FC0546002800F01A81214607F18C
:1081E000140024F023FFDFF864A2796989B1002329
:1081F000BB61B1F80B3003F50073A1F80B3007F148
:10820000180018F027F9024638B18849012027F0F4
:1082100081FF78692AF072FFD3E7D7F81480B8F1AC
:10822000000F03D0404628F0BDF88046414607F1D4
:108230001C0024F0FBFEF96985B179B1B1F80B306F
:1082400003F50073A1F80B3007F1200018F002F9D4
:10825000024670B17649012027F05CFFF8692AF0E8
:108260004DFF40462AF04AFF07F1140024F0CDFEEE
:10827000BBE707F128003C8C97F8226018F0FAF968
:1082800008B1F9F7DFFC4FF00009002207F13001D7
:10829000388DC7F8309018F0EBF9052810D043F26C
:1082A000030290420CD0A8B93B8EA34214D197F898
:1082B0003230B34210D1B7F82890B9F1000F0FD186
:1082C000386A18F0ADF95B4904460246012027F0F0
:1082D00021FF3EE0F9F7B6FC3B8D01333B85D4E747
:1082E000FC691CB1204628F05DF804460022524982
:1082F000204628F084F9002250490646204628F0FE
:108300007EF927F081FB0022B8604D49204628F015
:1083100076F927F079FBF860C6B1002307F1240154
:1083200030467B6226F0BBFB834620BB304628F0FC
:1083300095FA7862786024F04BFB7A6802F58073D6
:1083400083420ED93F49012027F0E4FE30462AF04F
:10835000D5FE20462AF0D2FE07F11C0024F055FE7F
:1083600069E7D31D23F00703ADEB030DEB46594638
:10837000304628F097FB7A6A002AE7D000217985F9
:108380003A85494607F12802BAF80000C7F82CB030
:10839000FDF712FF40F2915111F0B4FBBB6880F081
:1083A0000100C5B213B9FB68002BCFD0BAF800208A
:1083B0004FF6FF719142C9D0FB68BAF80000A7F8E8
:1083C00030900022002BC7F83220FA867A6A7A822F
:1083D00014BF0222012287F8322007F1300107F191
:1083E0001202C7E90E2BFBF73BFB30F00802ADD0C1
:1083F00043F204029042A9D043F201429042A5D038
:1084000040F2A65111F07EFB002818BF00259DE721
:10841000002C3FF4D6AE22460B49032027F07AFE0B
:10842000CFE600BFBCB50020608F0500888F050037
:10843000A18F0500D18F05006EA20500C18F050038
:10844000C88F050072930500F58F05006A2D002086
:108450002DE9F04F9BB000AF0D4604463C220021B1
:1084600007F12C00F7F75EF8022387F82C30284636
:10847000062387F82F302AF04DFB002879D0002200
:108480008449284628F0BBF838B127F0BDFA002807
:1084900014BF0223002387F82C3000227E4928468F
:1084A00028F0ADF838B127F0AFFA002814BF062342
:1084B000052387F82F3000227849284628F09FF8B6
:1084C0008146D0B1002307F10C01FB6026F0E7FAEA
:1084D000064600283CD1484628F0C0F98046F8609E
:1084E00024F076FA08F58073834225D96C4901207F
:1084F00027F010FE48462AF001FE2846002269496E
:1085000028F07DF8054640B13B6D6BB326F0AAFB21
:108510003B6D188028462AF0F1FD20462AF0F1FA3A
:1085200080B3B4F80B3003F50073A4F80B30204689
:108530006C37BD46BDE8F08F08F1070323F0070351
:10854000ADEB030D6E4642463146484628F0AAFA86
:10855000FA68002ACED084B06B464FF6FF713B65B7
:1085600019809A809E60C5E74F49032027F0D2FD0D
:10857000D0E7002DD1D04D492A46032027F0CAFD6F
:108580000024D4E720462AF09FFA05460028C8D1E7
:1085900020462AF0BFFA002876D0204625F09EF823
:1085A0000C235843073020F00700ADEB000D2146A7
:1085B00007F1080024F03AFDE846DFF8E4A044465D
:1085C000A946B868F8B987F85850C7F854801F23EF
:1085D00007F1080207F10C0107F12C003B81FCF7C1
:1085E000E5FA18B1324B5B68002BC9D040F2F63186
:1085F00011F088FA0028C3D107F10C01388924F062
:108600008EFF044693E727F0CDFE07F10C01834669
:10861000C7F80C9026F043FA0646BBF1000F10D0C5
:1086200078B9584628F01AF9F860786024F0D0F943
:108630007A6802F5807383421BD95146012027F0E6
:1086400069FD58462AF05AFDB86828B1B0F80B30D9
:1086500003F50073A0F80B3027F088F8FB68208042
:10866000A380A66007F1080024F0CFFC01350C348C
:10867000A7E7D31D23F00703ADEB030D6E4631468C
:10868000584628F00FFADCE7002CA0D02246094912
:1086900073E700BFAD8B0500B68B0500EB8A0500C4
:1086A00072930500FC8A0500C38B0500F78B05005B
:1086B000482E00202D8C050008B5064A136823F4C7
:1086C0000073136011F0ACFA40F20B21BDE80840D2
:1086D00011F018BABCB5002008B5054A136843F478
:1086E0000073136011F006F9BDE80840FEF754BBB3
:1086F000BCB5002008B512F023FC41EC100B08BDFE
:1087000010B50F4B1B884FF6FF729BB29342044685
:1087100003D10C4A1288934208D00B481EF098FEF1
:108720000A4A136843F00803136010BD2AF034FAB4
:10873000002814BF20460020BDE8104014F028BDDA
:10874000682D00206A2D0020978C0500BCB5002004
:1087500010B504462AF0DEF9224630B92CB10B4997
:108760000320BDE8104027F0D5BC094B09495868E3
:1087700027F0DCF811F044FC074B1B681B0704D5FD
:108780000020BDE81040FFF7BBBF10BDCA8E05003A
:10879000482E0020F38E0500BCB5002038B5104CE3
:1087A000104900220546606827F029FF26F0DEFF09
:1087B000C3B285B143F0010098420FD0646829F03C
:1087C000C9FE08490246204626F0A7FC0020BDE865
:1087D0003840FFF795BF03F0FE00EDE738BD00BF5E
:1087E000482E0020DC8D05002DE9F0418CB00646B6
:1087F00088462AF08FF940B93EB1324647490320F6
:1088000027F088FC0CB0BDE8F081002302930193AF
:10881000434B039302AB0593424B069303270B2371
:10882000ADF81C300DEB0703012208933E4B8DF889
:10883000032009933A4601AB03A94046ADF81070F6
:10884000ADF828700B9328F07DFD0028DAD002984F
:10885000364D374C2AF0AAFA48B1029A3549686871
:1088600026F042FC236843F00803236009E0029BE2
:10887000002B37D12F49686827F047F8236859063D
:10888000F0D402982AF03AFC9DF80330002B2ED049
:108890002368294968689A065EBF236843F0080385
:1088A000236027F032F832462449686827F03EF802
:1088B00042462349686827F039F8019A1AB12368BB
:1088C00043F0080323601F49686827F02FF80198D8
:1088D0002AF014FC236813F0180F1BD00020FFF7B8
:1088E0000FFF8FE71849384627F014FCC9E72368C3
:1088F0006F689B0648BF23684FF0000044BF43F0F9
:108900000803236029F01EFE0B490246384626F074
:1089100004FCC8E7304614F087FC73E7F58F0500C8
:10892000CC8C0500FB8E0500008F0500482E002032
:10893000BCB500200A8F0500398F0500428F050065
:108940004C8F0500568F0500148F050013B569463E
:10895000044617F0C3FD28B90749012027F0DAFBC8
:1089600002B010BD054B06495868224626F0BCFBF4
:108970000020FFF7C5FEF3E74E8D0500482E0020CE
:10898000848D050038B50A4C05462DB9094B002CDD
:1089900008BF1C46204638BD3CB120462FF024F9C4
:1089A000013D01300444EDB2EFE7024CF2E700BFB5
:1089B000158905001B02060070B50D4C064620788F
:1089C0000D4640B1FFF7DEFF0A490246012027F0BD
:1089D000A1FB002070BD09F0E1FA074B267018607A
:1089E000284629F0F9FC054B18600120F2E700BF8A
:1089F000C0B500209F890500B8B50020C4B500208F
:108A000037B50546002105208DF80610FFF7D4FF85
:108A100058B1074B186829F0DFFC01990446284635
:108A200010F0E4FF204603B030BD0446FAE700BF73
:108A3000B8B5002037B505460C4605200021FFF7E4
:108A4000BBFFB8B1214601A817F06EFC024638B151
:108A50000949012027F05EFB0024204603B030BD09
:108A6000064B186829F0B8FC01990446284610F016
:108A7000BDFFF2E70446F0E7BE8F0500B8B5002061
:108A800013B5002104208DF80610FFF795FF50B1B3
:108A9000064B186829F0A0FC0446019810F0ECFF82
:108AA000204602B010BD0446FAE700BFB8B500206A
:108AB00013B50C4604200021FFF77EFFB0B121461C
:108AC00001A817F031FC024638B10949012027F00E
:108AD00021FB0024204602B010BD064B186829F087
:108AE0007BFC0446019810F0C7FFF3E70446F1E76A
:108AF000BE8F0500B8B500202DE9FF410022884651
:108B00002649064627F07BFD00222549074627F027
:108B100076FD6946054617F0E1FC044658B929463A
:108B200038462AF0C6FB1F49032027F0F3FA2046F7
:108B300004B0BDE8F08138462AF0E0FA00221A4974
:108B4000304627F05CFD26F05FFF074620B1304637
:108B500009F084FA0446EAE731460220FFF72CFFC9
:108B600020B9002428462AF0C9FAE0E748210F4836
:108B700025F0D1FA04460028F3D00146022302AAC8
:108B80003846CDE902581BF0E7FC20462AF0B6FA39
:108B9000074B186829F020FC0446E3E7018A05002A
:108BA000CD8C0500768A0500218A0500B1BC020043
:108BB000B8B5002070B504460E4600200E4923F0DB
:108BC0005DFD054610B90025284670BD22460B49BB
:108BD00026F08AFA2846FEF715F9044628462AF0B8
:108BE0008DFA002CEFD031462046FFF785FF054671
:108BF00020462AF083FAE7E7B08E0500CD8C050009
:108C000070B5064650B129F085FF044630B92849B1
:108C10003246032027F07EFA204670BD0022254907
:108C2000304627F0ECFC054629F06BFF0446284649
:108C300024B92AF063FA2A461F49EAE72AF05EFAC5
:108C400000221E49304627F0DAFC28F0F9FD0246E2
:108C50000B4604460D462EF013FD30B900220023CA
:108C6000204629462EF0EEFC08B1154D00242B4677
:108C7000224614481BF088FB054601460120FFF7F9
:108C80009BFE78B10821104825F045FA044628B12A
:108C90003146FEF77BFD20462AF030FA0B4B186870
:108CA00029F09AFB044628462AF028FAB4E700BFC8
:108CB0005A8C05008F8C0500ED8D0500628B050038
:108CC00000409F4055B9020005BE0200B8B5002023
:108CD00030B500218FB0044609202AF01EFA164D47
:108CE0000190024680B115496868FF23CDE902135F
:108CF000002313498DF8103026F00FFA01A818F060
:108D00000AF801A818F00EF801A818F004F801A854
:108D100017F0FEFF22460B49686826F0E5F90A4B7A
:108D200002221A70B4F80B30204603F50073A4F841
:108D30000B300FB030BD00BF482E00200300FFFFF6
:108D4000EDEE0500FA94050000B6002017F050BDC6
:108D500017F092BC38B5054609B117F0FDFC0022AA
:108D60000D49284627F04BFC26F04EFE10B10B486B
:108D70002AF02BFA01460446284617F0EDFC20465F
:108D80002AF0BCF9012029F0DDFB054902462846FE
:108D9000BDE8384026F0C1B98B7D050068F80500B4
:108DA0006693050008B517F0D7FC002008BD000049
:108DB00070B58EB0044601A80E46154618F00CF8A2
:108DC00090B120460022094927F019FC044658B109
:108DD0003246074926F088F92A460649204626F0F9
:108DE00083F920462AF08AF90EB070BD2390050061
:108DF000279005003690050010B58EB0044601A8F6
:108E000017F0EAFF30B101A8214617F0A7FE01A82C
:108E100017F07EFF0EB010BD70B5064627F0C2FAFF
:108E2000054629F0B9FE044640B90E48294627F008
:108E3000C7F828462AF062F9204670BD28462AF075
:108E40005DF90949002023F019FC04460028F3D0FD
:108E5000002117F009FF32460449204626F044F964
:108E6000EAE700BF84940500FA890500AB94050089
:108E700070B5064627F096FA054629F08DFE0446A1
:108E800040B90E48294627F09BF828462AF036F9C3
:108E9000204670BD28462AF031F90949002023F008
:108EA000EDFB04460028F3D0012117F0DDFE324629
:108EB0000449204626F018F9EAE700BF849405002B
:108EC0006A930500AB94050030B591B0044603A841
:108ED0000D4617F081FF48B1002303A800932A46EE
:108EE000214617F01DFD03A817F012FF002011B056
:108EF00030BD30B58FB0044601A80D4617F06CFFA9
:108F000058B11DB129462046FFF7DEFF01A82146D2
:108F100017F024FE01A817F0FBFE0FB030BD0000D3
:108F200030B58FB0054601A817F056FFE8B1002113
:108F3000114817F0A7FE0446A0B1294601A817F072
:108F40005BFE29460122204629F094F8054670B1BF
:108F50000146204626F014FC28462AF0CFF8204689
:108F60002AF0CCF801A817F0D3FE0FB030BD0348AB
:108F700027F006F8F3E700BFB6940500BC9405009F
:108F80002DE9F04391B0804603A80F4614461E46D3
:108F900017F022FFB8B10021189827F0A3FE05466C
:108FA00029F00CFE78B3204625F05CFE8146304661
:108FB00025F058FE06461B2029F056FA044628B92B
:108FC00003A817F0A5FE11B0BDE8F08333464A466A
:108FD000394624F0B3FD0121189827F083FE064698
:108FE000284625F03FFE80B2009033462246414697
:108FF00003A817F095FCBC42E2D032462946204631
:109000002AF04AF9DCE728462AF078F825463C465B
:10901000E6E700002DE9F04F8BB08246019129F080
:10902000A6FE20B9002630460BB0BDE8F08F29F02F
:1090300017FB06460028F5D04FF000094FF0FF352A
:109040000022514605A824F039FCCB462C46A84600
:109050002F464A464B46DDE90501814200F2B680C3
:10906000B4F1FF3F08BF5C4608982AF047F8B8F112
:10907000FF3F08BFA046002F09DD7A1E00215046A1
:1090800024F089FDA3490246304626F046F8A2485E
:109090002AF09BF8A1490246304626F03EF8791C9A
:1090A000A8EB0102504624F076FD9D490246304669
:1090B00026F033F86FF000422146504624F06BFD55
:1090C000074625F0A1FC18B99649384624F08CFDD6
:1090D0003A469549304626F020F8691C14BF2A1BF1
:1090E0006FF000422146504624F055FD044625F01D
:1090F0008BFC18B98B49204624F076FD22468B491B
:10910000304626F00AF86A1C00F09E806FF000429C
:109110002946504624F03FFD02468549304625F059
:10912000FCFF09F1FF324FF6FE739A4240F2908045
:10913000022029F099F902467E49304625F0EDFFDC
:109140006B1C00F089806FF00042691C504624F0CF
:1091500022FD019B80469BB329F093FC044678BB1B
:109160000246414605A824F0A9FB29F079FA814678
:109170001B2029F079F905461B2029F075F90746CF
:10918000DDE905239A426BD3089829F0B7FF4046E2
:1091900029F0B4FF284625F037FC002800F08D8028
:1091A000284629F00FF93946054624F07BFE29466A
:1091B000484625F0F4FD394628462AF07AF8C84694
:1091C00042465D49304625F0A8FF2CE705A8CDE9C9
:1091D000022324F030F92F28DDE9022312D1B4F163
:1091E000FF3F08BF5C46012A03F1010306D1022BB1
:1091F00004D1791C02D13D463C465F46B8F1FF3FA1
:109200000DD118E03A2807D1791C02F10102F5D0FE
:10921000611CF3D1D8460EE0B8F1FF3F0ED0D8451F
:109220000CDA611C73D12F2805D9392803D83038BE
:109230000A2101FB09090BF1010B0CE73F28FAD1C8
:10924000601CF8D05D46F6E7022029F00DF963E7CF
:10925000484629F07FF96EE7022029F005F978E702
:1092600005A824F0E8F8262822D1284625F0CCFBD2
:10927000C0B1284629F0A6F83946044624F012FE6B
:109280002146484625F08BFD394620462AF011F844
:109290001B2029F0E9F805461B2029F0E5F80746D0
:1092A00000246DE7384625F0AFFB0028E1D167E7E1
:1092B00054B93D2820D1019C62E7384625F0A4FB33
:1092C00000287FF46DAF76E725280CD105A824F09F
:1092D000B2F8824605A824F0AEF80146504623F0C5
:1092E000ACFDC0B254B18DF8130001220DF1130191
:1092F000384624F060FCDEE72528E7D08DF813001F
:1093000001220DF11301284624F055FCC8E73F283F
:1093100098D090E7339605003C96050040960500EE
:10932000F6EE050036950500479605004C960500BB
:10933000559605005C960500619605002DE9F04FF5
:109340002DED028BA3B08B46154629F073F98246AA
:10935000002800F0C080584629F028FD002800F0C1
:10936000BA80284629F0D6FB002800F0908008AA91
:109370001892804A199206AA1B927F4A7F4B1C9230
:1093800004AADFF8049216931E920A237C4AADF8D1
:109390005C30002600274FF00008ADF86830ADF8CB
:1093A00074301F92ADF88030042202AB16A9284613
:1093B000CDE90867CDE90667CDE90489CDE9026703
:1093C000219327F0BFFF002800F085809DED028BE0
:1093D00032463B4651EC180B2EF020F9002851D1B3
:1093E000B0EE480AF0EE680A2BF026FD53EC102B85
:1093F000B0EE480AF0EE680ACDE900232BF00CFE2F
:10940000DDE9002355EC104BDDE9046730463946B1
:109410002DF09CFE3246804689463B46204605F1AB
:109420000041CDE90A892DF091FEDDE90823CDE95F
:109430000E01CDE91223304622462B4639462DF047
:1094400085FEDDE90623CDE90C01CDE91089CDE9E2
:1094500014230122594616A824F067FE16A823F00B
:10946000B2FD58B116A828F0FBF9064616A80F461B
:1094700025F06EFC16A823F0A6FD90BB16A823F0DD
:1094800076FD28E034463D4642464B46BCE728463A
:1094900029F08CFCC8B1284625F0D8FA06280446E5
:1094A00013D12946012216A824F03FFE0AAD16A8C2
:1094B00028F0D6F9E5E8020116A825F049FC013CA0
:1094C000F5D116A823F053FDC3E72E49032026F05B
:1094D00021FE4FF0000A504623B0BDEC028BBDE8E0
:1094E000F08F16A828F0BCF9044616A80D4625F002
:1094F0002FFCDDE90A23304639462DF027FEDDE951
:109500000E2380468946204629462DF01FFE02463E
:109510000B46404649462DF063FCDDE912232DF051
:109520005FFC41EC100B29F003F80146504625F092
:1095300045FDDDE90C23304639462DF007FEDDE917
:10954000102306460F46204629462DF0FFFD024611
:109550000B46304639462DF043FCDDE914232DF04F
:109560003FFC41EC100B28F0E3FF0146504625F08C
:1095700025FD73E711BB05001093050051BA0500E6
:10958000169305001D9305000000F03F2DE9F04FF4
:1095900093B00C46164629F04DF80546002800F019
:1095A0008480002C00F081802368062B7DD1214629
:1095B000012207A824F0B9FD01AF002407A826F076
:1095C0006FFF013447F8040B07A825F0C1FB062CF8
:1095D000F4D107A823F0CBFC304629F09BFA30B138
:1095E00000223549304627F00AF826F0BFF8DDF8AA
:1095F0000480059EDDF80890069FB8EB060448BF7E
:10960000A6EB0804B9EB070348BFA7EB09039C428C
:10961000A8BF1C46002C08BF01244FF4A04393FBB5
:10962000F4F4B4F5805F44DA40F299139C42B8BF79
:109630001C460028C8BF4FF480544A46C8BF94FB5C
:10964000F0F44146284625F0C3FCC4F5805BA246F1
:109650000BFB0BFC0AFB0BF04FEA2C3C049A40F38B
:10966000D3200CFB09F302FB0032039B0AFB0AF137
:109670000CFB08FC03FB00C3091301FB072201FBE1
:10968000063102F5006201F5006112130913284644
:10969000A24425F09DFCBAF5805FABEB040BD7DD4F
:1096A0003A463146284625F093FC284613B0BDE8DB
:1096B000F08F40F25554BCE7069205002DE9F04FBB
:1096C0009BB0014609A817F06BFE28B9002303934D
:1096D00003981BB0BDE8F08FBDF829309DF82F40EE
:1096E000DB06A4F1020347BFBDF82D70BDF82B6067
:1096F000BDF82B70BDF82D60012B70D9082CB8BFB8
:10970000082407FB04F31F33082C4FEA6313D8BF68
:109710004FF001094FEA83030093D4BF09FA04F91B
:109720004FF00009009B09EB490505F11A0803FBFE
:10973000068A504628F0BAFF03900028C6D024F0CD
:10974000B5F8422303704D2343700C2383733B12FF
:1097500080F802A0C3744FEA2A2A33124FF0010E98
:10976000082C80F803A080F80A808774067543757A
:1097700080F816E0047634DD0123A340013B069314
:10978000009A0823B3FBF4F30193E3100593731ECF
:1097900002FB0355431902934FF00008B04597DAD6
:1097A00008F101030493029B072C03F11A0547DD1E
:1097B0004FF00009B94549DA4246494609A817F071
:1097C000A0FD2A46002308339C4202F8010B4FEA11
:1097D0001020F8DC059B09F101091D44EAE7042487
:1097E0008FE79DF82F30032B00F11A0315D00021CD
:1097F0009DF82F200EFA02FC8C4503F10303BBDD1C
:10980000C1EB012292FBFCF2D2B203F8032C03F865
:10981000022C03F8012C0131EAE700224A4503F14A
:109820000303A9D042F3000103F8031C42F34001F3
:1098300003F8021C42F3800103F8011C0132EDE73A
:10984000DDF804B04FF0000ABA451CDB029B009A19
:10985000DDF810809B1A0293A0E74B1C424609A832
:10986000079317F04EFD069B1840079B09FA04F971
:1098700040EA090919465945EFD1019B05F8019BBA
:109880009A449B44E0E751464FF00009F3E700009B
:1098900038B5FFF713FF054610B90025284638BD37
:1098A0000BF08EF90446284629F028FC002CF4D051
:1098B0002146044826F0B6FB0546204629F01EFC4A
:1098C000ECE700BF5890050010B5FFF7E1FF044634
:1098D00008B11DF030FE204629F010FC0248BDE81A
:1098E00010401DF02CBE00BF67F8050000B593B016
:1098F000014601A817F054FD10B101A8FDF7E6F9E3
:1099000013B05DF804FB000000B593B0014601A858
:1099100017F046FDE8B1BDF8180010F460430AD016
:10992000B3F5005F124918BF00211A0405D429B904
:1099300028F010FE0DE00F49F7E70F49C304C0F30C
:109940000C0209D5C2F3851300F03F020B4826F044
:1099500069FB13B05DF804FB41F6FE73184203D0B7
:10996000074826F05FFBF4E7084629F02EFCF0E7F5
:10997000BD910500B6910500FF910500C19105005C
:10998000CA91050030B593B00C46014601A81546B2
:1099900017F006FD20B12A46214601A817F0B1FCB8
:1099A00013B030BD00B593B0014601A817F0F8FC24
:1099B00008B19DF80F0013B05DF804FB2DE9F041EC
:1099C000B2B00546884601460CA817F0E9FC00280D
:1099D00000F0D4800BAA1F92694A20920AAA229210
:1099E000684A694B239209AA1D9325920923674A65
:1099F000ADF87830ADF88430ADF890302692ADF8FF
:109A00009C3008AAADF8A830ADF8B43006AB289267
:109A10002E935F4A5F4B29922F9307AA0B230024B2
:109A20002B92ADF8C0305C4ABDF83770BDF8396094
:109A30008DF817400DF117034046CDE90A44CDE9F2
:109A40000844CDE906442C92319329F063F840B9DB
:109A50005249012026F05EFB0025284632B0BDE8C1
:109A6000F08107221DA9404627F06CFC0028EFD0AA
:109A70000B99099A00290A4404DA079B09925B1A98
:109A800007930B940A98089B0028034405DA06996B
:109A90000893091A069100210A91D21B002AC8BF17
:109AA00009990B98C8BF8A1AA3EB0603C8BF09928D
:109AB000002BC8BF089A0A99C4BFD31A0893079B02
:109AC000099A002B1A4404DAC31A0B930023099253
:109AD00007930698089B0028034404DA091A0A91A0
:109AE000002108930691D71B002FC8BF099A079938
:109AF0000698C8BFD71BA3EB0603C8BF0997002B66
:109B0000C2BF089AD31A0893DDE90823002B01DCB1
:109B1000002A2CDDCDE901100092DDF86B40DDE973
:109B20000A210CA8A0479DF8173003B3DDE9061001
:109B3000BDF95340099A089BA0420244B8BFADF852
:109B40005300BDF957008242C8BFADF85720BDF998
:109B500055209142BDF95920B8BFADF855100B44BE
:109B600093420CA8C8BFADF8593017F0F5FBB5F813
:109B70000B3003F50073A5F80B306EE705466CE774
:109B8000749005009FAA050071900500ACA805001F
:109B9000779005007D9005007A900500899005007A
:109BA00030B593B00D46014601A817F0F9FB002827
:109BB0004CD0BDF92720BDF92B309A4244DC28F067
:109BC0004FFD044618B3BDF9270028F0C3FC204917
:109BD0000246204625F0A1FABDF9290028F0BAFC7A
:109BE0001C490246204625F098FABDF92B0028F0C2
:109BF000B1FC19490246204625F08FFABDF92D0027
:109C000028F0A8FC15490246204625F086FAC5B181
:109C100000226FF07F038DF82B208DF82C308DF80B
:109C20002D208DF82E304FF0FF327F2301A88DF8C4
:109C300027208DF828308DF829208DF82A3017F04C
:109C40008BFB204613B030BD0024E0E70446F8E764
:109C50007190050074900500779005007A900500DA
:109C600070B592B004460D46014601A8164617F09D
:109C700097FB58B3BDF80930022D23F070039BB257
:109C80001ED0032D1FD0012D08BF43F03003ADF8C7
:109C900009304EB1BDF80930DA064CBF83F04003FD
:109CA00083F02003ADF8093001A817F055FBB4F894
:109CB0000B3003F50073A4F80B30204612B070BDD2
:109CC00043F06003E3E743F05003E0E70446F4E7C2
:109CD00070B592B004460E46014601A8154617F02D
:109CE0005FFB78B101A8ADF81A60ADF81C5017F011
:109CF00033FBB4F80B3003F50073A4F80B302046A7
:109D000012B070BD0446FAE7F0B593B004460E46B3
:109D1000014601A815461F4617F042FB08B3012E65
:109D20009DF81E10A8BF0126012DA8BF012546EAF7
:109D3000E67666F3010145EAE57565F3830187F38D
:109D4000020767F3051101A88DF81E1017F004FB38
:109D5000B4F80B3003F50073A4F80B30204613B0B1
:109D6000F0BD0446FAE700002DE9F04792B0044642
:109D70008A46014601A8914698461A9F17F010FBA3
:109D8000002859D0504628F0F2FF40B92B49012055
:109D900026F0C0F90024204612B0BDE8F087B9F1E2
:109DA000FF0F01D92649F2E7404628F0E0FF28B925
:109DB000404629F04FF808B92249E8E7C7F30726DB
:109DC000002E4FEA274308BF0126012B05DD022B99
:109DD0002CD0042B2DD01C49D9E74FF40045524616
:109DE0001A49204625F080F942461949204625F0B7
:109DF0007BF9F8B228F0AEFB16490246204625F062
:109E00008CF9484628F0A6FB13490246204625F067
:109E100084F9354401A8ADF8185017F09DFAB4F84C
:109E20000B3003F50073A4F80B30B4E74FF4204572
:109E3000D5E74FF44045D2E70446ACE7269205004B
:109E400043920500609205008A920500A8920500E1
:109E5000AD920500D0910500B2920500F0B593B027
:109E600004460F46014601A816461D4617F098FA0B
:109E7000A0B1189BADF8253001A8ADF81F70ADF862
:109E80002160ADF8235017F067FAB4F80B3003F5F2
:109E90000073A4F80B30204613B0F0BD0446FAE777
:109EA0002DE9F0419AB007460D46014609A814462F
:109EB00017F076FA4FF000080646002800F09D8063
:109EC00006AA05A909A8CDE90754CDE9058817F028
:109ED00085F908AA07A909A817F080F9059B079D2D
:109EE000089CBDF84120BDF84310BDF8450007911E
:109EF000ED1A069B0890E41ABDF82B3006929D429D
:109F0000C8BF1D46C3F10003C8BF4646AB42C8BF29
:109F10001D46BDF82D30C8BF00269C42C8BF1C4658
:109F2000C3F10003C8BF0026A342C4BF1C460026DD
:109F3000BDF83F30059346B1CDE901100092DDF840
:109F400063602246294609A8B047DDE90512BDF93C
:109F50004760DDE90730B142BDF94B60B8BFADF8ED
:109F60004710B342BDF94960C8BFADF84B30B242AB
:109F7000BDF94D60B8BFADF84920B042C8BFADF8DB
:109F80004D00002D23DD6B180D9DDDF85760CDE9E8
:109F90000005013B09A8B047002C23DD069A0D9B64
:109FA00001931444013CDDF85750079B0094059938
:109FB00009A8A84709A817F0CFF9B7F80B3003F59F
:109FC0000073A7F80B3038461AB0BDE8F081E3D033
:109FD0000D99DDF8576003F1010CCDE900010CEBA0
:109FE0000501D7E7E6D0089B0D99DDF857505A1CBC
:109FF000CDE900312244079BD9E70746E3E700009B
:10A000002DE9F04FCDB005460E46014617A817467C
:10A010000293569C17F0C4F9002800F06783382299
:10A02000002109A8F5F77EFA304628F073FD0028D4
:10A0300054D0B049304626F045FD00284ED0314678
:10A0400028A817F0ADF9002800F0A8809DF8A4809A
:10A05000B8F1000F40F0A280BDF8A7300993BDF819
:10A06000A930A5490A9342469DF8AB300B93304680
:10A0700026F0C5FA064623F0FDFB0E90304629F087
:10A080003DF8CDF83C809DF8303013B94FF0FF33E8
:10A090000D93109B5BB90B9B012B08D11B9AADF85C
:10A0A00054201A9AADF8562015AACDE910230E981F
:10A0B00028F05DFE064648B10999002906DD0A9B95
:10A0C000002B03DD0B9B202B40F32C818B490120BF
:10A0D00026F020F80E9829F011F85FE0304628F0BD
:10A0E00019FD002872D000228549304626F087FAF3
:10A0F00025F03CFB002283490990304626F07FFA88
:10A1000025F034FB002280490A90304626F077FA89
:10A1100025F02CFB0028CCBF0B9001234FF0000250
:10A120007A49D8BF0B93304626F069FA031C18BF52
:10A1300001238DF8303025F019FB00220D90744971
:10A14000304626F05CFA804688B328F0BDFC50B358
:10A15000B8F80430022B26D1002328A940462893C2
:10A1600024F09DFC1090404628F0C8FF289B102B3F
:10A1700005D9B3F5807F06D00023109305E0654A2A
:10A18000DA40D107F8D5013B1193DDF84080B8F1F2
:10A19000000F0CD16049012025F0BCFF00252846A6
:10A1A0004DB0BDE8F08F404628F0A8FFEDE7002253
:10A1B0005149304626F023FA064623F05BFB0E9009
:10A1C000304628F09BFF00230F935CE7304628F0D1
:10A1D000CEFD58B1304628F077FC70B9B6F80B3098
:10A1E0000E9603F50073A6F80B300AE0304628F00F
:10A1F0006BFC0028EED14949CDE7304623F03AFB0D
:10A200000E9000210E9823F081FC012109900E98F8
:10A2100023F07CFC02210A900E9823F077FC0206C2
:10A220000B902CD500F07F0001230B9003210E989A
:10A230008DF8303023F06AFC04230D900B9E0F93B1
:10A2400073067FF520AF06F03F064FF0010808FACD
:10A2500006F808F1FF39022E0B96CDF8449028DC61
:10A26000DDF83C9015AB4FF0000AD04509DC15AB8A
:10A270001093022303FA06F60F9B3344A4E703234B
:10A28000DCE749460E98039323F040FC09F10202F3
:10A29000834609F101010E98009223F037FC039BDD
:10A2A000009A4BEA002023F8020B0AF1010A9146BA
:10A2B000DBE7082E16DC002328A90E982893DDF88A
:10A2C0003C8024F0ECFB0B9B082B0BDC50B10223F1
:10A2D000B340289A434493423FBF0F9BCDF844902C
:10A2E000C0181090DDF84080B8F1000FC1D10C49C2
:10A2F00051E700BFAC9005001EA805008C91050039
:10A30000B5900500BB900500C2900500C690050001
:10A31000D290050014010100DA9005005791050064
:10A320002591050001229A40013A072B1292DCBFC9
:10A33000082292FBF3F203FB01F3D4BF02F1FF32D8
:10A34000002207331392DB10DDE90E1204A81493E8
:10A3500023F0B4FA002C40F08C80BDF8613013F08B
:10A36000700F1AD0DFF89CA3029E4FF000084446FD
:10A370000A9B029A1344B34279DC079828F0BEFE88
:10A380000E9828F0BBFE17A816F0E6FFB5F80B30C4
:10A3900003F50073A5F80B3001E7BDF87700BDF8B1
:10A3A0007910029B099ABDF87DC08742B4BF34463C
:10A3B00038463A448B42BDF87B30A8BF029902F17F
:10A3C000FF3EB8BF34469E45C8BF9E460A9A029BD0
:10A3D000134403F1FF33C8BF34466345C8BF634627
:10A3E000BDF97FC0BDF98120C8BF34468445C8BFD0
:10A3F000ADF87F00BDF98300C8BF34467045BCBFCF
:10A400003446ADF883E08A42BDF98520C4BFADF87B
:10A41000811034469A4202DAADF88530A2E7002C6A
:10A42000A0D1DDF88BA09FE704A823F004F808343E
:10A4300040EA08280B9BA342F6DC129AE41A28FA99
:10A4400004F313400D9A9A4209D0109A1AB1119947
:10A450000B4032F813303246494617A8D04709F16D
:10A460000109099B3B444B45E4DC013680E7B946D2
:10A47000F7E7204628F04EFB00283FF47EAF00228D
:10A480009D49204626F0BBF827F0DAF9824621F0F4
:10A4900000498B464FF0FF32984B504649462DF00D
:10A4A000EFF870B94FF0FF32944B504649462DF00B
:10A4B000DDF830B900220023504659462DF0C2F88D
:10A4C00018B1DFF844B24FF0000A00228C49204650
:10A4D00026F095F827F0B4F9CDE90001DDE9008315
:10A4E00023F000494FF0FF32844B404649464FF07D
:10A4F00001042DF0C5F840B94FF0FF327F4B4046C4
:10A5000049462DF0B3F800B9044684F001044FF039
:10A51000FF327A4B40464946E4B22DF0B1F838B9E3
:10A520004FF0FF32754B404649462DF09FF818B169
:10A530009FED6F7B8DED007B029B299309AE0FCEC3
:10A54000289731AF0FC70FCE0FC70FCE0FC796E8B2
:10A55000030004AE87E803000FCE3FAF0FC79DEDA9
:10A56000007B33683B6028A80023CDE92EAB8DED3E
:10A570002C7B8DF8C0408DF8C130F7F7A3F8BDF8FB
:10A580007780289BBDF879402A9F2B9E9845B8BFBD
:10A590009846299B9C42B8BF1C46BDF87B30013FC2
:10A5A0009F42A8BF1F46BDF87D30013E9E42A8BF16
:10A5B0001E46BDF97F309845BDF98330B8BFADF870
:10A5C0007F809F42BDF98130C8BFADF88370A34240
:10A5D000BDF98530C8BFADF881402246B34241463F
:10A5E00028A8B8BFADF88560FCF7A1F9BDF86130C7
:10A5F00013F0700F0CBFDDF88BA0DFF808A1B44298
:10A6000006DD3FAE0FCE04AC0FC433682360B4E662
:10A6100028A8FCF783F9C146B94504DD28A8FCF752
:10A6200054F90134EBE74A9A7F322BD44B9B13F158
:10A630007F0B27D4449B9A4224DA459B9B4521DA21
:10A640004FEA222C339A082A4FEA2B2BDDE93610E9
:10A6500023D13C9A0CEB000302FB0B323FA823F002
:10A66000AFF9439B0BB13F9A9B5C359A9A4209D054
:10A67000389A1AB139990B4032F8133022464946BC
:10A6800017A8D0474A9B469A13444A93479A4B9B34
:10A690009B1A4B9309F10109BEE7319B03FB0BCBDE
:10A6A0000BFB02F200EBE2023FA823F089F9439B87
:10A6B0000BB13F9A9B5C08213398814207DB3B9AA0
:10A6C00022EA0B0250433A9AC3401340CDE73FA819
:10A6D0000091029322F048FD029B439A00991B02CD
:10A6E0000AB13F98125C13430831E5E7054656E589
:10A6F000000000000000000010930500FFFFEF7F46
:10A70000169305003B1304000000F03F70B594B0B1
:10A7100004460E46014603A8154616F041FEC0B198
:10A720003346BDF92420BDF92210009503A816F088
:10A7300073FD03A8ADF82260ADF8245016F00CFEAE
:10A74000B4F80B3003F50073A4F80B30204614B0B6
:10A7500070BD0446FAE7F0B595B004460D460146D3
:10A7600003A816461F4616F01BFE98B11A9B0093CD
:10A7700032463B46294603A816F04EFD03A816F0C4
:10A78000EBFDB4F80B3003F50073A4F80B30204652
:10A7900015B0F0BD0446FAE72DE9F04F99B0074631
:10A7A0000E46014607A816F0FBFD00283AD0BDF87A
:10A7B000304004F46048E3040FFA88FA54BFC4F34D
:10A7C0000C0404F03F04BAF1000F2EDA00223149E4
:10A7D000384625F014FF00222F490546384625F05B
:10A7E0000EFF24F0C3FF0746304625F03FF9002254
:10A7F0000146814602A823F061F80026A3000093D9
:10A80000B346DDE902218A4212D3059828F076FC8E
:10A81000284628F073FC484628F070FCB34558469B
:10A82000B8BF304619B0BDE8F08F00273D46DBE7E2
:10A83000069939B1895C0A2904D15E45B8BF5E46E4
:10A840004FF0000BB8F1000F07D12046F6F7EEFDF0
:10A85000834402A822F088FCD3E7B8F5005F02D158
:10A86000009B9B44F5E7BAF1000FF2DA284601910C
:10A8700028F07DFA48B10199B942EADBC91B2846A4
:10A8800023F044F900FB04BBE3E7284624F0EAF98F
:10A89000F8E700BFAD920500B2920500F0B595B0A3
:10A8A00004460D46014603A816461F4616F078FDDD
:10A8B000A8B1079B01931A9B009332463B46294659
:10A8C00003A816F006FD03A816F046FDB4F80B30F9
:10A8D00003F50073A4F80B30204615B0F0BD044614
:10A8E000FAE7F0B595B004460D46014603A81646B2
:10A8F0001F4616F055FDA8B1069B01931A9B0093C5
:10A9000032463B46294603A816F0E3FC03A816F09E
:10A9100023FDB4F80B3003F50073A4F80B30204688
:10A9200015B0F0BD0446FAE72DE9F04FE5B00D464D
:10A9300005901C4601469DF8B831199328A8924607
:10A9400016F02EFD002800F0B082BDF8B430D90416
:10A9500003F46042C3F30C09099228A843BFC9F36A
:10A960008512069203F03F09CDF81890FCF7AEF976
:10A97000BDF924301090002B159380F29280099B32
:10A98000B3F5204F00F08B80B3F5404F14BF012387
:10A9900004230022AF490598079325F030FE0022DA
:10A9A0001290AD49059825F02AFE00220A90AB4985
:10A9B000059825F024FE24F0D9FE08909DF8BA20D1
:10A9C000BDF8A530ADF8683002F03002102A9BB215
:10A9D0006FD183F03003BDF8A720ADF8A5300AF1A0
:10A9E0000103A246D41A9DF8BA3003F00303012BE9
:10A9F0000DD829460598FFF7CFFE9DF8BA3003F031
:10AA0000030303FB000000EBD070AAEB600A9DF883
:10AA1000BA30C3F38103012B9FBF109A03FB0223BB
:10AA200003EBD373A4EB6304BDF8BB300E93BDF806
:10AA3000BD300C93BDF8BF300D93BDF8C1300B9302
:10AA4000BDF8A530DB0607D50E9B0C9A0E920C9331
:10AA50000D9A0B9B0D930B92284625F007F80022C8
:10AA60001690014623A822F029FF079A012393405C
:10AA7000013B1D934FEA89031C93C2F1080356461C
:10AA80002193DDE923239A4244D223A822F0D3FC68
:10AA90000A2805462BD1109B56461C44F1E7022399
:10AAA00077E701230022CDE9073200230A931293AE
:10AAB00084E7202A0ED183F06003BDF8A720ADF80B
:10AAC000A5300AF10103A2EB030ABDF8A930013455
:10AAD0001C1B88E7302A86D183F05003BDF8A920DB
:10AAE000ADF8A530631C5446A2EB030A7BE7099B33
:10AAF000002B40F08F8001464846F6F797FC0E9BEE
:10AB00000F901B1AB34222DB0F9B1E4421F058FF0B
:10AB10000028B6D0269828F0F1FA169828F0EEFA18
:10AB20000A99129828F0C5FBBDF86830ADF8A53039
:10AB300028A816F011FC059B059AB3F80B3003F515
:10AB40000073A2F80B30059865B0BDE8F08F0D9B3F
:10AB50009E42D9DA0C9B069A9B1AA342D4DA0B9B2D
:10AB60009C42D1DA202DCFD93D49099AA5F1210384
:10AB70003C4DDBB20846D7B29F422AD3C75C002DBA
:10AB8000C2D023014FEA0618083BA8F10808119328
:10AB90002F444FF00D0BBD42B6D015F8011BC8294C
:10ABA00021D8314B314A5B5C18932F4B00205FFA60
:10ABB00080FE8E4512D3189B39A802EB030C9445F6
:10ABC00000F1040011D139AA189928A816F088F9C3
:10ABD000E1E711F8017B01323D44CCE713F801EBCA
:10ABE00001307244E3E70022E5E712F801EB069B2F
:10ABF000BEFBFBF10BFB11EE023911FB03F1119BC4
:10AC00005FFA8EFE0EFB098E194420F804EC20F842
:10AC1000021CD4E7099BB3F5005F29D10E9B033BCF
:10AC2000B34214DC0D9B9E4211DA0C9B053BA34200
:10AC30000DDC0B9B9C420ADA199B0293069B224671
:10AC4000CDE900933146034628A816F0BDFD1C9BB4
:10AC50005BE700BFA8920500AD920500B292050027
:10AC60008B7E05006A7F0500C58005008E8105008A
:10AC7000159B002BBFF64AAF0A9828F078F80028F9
:10AC800060D0089BAB4200F30D810DF1E408002277
:10AC90000A99404622F012FE089B0027ED1ADDE9D2
:10ACA00039239A4203D23B9B1344AB4243DB3D9B87
:10ACB000002B45D013F802803C9828F01FFA0E9B19
:10ACC000A3EB0803B34247DA0D9B9E4244DA0C9B88
:10ACD000109A9B1AA3423FDA0B9B9C423CDA134624
:10ACE000069A93FBF2F3079A179353435F43FA10C4
:10ACF000129939A822F0E2FD3D9D07F007070DB13A
:10AD0000399BED5C079B7B439D4006EB0903119348
:10AD100000231393139B434580F2C080119BA3EB48
:10AD200009032093119B013B1F93069BE3180F938C
:10AD30000023149378E0404622F07DFB0744AEE701
:10AD40009846B9E70A9823F08DFF089BEF1AAB42AB
:10AD5000804600FB07F7B2DD08FB0966D6E6219BBB
:10AD6000E8B21841199B0BB9002851D0069A0F9BE5
:10AD70009DF8ABC09B1A1B930F9B013B1E930002D7
:10AD80001D9BB0FBF3F0B0F5807F0146A8BF4FF4E8
:10AD90008071BCF1080FDDE92B3223D9BCF1100F13
:10ADA0004DD1C3F34510C1F5807EC2F3451C484325
:10ADB000C3F3C42B0EFB0C0C01FB0BFBC2F3C42032
:10ADC0000EFB00B0000A03F01F034B434FEA1C2C9C
:10ADD000C00202F01F0240EA4C1C0EFB02324CEA99
:10ADE00012230CE04FF48A7E2EFA0CFC1CF0010FAB
:10ADF00047D0C1F580704B4302FB00331B0A01931F
:10AE00001E9B00931B9A1F9B209928A816F061FA9D
:10AE1000079B1F44072F38DC9D40149B069A013383
:10AE200014930F9B13440F93149B179A934296DB32
:10AE3000139B01331393119B4B4411936AE7BCF1AD
:10AE4000180F1ED1C3F30720C1F5807EC2F3072C73
:10AE500048435FFA83FBC3F307430EFB0C0C01FB73
:10AE60000BFBD0B24B43C2F307422CF0FF0C0EFB9E
:10AE700000B00EFB02334CEA10201B0A40EA0343E9
:10AE8000BDE77F28D8BF1346B9E739A822F06CF98F
:10AE90003D9D0DB1399BED5C0027BEE73C9828F045
:10AEA0002DF959E74FF0000856E705904BE600BF33
:10AEB00030B595B00546014603A816F071FAA0B169
:10AEC00027F0B8FB044668B1094828F07EF901462E
:10AED000204624F073F801220094064B11462846C0
:10AEE00007F048FB204615B030BD0446FAE700BF26
:10AEF000BD910500F9AE020038B5054608460C467E
:10AF000023F082FD072824D901221249204623F08C
:10AF100053FDF0B11049204623F056FDC8B90F4942
:10AF2000204623F051FDA0B90D49204623F04CFDE9
:10AF300078B96FF000420721204622F02CFE04462B
:10AF40000146284624F00EF82046BDE8384028F097
:10AF5000D5B838BDD5910500DD910500EB91050010
:10AF6000F8910500000000002DE9F04F97B09046E1
:10AF70000191014605A81F4616F012FA002856D086
:10AF8000019827F0F4FE002879D00023092202A9B5
:10AF900001988DF81030CDE9023323F0EFFD9DF8D4
:10AFA0000C609DF809009DF80A909DF80B70002E2A
:10AFB00040D121F02DFF2CF05FF80022904B2CF0B7
:10AFC000EFF9044648460D4621F022FF2CF054F8D4
:10AFD00000228B4B2CF0E4F9824638468B4621F058
:10AFE00017FF2CF049F8864B00222CF0D9F90022EB
:10AFF00006460F460023204629462CF019FB88B947
:10B0000000220023504659462CF012FB50B9002272
:10B010000023304639462CF00BFB18B99DF80F3051
:10B02000002B3BD00120774925F074F8002017B0A1
:10B03000BDE8F08F494621F000FF2CF01DF86EA30B
:10B04000D3E900232CF0ACF904460D4638463146CE
:10B0500021F0F3FE2CF010F867A3D3E900232CF0C5
:10B060009FF982468B469DF80D009DF80E1021F049
:10B07000E4FE2CF001F860A3D3E90023B5E70198C2
:10B0800025F082FE404655EC104B25F07DFE3846FB
:10B090005BEC10AB25F078FE57EC106B25F0004907
:10B0A0004FF0FF32584B204649462CF0E9FA002871
:10B0B00040F09E804FF0FF32534B204649462CF023
:10B0C000D5FA002840F094802BF000494FF0FF3271
:10B0D0004D4B504649462CF0D3FA002840F088806A
:10B0E0004FF0FF32484B504649462CF0BFFA00283B
:10B0F0007ED127F000494FF0FF32434B304649469E
:10B100002CF0BEFA002873D14FF0FF323E4B304690
:10B1100049462CF0ABFA00286AD100223B4B20466E
:10B1200029462CF013F82CF0C1FA0022374B0446C4
:10B13000594650462CF00AF82CF0B8FA0022334B4E
:10B140000546394630462CF001F82CF0AFFABDF830
:10B15000191011F4607184F3080385F3080280F379
:10B16000080008D0B1F5C07F19D010D880291AD0B6
:10B17000B1F5807F1CD09DF81F1010291FD19110B0
:10B18000DA10D20242EA411242EAE0004FE7B1F59A
:10B19000007F11D0B1F5207FEDD1114601E01946B5
:10B1A0001346024606E01946034610460A46E2E701
:10B1B000194603460846DEE719461346F6E72029F6
:10B1C00006D11B0443EA0223034343F07F402EE7EA
:10B1D000182904D11B0443EA0223184327E7134428
:10B1E0000344B3F5C07F4FF0FF30B8BF00201EE727
:10B1F000019823F037FD1AE70000000000E06F40DF
:10B2000000002E40CF920500FFFFEF7F000070404E
:10B2100070B5044608460D4627F07CFC002875D022
:10B2200000223E49284625F0EAF9064650B100239F
:10B230001A4601462046FFF797FE394B1860304604
:10B2400027F05CFF00223749284625F0D8F906464A
:10B2500050B100231A4601462046FFF785FE304BC9
:10B260005860304627F04AFF00222F49284625F033
:10B27000C6F9064650B100231A4601462046FFF79C
:10B2800073FE274B9860304627F038FF002227498D
:10B29000284625F0B4F9064650B100231A46014667
:10B2A0002046FFF761FE1E4BD860304627F026FF90
:10B2B00000221F49284625F0A2F9064650B1002376
:10B2C0001A4601462046FFF74FFE154B18613046DF
:10B2D00027F014FF00221749284625F090F906466A
:10B2E00050B100231A4601462046FFF73DFE0C4BA5
:10B2F0005861304627F002FF00220F49284625F00A
:10B300007EF918B124F080FB054B1876B4F80B30A9
:10B3100003F50073A4F80B30204670BDB79205000A
:10B32000C8B50020B0980500BA920500BE9205008D
:10B33000C2920500C6920500CA920500F0B593B00E
:10B3400004460E46014601A815461F4616F028F889
:10B35000F0B1AFB9049B2A46314601A815F0EDFFC4
:10B3600001A8ADF81A60ADF81C5015F0F5FFB4F85F
:10B370000B3003F50073A4F80B30204613B0F0BD7A
:10B3800000231A4639462046FFF7EEFD0346E2E762
:10B390000446F2E72DE9F04F9DB00BAD80460F4615
:10B3A0000146284616461C4615F0FAFF0290002872
:10B3B00000F09B80269B0A9308AA07A92846CDE99E
:10B3C0000776099415F00AFF0AAA09A9284615F07C
:10B3D00005FF0798099B08990A9CC21802EBD272D4
:10B3E00052101B1A009203EBD3730A19641A5B10F4
:10B3F00004EBD474641005935B43039302EBD272A5
:10B4000004FB04F3521004930192DDE90332660059
:10B41000013E03FB16260027009B03EB070B019B55
:10B4200003EB040A52460E9B5946284615F044FE8B
:10B43000009BA3EB070952460E9B4946284615F090
:10B440003BFE019BA3EB040A52460E9B594628463D
:10B4500015F032FE28460E9B5246494615F02CFE4A
:10B46000049A7B0003FB022271009142BFBF049A41
:10B470000298033302FB03664FEA440C039BCCF1B2
:10B48000010203FB02F2B4BF01370020914208DD44
:10B49000039AACF10303013C02FB1366002CBBDAF8
:10B4A00001E00028FAD1059BBB4207F101040CDC46
:10B4B000284615F051FFB8F80B3003F50073A8F8D3
:10B4C0000B3040461DB0BDE8F08FDDE900120E9B49
:10B4D0002144284615F0F0FDDDE900120E9B091B02
:10B4E000284615F0E9FD2746DDE7DDF80880E8E7A6
:10B4F00013B51C4613440093121B0B19091BFFF7CD
:10B5000049FF02B010BD2DE9F04F9FB00DF1340A94
:10B5100080460E460146504615461C4615F040FF33
:10B520000390002800F08980289B0C930AAA09A99F
:10B530005046CDE909650B9415F050FE0CAA0BA9F5
:10B54000504615F04BFE09990B9B0C9CCDF818A0AA
:10B55000CA1802EBD272521002920A9A1519A41A52
:10B560005B1A04EBD474641003EBD3735B106600B6
:10B5700005EBD575059304FB04F95B43013E6D10A3
:10B58000049303FB169600277B0003FB09927100CE
:10B590009142BCBF033309FB03660498B8BF039A0A
:10B5A0004FEA44030793C3F1010300FB03F3B4BF65
:10B5B0000137002299421FDD029B069803EB070A20
:10B5C000A3EB070B109B2A19CDE9002351465B46DC
:10B5D00015F036FC109B06982A1BCDE90023514636
:10B5E0005B4615F02DFC079B049A033B013C02FBD4
:10B5F0001366002CC8DA01E0002AFAD1059BBB4291
:10B6000007F101040CDC0DA815F0A6FEB8F80B300C
:10B6100003F50073A8F80B3040461FB0BDE8F08F6B
:10B62000109B0299CDE90053029B2A461B1B214423
:10B630000DA815F005FC2746E0E7DDF80C80EBE7E8
:10B6400013B51C4613440093121B0B19091BFFF77B
:10B650005AFF02B010BDF0B599B004460F4601463E
:10B6600007A816461D4615F09BFE002840D01E9BDD
:10B67000069304AA03A907A8CDE90376059515F05A
:10B68000ADFD06AA05A907A815F0A8FD049A0A9B16
:10B690000399CDE9002307A8059B15F0D1FB0A9B70
:10B6A0000193069B0093DDE9042307A8194615F0D2
:10B6B000C7FB069A0A9B0399CDE9002307A8059BBF
:10B6C00015F0BEFB0A9B0193049B0093039B069A13
:10B6D000194607A815F0B4FB07A815F03DFEB4F80D
:10B6E0000B3003F50073A4F80B30204619B0F0BD01
:10B6F0000446FAE72DE9F0478AB0804627F037FB89
:10B70000044638B94849032024F004FD20460AB015
:10B71000BDE8F08700224146684622F0CFF80027B6
:10B720003D463E463C464FF00009DDE900329A4274
:10B7300025D8039827F0E2FC26F092FF0446002863
:10B74000E4D0304626F006FF38490246204623F072
:10B75000E4FC284626F0FEFE35490246204623F04A
:10B76000DCFC05FB06F007300021C01027F0D5FCFB
:10B770000546C0B9204627F0C1FC2C46C6E76846FE
:10B7800021F059FE0A2805D159EA040308BF012710
:10B790000134C8E7AC4209F10109A8BF651C4E4558
:10B7A000B8BF4E46C1E73A464146684622F086F8A1
:10B7B0004FF0000847464FF08009DDE900239A4228
:10B7C00008D3039827F09AFC2A461A49204623F00A
:10B7D000A4FC9BE7684621F02EFE0A2803D108F15D
:10B7E00001080027E9E720281CD0284627F0BFFAE7
:10B7F000C0B106FB087A29464FEADA0205A822F012
:10B800005DF8099909B1059BC95C0AF0070A49FA74
:10B810000AFA41EA0A0105A8C9B221F0BBFD08985D
:10B8200027F06CFC0137C8E799900500B59005003A
:10B83000BB9005001EA80500024B03495868002272
:10B8400024F0DDBE482E00209589050070B5174B09
:10B850001C7884420DD0FDF795F805462046FDF78B
:10B8600091F82A46034612490420BDE8704024F0AE
:10B8700051BC104C00201870206840B189B11146AD
:10B8800003F05EFF206827F039FC002323600A4C98
:10B89000206827F033FC00232360084B01221A7034
:10B8A00070BD114604F094F8ECE700BFC0B500206D
:10B8B00064890500B8B50020C4B50020E1B50020BA
:10B8C00010B50A460C460021FFF7C0FF2046BDE830
:10B8D000104027F013BC000038B5194D2A884FF6E8
:10B8E000FF719142044613D001460320FDF764F82E
:10B8F00018B1144B186826F06FFD044613212888F0
:10B90000F9F7ACF840F66B410EF0FCF8204638BD74
:10B910000D4B1D78022D0DD10C4827F056FC014629
:10B920002846FFF7CDFFFAF7CCFF2046BDE83840A8
:10B9300006F094BB0649012024F0ECFBF5E700BFBC
:10B94000682D0020B8B50020C0B50020088A050089
:10B950001D8A050010B5094B1C78012C0CD1002163
:10B960000846FBF713FF064827F02FFC0146204648
:10B97000BDE81040FFF7A4BF10BD00BFC0B5002058
:10B98000768C05000A460021FFF760BFF7B500225C
:10B990003449044624F033FE23F0E8FE324B3349A9
:10B9A00006460322586824F02AFE054630B1224696
:10B9B000B1B223F020FB284627F0A0FB00222C493F
:10B9C000204624F01CFE0746002839D121460820D5
:10B9D000FCF7F2FF18B90025284603B0F0BD254B4F
:10B9E000254E186826F0F8FC33884FF6FF729A420D
:10B9F000054607D1214827F0E8FB01460820FFF75C
:10BA00005FFFE9E73A461749204624F0F8FD23F0A6
:10BA1000ADFE013080B2ADF80400ADF8060001A91A
:10BA200030880EF07DFC0DF07DFF04460028D3D059
:10BA300001460820FFF7A6FF204627F05FFBCBE773
:10BA400027F05CFB00210920FCF7B6FF0028C2D0DC
:10BA5000084B186826F0C0FC0121054620460EF070
:10BA6000EFFBB9E7428A0500482E00204F8A050007
:10BA7000368A0500B8B50020682D00201D8A050013
:10BA800070B5014606460720FCF796FF68B3184BD1
:10BA9000184D186826F0A0FC2B884FF6FF729A42CA
:10BAA000044608D1144827F090FB01460720FFF711
:10BAB00007FF204670BD00221049304624F09FFD4C
:10BAC00023F054FE2B8881B2002218460EF026FC8B
:10BAD0000DF028FF05460028EBD001460720FFF7B0
:10BAE00051FF284627F00AFBE3E70446E1E700BFE1
:10BAF000B8B50020682D00201D8A0500428A050087
:10BB00002DE9F04F85B00D4600AF00238046394641
:10BB100028463B6022F0C3FF0446002D39D0F8B917
:10BB2000284624F09BFE0646386020F051FF06F5BB
:10BB30008073834209D93749012024F0EBFA0026AB
:10BB400030461437BD46BDE8F08FF31D23F00703E0
:10BB5000ADEB030D6C4632462146284624F0A2FF89
:10BB600000210620FCF728FF0028E8D02A4B2B4DA7
:10BB7000186826F031FC2B884FF6FF729A42064671
:10BB80000AD1274827F021FB01460620FFF798FE3F
:10BB9000D6E70028E4D1D2E700222249D7F8009066
:10BBA000404624F02CFD23F0E1FD00221FFA80FA2C
:10BBB0001D49404624F023FD834640B300221B4923
:10BBC00024F01DFD23F020FF8046584627F096FA0A
:10BBD000002398453B8114BF022301233B71391D8B
:10BBE000012328887B71FC60A7F806A0A7F80A90BB
:10BBF0000EF024FB0DF096FE04460028A0D001466E
:10BC00000620FFF7BFFE204627F078FA98E7804627
:10BC1000DEE700BF72930500B8B50020682D002054
:10BC20001D8A0500428A0500568A0500618A0500C2
:10BC300038B50D4601460A20FCF7BEFE60B3174B2F
:10BC4000186826F0C9FB164B1A884FF6FF7191420F
:10BC5000044608D1134827F0B8FA01460A20FFF736
:10BC60002FFE204638BD18880F4B1B7880B28BB151
:10BC700000232A461946F8F7B9FC0DF053FE054695
:10BC80000028EED001460A20FFF77CFE284627F068
:10BC900035FAE6E70820F0E70446E2E7B8B5002009
:10BCA000682D00201D8A050070B1002000000000F2
:10BCB000F0B58BB06D460C46294614F00FFC0028F9
:10BCC00000F084800022012395E80300ADF81820DD
:10BCD0008DF81830A023ADF81A303F4BADF80C109A
:10BCE000CDE907323D4B0290090C58688DF80E10D3
:10BCF0003B49099224F083FC23F038FDC3074CBF75
:10BD0000384B394B089320464FF0C873099326F0FF
:10BD100001FF002841D000223449204624F06FFC66
:10BD200025F08EFD02460B4606460F462BF0A8FC7A
:10BD300090B900222E4B304639462BF007FA24A347
:10BD4000D3E900232BF02CFB00222A4B2BF048F8E0
:10BD50002BF0D4FCADF8200000222749204624F027
:10BD60004EFC25F06DFD02460B4604460D462BF0B9
:10BD700087FC90B900221E4B204629462BF0E6F99D
:10BD800013A3D3E900232BF00BFB0022194B2BF05C
:10BD900027F82BF0B3FCADF8220002AB93E80300C8
:10BDA000ADF81410090C04908DF8161008AA06A915
:10BDB00004A80EF0B7FA0DF0B5FD044630B1014607
:10BDC0000220FFF7DFFD204627F098F90BB0F0BD09
:10BDD000000000000088934090000400482E0020DE
:10BDE000DC8D0500900120031000A000C48D05002B
:10BDF00000408F400000E03FD08D05000A46012141
:10BE0000FFF724BD70B50D4B1C78012C054613D1EE
:10BE100000210846FBF7BAFC2146094826F00DFC34
:10BE2000064608F081FB304627F068F9294620468F
:10BE3000BDE87040FFF7E2BF70BD00BFC0B5002095
:10BE4000C4B500207CDF70472DE9F04F964C85B0DB
:10BE5000236800AF054603F0040308460E463B6026
:10BE600026F058FE002800F0AB8000228F493046B3
:10BE700024F0C5FBB0B123F079FC4FF47A7358433A
:10BE800040F2712390FBF3F080B2B0F5804F884B05
:10BE900028BF4FF4804020281A8838BF20208242D3
:10BEA00018BF188000228349304624F0A8FB38B11F
:10BEB00023F0AAFD2368002862D023F400632360E6
:10BEC00000227D49304624F09AFB38B123F09CFDD6
:10BED0002368002857D023F4805323600022774939
:10BEE000304624F08CFB8146002873D0002307F1F4
:10BEF0000C01FB6022F0D3FD8046002852D1484659
:10BF000024F0ACFC8246F86020F062FD0AF58073F4
:10BF100083423BD96A49012024F0FCF8484627F0C7
:10BF2000EDF8284626F0F6FD814608B9002D54D1DB
:10BF300031462846FCF78CFA002D40F0B2800025EF
:10BF4000604C614960682A4623F0F0FC32465F4944
:10BF5000606823F0EBFC284627F0D0F83B680BB173
:10BF60000DF0C8FC4FF45B7140460DF0CBFD3B6813
:10BF700063B30DF055FE40F26E310DF0C3FD25E0C8
:10BF800043F400639BE743F48053A6E70AF10703F9
:10BF900023F00703ADEB030DE84652464146484601
:10BFA00024F080FD11234146BA893B7207F1080055
:10BFB000FFF748FF40F22D3180460DF0A3FDADE7BD
:10BFC00046B132464249032024F0A4F81437BD4656
:10BFD000BDE8F08F4FF00008A3E7284626F091FD5A
:10BFE000786000284BD0B5F80B3003F50073A5F846
:10BFF0000B30236823F07F7323F40033294607F1C5
:10C000000C00236021F012F8CB46F86850B9B9F162
:10C01000000F95D0BBF1010F92DD236843F400338C
:10C0200023608DE724F0BEF9824626F073FD10B937
:10C03000BAF1000F0FD131465046FCF709FA81469C
:10C04000F86810B1494621F061FB484627F056F8E0
:10C05000D7F8049009E0504626F053FD0028F7D1A8
:10C06000504626F031FD0028F2D1504627F046F820
:10C0700007F10C000BF1010B20F0C7FFC5E72846C4
:10C0800026F022FD00283FF45AAFB5F80B3003F537
:10C090000073A5F80B30236823F07F7323F400337B
:10C0A000BEE705464CE700BFBCB500208C8D0500FF
:10C0B0002C2D0020958D0500A18D05007C95050097
:10C0C00072930500482E0020AB8D0500B58D05004C
:10C0D000F78B050072DF7047F0B5284B284983B015
:10C0E000044600AF0246586823F020FC204626F0A4
:10C0F00008FD48B10023391D20467B6022F0CFFCAB
:10C1000005466CB970BB1BE0204626F0DDFC00281C
:10C11000F0D1CCB122461B49032023F0FBFF13E0F2
:10C1200000BB204624F09AFB0646786020F050FCC5
:10C1300006F5807383420AD91349012023F0EAFFF0
:10C140001249032023F0E6FF0C37BD46F0BDF31D76
:10C1500023F00703ADEB030D6D463246294620461A
:10C1600024F0A0FC00213B792A460846FFF7B2FFE5
:10C1700040F225410DF0C6FCE6E700BF482E002046
:10C180004A8E05007F8E050072930500538E0500D0
:10C1900070B5294C29492068002224F030FA054660
:10C1A00018B1002101200DF079FB284626F0A6FFEA
:10C1B00000222349206824F022FA054610B101200C
:10C1C0000EF0B6F8284626F099FF00221D49606857
:10C1D00024F015FA002205461B49606824F00FFA86
:10C1E000014606462846FFF72FFE2846314627F02F
:10C1F00060F800221549606824F001FA054611F044
:10C2000013F8284626F07AFF60681149002224F0CE
:10C21000F6F9044608B1FFF75FFF204626F06EFFEF
:10C220000DF0EEFE0B4B1B689B0503D5BDE870407F
:10C23000FCF742BA70BD00BF482E00203F8E0500BB
:10C240002B8A0500AB8D0500B58D0500428F0500DA
:10C250004A8E0500BCB500202DE9F043B0F80B3044
:10C2600091B003F500730446A0F80B3003A888468C
:10C27000174614F0B1FD90B30121294814F002FDD6
:10C28000054648B31FFA88F026F064F925490246AE
:10C29000204622F042FF00222349204624F0AFF935
:10C2A000DDF82690009006461FFA88F300223946F2
:10C2B00003A8C847002816DA1C49042023F02AFFE7
:10C2C000012026F03FF91A490246204622F025FFB8
:10C2D0002946304626F0EDFF03A814F019FD20464C
:10C2E00011B0BDE8F083013026F034F9114902465F
:10C2F000204622F012FF022F0DD101210E4814F02A
:10C30000C1FC07460028E3D0214622F02BFE384628
:10C3100026F0F4FEDCE72146284622F023FED7E78C
:10C32000B69405005C96050023900500CE940500A8
:10C33000E7940500EE940500F394050037B50190ED
:10C34000B0F80B300C4C03F50073A0F80B300D4621
:10C35000214622F0C9FE294602220198FFF77CFF00
:10C3600026F0CCFE0198012301AA214618F02CF9F1
:10C37000019803B030BD00BF1B9005002DE9F047C8
:10C380008EB005468846164626F0F1FC814620B15F
:10C3900028460021FCF73EFE0546284626F0BAFB5B
:10C3A000044638B94648294623F00AFE20460EB016
:10C3B000BDE8F087B8F1000F07D0404626F0ECFB4F
:10C3C000044610B941463F48EEE7022E16D101A8B7
:10C3D00014F0A8FC90B100223B49284624F00FF944
:10C3E00023F0C4F9DDF80D30834204DACDF80D00F6
:10C3F00001A814F090FC01A814F08AFC0121334834
:10C4000014F040FC0746002858D0012E4BD130498B
:10C41000002020F033F9044648B9384626F06EFE75
:10C42000B9F1000FC2D0284626F068FE2CE0294959
:10C43000002020F023F9A2460446F4B131462046FC
:10C4400014F012FCB8F1000F06D0234A41462046F2
:10C4500022F077FE26F052FE2146384622F082FD79
:10C46000BAF1000F04D052461C49204622F03CFE8F
:10C470002A461B49204622F037FE3946504626F010
:10C4800018FFB9F1000FCED1002E8FD101A814F002
:10C49000A3FC00288AD001A8214614F0CBF901A8FA
:10C4A00014F036FC82E7022E0CBF0E490E49002024
:10C4B00020F0E4F84FF0000A0446BEE70446E0E747
:10C4C00022940500849405005294050061940500AF
:10C4D0006894050070940500AB940500F69F050074
:10C4E00023900500789405007D940500F0B58FB089
:10C4F000054601A80F4614F06FFCA0B3284626F0AD
:10C5000009FB58B1194826F060FE194A0146044655
:10C51000284622F009FE214626F0CBFE384623F0BD
:10C5200041FF064668B126F037FB044648B911487A
:10C53000314623F045FD304626F0E0FD20460FB0A1
:10C54000F0BD304626F0DAFD012239462846FFF7D5
:10C5500015FF044618B1014601A814F0FFFA01A81E
:10C5600014F0D6FBEAE70446E8E700BF3C96050076
:10C57000409605008494050070B592B004460D46BF
:10C58000014601A8164614F00BFF60B33EB141F618
:10C59000FF739D42A8BF1D46012DB8BF0125BDF9FF
:10C5A0001830002B11DA2B040FD41049204623F049
:10C5B000ACF90F49204623F0A8F90E49204623F094
:10C5C000A4F90D49204623F0A0F901A8ADF81850B0
:10C5D00014F0C2FEB4F80B3003F50073A4F80B306E
:10C5E000204612B070BD0446FAE700BFA8920500CD
:10C5F000AD920500D0910500B29205002DE9F047FB
:10C60000074608460D46144626F0B1FB002800F008
:10C61000A88001225449284622F0CEF90646002877
:10C6200057D0284622F0F0F9062894BF4FF0FF3982
:10C630004FF006093A21284621F045FA00284BDB45
:10C6400000F101096FF000424946284621F0A3FAA3
:10C650007821824621F037FA041E47DB224600216A
:10C66000504621F098FA23F081F8611C80466FF063
:10C670000042504621F08FFA23F078F888F306083C
:10C6800080F3060048EA801848F48054504626F0AB
:10C6900035FDB9F1010FB8BF4FF00109284609F186
:10C6A000FF32002121F077FA054641F6FF708442FF
:10C6B000A8BF0446012CB8BF0124E6B1A4B22846A5
:10C6C00026F01CFD324621463846BDE8F047FFF70C
:10C6D00053BF4FF0FF39ADE7B9F1FF3FB2D1B5F825
:10C6E0000B3003F50073A5F80B30DEE7504622F05F
:10C6F000B9FA0446CAE715B904F50054DEE728463E
:10C7000022F082F90028F7D01849284622F05CF977
:10C710000028F1D12946164823F084FC3246014610
:10C72000804638461AF060FC8146B8B1334632463E
:10C7300039461FF055FA26F0E1FCA4F50044A4B2F6
:10C740004146484626F0B5FD4FF6FF739C42B6D1F0
:10C750002A460849012023F0DDFCB0E74FF6FF74BC
:10C76000EEE7BDE8F08700BFB6910500BD9105007A
:10C770000C9205001692050070B592B00546014670
:10C7800001A814F00DFE68B39DF80830012B83BF9B
:10C79000154B1A6804924FF0FF338EBF5B68049309
:10C7A00000230593BDF80B30013BADF82330BDF8F5
:10C7B0000D30013BADF82530079B03F44003002406
:10C7C00042F2010643F4702301A806960793ADF8E0
:10C7D00020408DF8224014F0BFFD22463146284605
:10C7E000FFF7CAFE12B070BDC8B5002010B50446F0
:10C7F00094B019B1FFF7C0FF26F080FC214603A8D2
:10C8000014F0CEFDC8B1079A0192BDF81520BDF80D
:10C810001330013A00920022013B114603A814F0A4
:10C820000FFB03A814F098FDB4F80B3003F5007368
:10C83000A4F80B30204614B010BD0446FAE710B53A
:10C8400092B00C46014601A814F0AAFD60B1BDF8F3
:10C85000093003F010031CB123B1BDF80B0003E055
:10C86000002BFAD0BDF80D0012B010BD2DE9F04F2D
:10C8700099B006460D46014607A814F091FD0446FE
:10C8800020B90024204619B0BDE8F08F8DB15C4975
:10C89000284622F099F8804658B95A49284622F08D
:10C8A00093F8044630B92A465749012023F032FC58
:10C8B000E8E7A04600213046FFF7C1FF012183468B
:10C8C0003046FFF7BCFF9DF8277000FB0BF47C435C
:10C8D00007340646E410B8F1000F35D025F0C0FE4D
:10C8E00005460028CDD0584625F034FE474902467B
:10C8F000284622F012FC304625F02CFE4449024620
:10C90000284622F00AFC012F07D0384625F022FEE7
:10C9100040490246284622F000FC9DF82030ABB981
:10C92000082F05D0BDF8213003F00F03042B0DD1E3
:10C9300000223949079823F062FE0246364928460C
:10C9400022F0EBFB2C469DE70334454620460021B0
:10C9500026F0E3FB044618B9284626F0CFFB91E702
:10C960000146002202A820F0A9FFB8F1000F0CD167
:10C970005FFA8BF102A820F0D8FCF1B202A820F0F7
:10C98000D4FC394602A820F0D0FC0026B14633463C
:10C99000B24627E01A46514607A8009314F0B1FCAE
:10C9A0000AF1010A09FA07F9D34549EA000907EB38
:10C9B0000602009B02DC01334FF0000A16460AE033
:10C9C000083E29FA06F1C9B202A8CDE9003220F0EA
:10C9D000ACFCDDE90032072EF2D8D6086FF0070173
:10C9E00001FB0626DDE902129142D3D3059826F019
:10C9F00085FBB8F1000F3FF445AF22469EE700BF2C
:10CA000042EF05004A9C050042900500B5900500E4
:10CA1000BB900500C29005001EA8050001381F2824
:10CA20009DBF034B23FA00F000F001000020704787
:10CA30008B80808030B551EC100B85B053EC112BFE
:10CA40008DED000B55EC124B8DED021B2AF0F0FD25
:10CA50009DED000B28B19DED021BB0EE410AF0EEFA
:10CA6000610A53EC102B204629468DED000B2AF06D
:10CA7000DFFD9DED000B08B145EC104B05B030BD5E
:10CA800038B555EC104B0022002310EE100A294651
:10CA90002AF0CEFD10B105F100431D4645EC104BC8
:10CAA00038BD10B413460A4653F8044B0021A4467F
:10CAB0005DF8044B60472DE9F843884691460546EA
:10CAC00018B1077A0024A74201D8BDE8F8832B6883
:10CAD000686833F83430184426F077FB0146064680
:10CAE0004846C047304626F009FB0134EBE722F008
:10CAF0003CBF0000002201491AF0FCBAD99B050096
:10CB000010B5044630B902460649032023F002FB63
:10CB1000204610BDB0F80B3003F50073A0F80B30C1
:10CB2000F6E700BF649D0500024B034958680022E8
:10CB300023F065BD482E002071C0050070B5044685
:10CB400025F0E8FF30B900242546204626F0D6FA25
:10CB5000284670BD00221449204623F050FD0546AA
:10CB600025F0D8FF044618B9284626F0C7FAEBE7A7
:10CB7000002DE8D000220D49284623F040FD044650
:10CB800026F00AF850B1284626F0B8FA002CDBD07F
:10CB9000074D2368EB1A5D425D41D6E729462046E2
:10CBA00026F087FBCFE700BFD99B0500E6AA05006A
:10CBB000C11F0300014900201FF060BD89990500D5
:10CBC000014900201FF05ABD39A10500014900208C
:10CBD0001FF054BD50A005002DE9F04390461D46BE
:10CBE000421E47F6FE739A4293B006460F4602D89D
:10CBF0004A1E9A4208D93249012023F08BFA0024B8
:10CC0000204613B0BDE8F0834046FFF707FF044617
:10CC100020B92C49012023F07DFAF1E7284625F0C0
:10CC200079FFD8B100222849284623F0E8FC0022E9
:10CC300004462649284623F0E2FC2546814628463C
:10CC400025F0AAFF044688B92A462149012023F08D
:10CC500061FA4946284626F02CFBD1E7B5F80B309F
:10CC600003F50073A5F80B308146E8E7B9F1000F32
:10CC700006D0484625F090FF044608B94A46E4E746
:10CC8000144900201FF0FAFC04460028B8D0012304
:10CC90008DF808303A464346314601A814F044FD69
:10CCA0002A460D490194204622F01EFA4A460B49B5
:10CCB000019822F019FA01A814F04EFBC9E700BF51
:10CCC000D4980500E1980500ED980500F698050058
:10CCD000FF980500AC900500339905003D990500CB
:10CCE00038B500220849054623F089FC044640B9BE
:10CCF00006491FF0C3FC044904460246284622F0B8
:10CD0000F3F9204638BD00BF11F60500FA9F050073
:10CD10002DE9F04391461D46421E47F6FE739A42A6
:10CD200093B00746884602D84A1E9A4205D95E4902
:10CD3000012023F0EFF9002408E04846FFF76EFEDB
:10CD4000044638B95949012023F0E4F9204613B0CC
:10CD5000BDE8F083564900201FF090FC04460028EF
:10CD6000F4D0002601A84B46424639468DF80860AB
:10CD700014F0DAFC28468DF809608DF80A600194F9
:10CD800025F0C8FE00285CD032464A49284623F0E8
:10CD900036FC22F039FE28B1BDF8093043F001031A
:10CDA000ADF8093000224449284623F028FC22F03F
:10CDB0002BFE28B1BDF8093043F00403ADF809306B
:10CDC00000223E49284623F01AFC22F01DFE28B11D
:10CDD000BDF8093043F00803ADF8093000223849A6
:10CDE000284623F00CFC22F00FFE88B19DF80F00BE
:10CDF00001280BD1BDF8093043F00203ADF809302A
:10CE0000BDF80D305B0703D02E4992E72E498FE71E
:10CE1000284600222D4923F0F2FB054688B12C4913
:10CE200021F0D2FD50B92B49284621F0CDFD78B92B
:10CE3000BDF8093043F08003ADF80930284626F0EC
:10CE40005DF901A813F0E2FF01A814F085FA7DE76F
:10CE50002149284621F0B8FD20B9BDF8093043F436
:10CE60008073E9E71D49284621F0AEFD20B9BDF8E1
:10CE7000093043F4C073DFE71949284621F0A4FDC7
:10CE800020B9BDF8093043F40073D5E715492846A9
:10CE900021F09AFD20B9BDF8093043F42073CBE7A7
:10CEA000114823F06DF8C9E7D4980500E198050012
:10CEB000AC90050001980500089805000C98050045
:10CEC0001898050056980500269805008F980500CB
:10CED0009B9805009F980500A3980500A79805005A
:10CEE000AB980500AF980500B3980500000000005E
:10CEF00008B500222DED028BB0EE408AF0EE608A7C
:10CF0000002351EC100B2AF0A7FB98B1B0EE480AB1
:10CF1000F0EE680A28F068F90B4B51EC100B002278
:10CF20002AF014F9BDEC028B41EC100BBDE808406F
:10CF300028F0D6B8BDEC028B9FED010B08BD00BFF9
:10CF4000000000000000F87F0000E03F000000004B
:10CF5000F8B555EC104B25F000474FF0FF32284B49
:10CF6000204639462AF08CFB60B94FF0FF32244B43
:10CF7000204639462AF07AFB20B9B5F1004F08BFA8
:10CF8000002C05D145EC104BBDE8F84025F0D0BA97
:10CF900000220023204629462AF04AFBC8B912A1E4
:10CFA000D1E900012B46224629F01AFF06460F461A
:10CFB0002AF02CFC04460D4654EA05030DD100224C
:10CFC0000023304639462AF033FB30B19FED080B81
:10CFD000DAE709A1D1E90001E4E720462946BDE8E6
:10CFE000F84025F04DBB00BF2083E4FFFFFFDF3F8B
:10CFF00000000000000000802083E4FFFFFFDFBF8F
:10D00000FFFFEF7F28F068B827F0EABC38B555EC91
:10D01000104B10EE102A2B4610EE100A29462AF06B
:10D0200095F802460B460020094929F0D7FE41EC4D
:10D03000100BFFF75DFF204653EC102B29462AF01A
:10D04000AFF9BDE8384041EC100B27F0C9BC00BF78
:10D050000000F03F27F0E0BF30B591B0054625F065
:10D06000A5FE044638B92A461F49032023F052F88A
:10D07000204611B030BD0122294605A821F055F8FF
:10D0800000231A4605A9194814F01EFC044605A8F9
:10D090001FF06DFF2046002126F03FF8044618B926
:10D0A000134822F08DFFE3E72946012205A821F06D
:10D0B0003CF821460022684620F000FC6B460D4AF1
:10D0C0000A4805A914F000FC039826F017F805A8F3
:10D0D0001FF04DFF0021204621F020FD054620468F
:10D0E00026F00CF82C46C3E7479905000FFB030018
:10D0F0006C99050031FB030030B591B0054625F071
:10D1000055FE044638B92A461F49032023F002F889
:10D11000204611B030BD0122294605A821F005F8AE
:10D1200000231A4605A9194814F0C2FC044605A8B4
:10D130001FF01DFF2046002125F0EFFF044618B91F
:10D14000134822F03DFFE3E72946012205A820F01D
:10D15000ECFF21460022684620F0B0FB6B460D4AEA
:10D160000A4805A914F0A4FC039825F0C7FF05A8F8
:10D170001FF0FDFE0021204621F0D0FC0546204690
:10D1800025F0BCFF2C46C3E7479905000FFB0300C1
:10D190006C99050031FB0300F8B5051E0C4606DC52
:10D1A0002949012022F0B6FF00242046F8BD084698
:10D1B00025F0B0FC0646A8B100222449204623F001
:10D1C0001EFA22F021FC002221490646204623F0C7
:10D1D00016FA22F0CBFA30F0080309D0102809D053
:10D1E0001C49DEE724B122461B49012022F092FFB0
:10D1F000012400E002242946204620F0A7F9074632
:10D200009EB12946204620F0A1F905461349002089
:10D210001FF034FA044610B10FB146B13DB92A46A9
:10D220003946204626F038F8BEE73546EEE73A465E
:10D230000B49204621F071FF002DB6D02A4609493E
:10D24000204621F06AFFB0E774A2050093A2050012
:10D25000B2A20500A0A20500B7A20500EEA205003B
:10D260001EA80500F7A2050038B5044625F052FCBB
:10D2700088B100220949204623F0C1F9054625F06E
:10D2800076FD10B1284621F0BFFB0446284625F064
:10D2900035FF204638BD0446FBE700BF27A2050046
:10D2A00070B506460D4625F062FD044630B932469B
:10D2B0001349032022F02EFF204670BD11490020A3
:10D2C0001FF0DCF932461049044621F00DFF45B14C
:10D2D000284625F04CFD68B932460949032022F062
:10D2E00019FF002025F036F908490246204621F0B2
:10D2F00014FFE1E72A460649204621F0F5FEF0E753
:10D3000007A0050032A0050039A0050046A00500D1
:10D3100040A00500F8B506460D460AB3104621F0B8
:10D32000A1FC002D044603DA304621F06DFB0544D4
:10D33000002C03DA304621F067FB04441B2025F063
:10D3400093F825EAE57524EAE474074630B1A5426E
:10D3500004DA631B2A46314620F0F0FB3846F8BD5C
:10D3600000296FF00044E9DADEE7F8B505460C461F
:10D37000C2B1104621F076FC20EAE076002C05DAF6
:10D38000284621F041FB044424EAE4741B2025F0E4
:10D390006BF8074620B133462246294620F0CEFBE3
:10D3A0003846F8BD6FF00046E8E7F8B507460C468A
:10D3B000CAB1104621F056FC20EAE07524EAE47474
:10D3C000A542B8BF23464FF01B00BCBF2C461D46EC
:10D3D00025F04AF8064620B12B1B2246394620F09C
:10D3E000ADFB3046F8BD6FF00040E5E770B50D1EAF
:10D3F000064606DA0B49012022F08CFE0024204666
:10D4000070BD1B2025F030F8044615F1FF35F6D32A
:10D410001FF0D6FA0028F2D13146204620F0B6FBA4
:10D42000F3E700BF60A20500F8B506460F461546B3
:10D4300025F09DFC044698B1284625F0BFFB88B135
:10D44000284621F00FFC0446384622F00FFB054623
:10D4500021F0DAFA241A09D50024284625F04EFED8
:10D460002046F8BD304621F0CFFAECE7284621F0FF
:10D47000CBFA0719304621F0C7FA8742ECDC224686
:10D48000012329463046F3F73FF9B0FA80F46409E6
:10D49000E3E7F8B507460E46154625F068FC044656
:10D4A00048B1304622F0E2FA002D064605DA0024A3
:10D4B000304625F023FE2046F8BD21F0A5FA441998
:10D4C000384621F0A1FA8442F1DC01232A46314694
:10D4D0003846F3F719F9B0FA80F46409E8E72DE962
:10D4E000F04186B022F0C2FA0546E0B101460022C2
:10D4F00001A820F0E3F94FF0FF340026DDE90183B5
:10D50000984514D3049825F0F9FDA642DABFA21B72
:10D51000013200223146284620F03DFB04462846D1
:10D5200025F0ECFD2546284606B0BDE8F08101A8AF
:10D53000039F1FF080FF1FF09DFC0028DED107EB4A
:10D54000080336EA240628BF1E461C46D6E700001C
:10D5500070B5002286B00E46114923F050F80546FA
:10D5600025F005FC044660B10022294601A820F000
:10D57000A5F90024DDE901239A4208D3049825F097
:10D58000BDFD284625F0BAFD204606B070BD01A8B5
:10D590001FF051FFB04208BF44F00104E4B2E9E7D4
:10D5A00040A0050008B508B1036823B91B20BDE8F9
:10D5B000084024F059BF002123F094FBBDE8084047
:10D5C00024F0ECBD08B520F0A1FA08BD70B5054601
:10D5D00086B01B200E4624F047FF0446E0B12846E3
:10D5E00025F0C5FBC0B1002E16DB3246294601A846
:10D5F00020F064F9DDE901239A420AD2059B03B1C8
:10D600009B5C8DF8033001220DF10301204620F0D0
:10D61000D2FA049825F072FD204606B070BD37B5E9
:10D6200005461B2024F020FF044628B1294601A806
:10D630001FF0FCFC019810B9204603B030BD22F069
:10D64000B1FE22F093F801228DF803000DF10301E1
:10D65000204620F0B0FA01A81FF0D7FCEAE700004E
:10D66000F8B507460E4625F055FA88B30022194949
:10D67000384622F0C4FF054625F079FB18B328464A
:10D6800021F0C2F9002E01DD86420AD31149384645
:10D6900022F03BF92C460025284625F02FFD204698
:10D6A000F8BD32460021284620F075FA314604467E
:10D6B0006FF00042284620F06EFA064902463846CE
:10D6C00021F02BFDE8E71B2024F0CEFE0446E3E723
:10D6D0000446E4E727A205002DE9F041CB1D23F025
:10D6E000070300AFADEB030D134614466E460D461F
:10D6F00053F8048B0A463146C047A3692B44A36103
:10D7000063692B44636135441C34AE4202D1BD468B
:10D71000BDE8F081204616F8011B1FF042FE2046AE
:10D720001FF048FDF1E700002DE9F04F93B000AF86
:10D730000E46154681461AF075FC4FF0010A044664
:10D7400007F11701304687F817A0F3F797FF002D70
:10D75000804606DC4FF0000840464C37BD46BDE829
:10D76000F08F1FF035F905F58073834204D96049C5
:10D77000504622F0CFFCEDE7EB1D23F00703ADEBA5
:10D78000030D122C6E463BD15A4B1B78CBB10023B4
:10D7900007F120024FF040215748C7F82230C7F860
:10D7A00026307B8587F820A087F8218087F82250D3
:10D7B0007E62F7F7DBFD024618B15049042022F0E3
:10D7C000A9FC294601201FF0C1FE80460028C1D0D7
:10D7D0000146002207F1200020F097F8354416F8A2
:10D7E000011B07F120001FF0DCFD07F120001FF0F6
:10D7F000E1FCB542F3D107F120001FF0B2FBABE72B
:10D80000002CA7D13E492246484622F0F8FE824627
:10D81000014607F1180015F05FFC00285CD0224695
:10D820003849484622F0EBFE22F0EEF83B7FB8770D
:10D83000FF2B51D07A7FFF2A4ED087F8212087F81E
:10D840002030BA69304B93FBF2F37B62FB7FF97DAA
:10D8500087F82200002B07F120002C4BF96008BF4D
:10D860000023BB6215F0FEFB4FEA480101F4FF7193
:10D8700041F0010107F1200015F0ACFB60B305F1A8
:10D88000FF38A8EB04035942594108224FF0000B1E
:10D8900007F12000C7E9011215F03CFBBA6879686E
:10D8A0004FEA4B0B013A40EA0B0BF1D107F1200094
:10D8B00015F060FB97F8210015F01CFB06F804B08A
:10D8C0000134A542DDD1FB681BB107F1200015F042
:10D8D00093FB97F82230BB77B87F24F033FE0949D9
:10D8E0000246484621F000FC514625F0E2FC68E77C
:10D8F0008D99050098B500203CAE0020C299050026
:10D90000D5990500DE99050090D00300A08601009E
:10D910002DE9F04F89B000AF0D46904606461AF04B
:10D9200081FB4FF0010AF91D0446284687F807A03D
:10D93000F3F7A4FE0023834607F108014046BB60CD
:10D9400021F0ADF80546B8F1000F43D0F0B94046DC
:10D9500022F084FF8146B8601FF03AF809F5807321
:10D96000834207D94949504622F0D4FB2437BD46AB
:10D97000BDE8F08F09F1070323F00703ADEB030DBA
:10D980006D464A462946404623F08CF8BB68002B7A
:10D99000ECD0122C21D13E4A1278002AE6D0F97937
:10D9A0003C48BD61002291427A61FA61BB754FF03B
:10D9B000402114BF1346202307F1140287F815B045
:10D9C000F7F7D4FC02460028D0D03349042022F0D7
:10D9D000A1FBCBE70028C9D0D8E7002CC6D12F493E
:10D9E0002246304622F00BFE8046014607F10C002D
:10D9F00015F072FB60B322462949304622F0FFFD44
:10DA000022F002F83B7CB874FF2B21D07A7CFF2AED
:10DA10001ED07A753B75FA68224B93FBF2F3BB611B
:10DA2000FB7CB875002B07F114001F4BD7F808A03A
:10DA300097F8079008BF0023FB6115F013FB4FEA2E
:10DA40004B0101F4FF7107F1140015F0C3FA88B916
:10DA5000B87C24F077FD12490246304621F044FBA1
:10DA6000414625F026FC81E7295D07F1140015F0F9
:10DA7000B1FA0134A245F7DCB9F1000F03D007F188
:10DA8000140015F0B9FABB7DBB74E1E77293050091
:10DA900098B500203CAE0020329A0500D5990500CB
:10DAA000DE99050090D00300A08601002DE9F74F14
:10DAB0000D4603210446CDE900230DF0E1FF4FF0B0
:10DAC000000B4FF0010A4FF08008D94615F1FF35E1
:10DAD00002D203B0BDE8F08F009B0AEA0306019B67
:10DAE0000BEA030756EA070316D088F311880021D2
:10DAF00020460DF0D5FC0A20F3F71AFF012120463D
:10DB00000DF0CEFC89F311883720F3F711FF1AEBE3
:10DB10000A0A4BEB0B0BD9E788F31188002120464A
:10DB20000DF0BEFC4120F3F703FF012120460DF06C
:10DB3000B7FC89F311880520E7E710B40C7802469A
:10DB40000023204608215DF8044BFFF7AFBF00001B
:10DB50002DE9F04F89B0894600901AF063FA4946E2
:10DB6000044602A815F0B8FAF0B1122C40F0F88083
:10DB70009DF80C4020461AF0E5FA9DF80D5018B1BA
:10DB800028461AF0DFFA90B922462946854822F045
:10DB900017FAB9F1000F00F00081834A0098494656
:10DBA00021F0C2FA25F0AAFA09B0BDE8F08F7F494A
:10DBB000029E7F4B04EB440405EB45050C440D44E9
:10DBC0009E4294F801806F7858DD7A4B9E42D4BF14
:10DBD0004FF080664FF0CD66774A784C13785BB390
:10DBE00023681BB1764B1021C3F880104FF04023FF
:10DBF0004FF0FF31C3F80813D3F800120021C3F827
:10DC00000012C3F80015012184F8221094F827109F
:10DC100079B9D3F808154FF0A04001F5E07140F252
:10DC2000023540F82150D3F80C3503F5E07340F885
:10DC30002350002384F8223094F8223001251570F7
:10DC4000FBB108225F49042022F064FA9DF80C40E1
:10DC500020461AF077FA20B14FF4207120460DF0DB
:10DC60008FFD9DF80D4020461AF06CFA002890D0E8
:10DC70004FF4945120460DF083FD8AE74FF0CC76A7
:10DC8000AAE79DF81E2084F827209DF81D20A36098
:10DC9000C4E9003384F8253084F8243072B34FEAA5
:10DCA0008800B90000F1A04001F1A04140F20C62EF
:10DCB0004FF0A04BC0F8002705FA08FAC1F800277A
:10DCC000BD4040F20D620193CBF808A5CBF8085592
:10DCD000C0F80027C1F800270420F3F7E5FD019BF9
:10DCE000DBF810150D422BD043B14FF0A04A0420B1
:10DCF000CAF80C55F3F7D8FDCAF808554FF0A04301
:10DD000008F5E07140F20C6243F8212007F5E0715C
:10DD100043F821204FF040231D46C3F80885C3F87F
:10DD20000C75C3F8246522681AB106210420F7F7A0
:10DD3000F9FC0523C5F80035022384F8223085E775
:10DD400001930420CBF80CA5F3F7AEFDCBF808A5A2
:10DD50000420F3F7A9FD019B0133092BC0D1C4E7CF
:10DD6000002C7FF416AF9DF80C00FF2807D001218E
:10DD70000DF096FB03219DF80C000DF081FE9DF83F
:10DD80000D00FF283FF405AF01210DF089FB0321B1
:10DD90009DF80D000DF074FEFBE60349009821F09C
:10DDA000B4FD01E7E6990500D5990500BC7D0500A5
:10DDB00097AB020087F5040098B500203CAE002028
:10DDC00000E100E0159A0500F0B58DB00D4616464D
:10DDD0001C461AF027F911289DF8487005D02F49E4
:10DDE000012022F097F90DB0F0BD16B90CB90F243F
:10DDF00003262B4B1B78F6B2E4B25BB92949ADF888
:10DE000010306FF0FF02CDE9011201A8264A0392FB
:10DE10000DF0D4FCFF2F03D0002138461AF09EFCF1
:10DE2000284624F0CBFE80B1284620F01BFF224676
:10DE30003146C0B2F3F7C4FAF3F772F9FF2FD2D02C
:10DE4000012138461AF08AFCCDE7284624F0AEFFBF
:10DE5000E8B1802383F311880122294601A820F02C
:10DE600064F901A81FF0AFF8054601A825B91FF015
:10DE70007EF885F31188DFE722F012FB2246314657
:10DE8000C0B2F3F79DFA01A820F062FFE9E72A4645
:10DE90000649012022F03EF9CEE700BF3DA1050072
:10DEA0007CB50020A08601000001080065A10500E6
:10DEB000F0B58DB00D4616461C461AF0B3F8112881
:10DEC0009DF8487005D03049012022F023F90DB0AB
:10DED000F0BD16B90CB9032401262C4B1B7806F0B3
:10DEE0000F0604F00F045BB92949ADF810306FF04C
:10DEF000FF02CDE9011201A8264A03920DF05EFC53
:10DF0000FF2F03D0002138461AF028FC284624F0C1
:10DF100055FE80B1284620F0A5FE22463146C0B20B
:10DF2000F3F70EFAF3F7FCF8FF2FD0D001213846B3
:10DF30001AF014FCCBE7284624F038FFE8B1802320
:10DF400083F311880122294601A820F0EEF801A8E8
:10DF50001FF039F8054601A825B91FF008F885F328
:10DF60001188DFE722F09CFA22463146C0B2F3F76F
:10DF7000E7F901A820F0ECFEE9E72A46064901206E
:10DF800022F0C8F8CEE700BF15A105007CB500203F
:10DF9000A08601000001080065A10500F0B58BB066
:10DFA00004460D461AF03EF801AE07463246694671
:10DFB000204614F0D9FD98B3009B059396E80F0016
:10DFC00006AC07C423807DB3296800292CDD013904
:10DFD000284622F087FE064624F060FF10B3304644
:10DFE0001AF08FF80446284621F059FC25F086F8EF
:10DFF000304625F083F8FF2C03D0002120461AF08C
:10E00000ADFB05AA0949284622F02EFB112F01D1AC
:10E01000F3F786F8FF2C03D0012120461AF09EFB6F
:10E020000BB0F0BDFF24E3E7FF24EAE7A3CA020038
:10E030002DE9F041B8B00D46164607A908AA14F01C
:10E0400093FD002877D0FF2E03D0002130461AF030
:10E0500085FB284624F0B2FD80462846B8F1000F23
:10E0600018D020F0FFFD18A98DF8600008AB084615
:10E070000122079CA0479DF8600024F06BFA04463B
:10E08000FF2E03D0012130461AF068FB204638B03D
:10E09000BDE8F08124F06BFE0746002831D01B203C
:10E0A00024F0E2F942460446294602A81FF006FC85
:10E0B000DDE902239A4203D3059825F01FF8DFE734
:10E0C0001EF07EFC0028F7D101AA694602A81FF0C5
:10E0D00022F8019D002DEBD0802D28BF802508ABB4
:10E0E0002A4618A90098079FB8472A4618A920462B
:10E0F0001FF061FD019B5B1B0193009B1D4400957C
:10E10000E7E7284622F0AAFB014601201FF01EFA8D
:10E1100004460028B4D03A4601460EA8CDE90C7753
:10E120001FF0F3FB07AA0549284622F09DFA0EA826
:10E130001EF017FFA4E70446A8E700BFD9D60200E7
:10E140007FB50C46054619F06DFF21460646684628
:10E1500014F070FC60B1112E0CD168460DF02EFB4E
:10E1600004B3134A2146284620F0DEFF24F0C6FF00
:10E1700004B070BD002EFBD19DF80500FF2802D031
:10E1800001210DF07DFC9DF80600FF2802D004213E
:10E190000DF076FC9DF80700FF28E1D001210DF07D
:10E1A0006FFCDDE70249284621F0AFFBE0E700BF46
:10E1B000D59905002DE9F04300228DB0244906468B
:10E1C00022F01DFA05AD0146284625F0F5FB1B227D
:10E1D000541E295D09B1144602E02246002CF7D1F5
:10E1E0000CAB4FF001081C440DF1240904F81C8C01
:10E1F00099E807008DE8070095E80F0025F02DFA53
:10E2000008F1010807460028F0D1012024F0A2F906
:10E2100010490246304620F080FF384624F09AF933
:10E220000D490246304620F078FF384624F092F936
:10E230000A490246304620F070FF384624F08AF939
:10E240000749024630460DB0BDE8F04320F065BFF7
:10E250007C950500B6A10500BCA10500C3A1050081
:10E260005CB305002DE9F04F00229BB00C469B49A2
:10E27000054622F0C4F921F079FAC0B2772808D017
:10E28000612806D09649012021F044FF1BB0BDE86B
:10E29000F08F204621F0EAFB07460028F6D020F058
:10E2A000B3FB81460028F1D000228E49284622F097
:10E2B000A6F921F05BFA00228B498246284622F01B
:10E2C0009EF921F053FA002288498346284622F01D
:10E2D00096F921F04BFA002285498046284622F023
:10E2E0008EF90BAC0146204625F066FB1B22531E1F
:10E2F000E15C09B1134602E01A46002BF7D11AAAD5
:10E300001A44CDE9082302F83C8C7A4900222846B9
:10E3100022F075F921F02AFA0646002845D0099B1B
:10E32000A0F120020DF1480E10685168F446ACE8E7
:10E3300003000832B242E646F6D15A1C214613A821
:10E3400029F00AFCA8B112AB03930FAB93E80700C6
:10E350008DE8070094E80F0025F08DF8064608B90F
:10E36000654990E724F0F6F862490246284620F015
:10E37000D4FEABEB0A0BD94556444FDB5A4600217D
:10E3800038461FF008FC3146824606F021FF504611
:10E3900024F0B4FEB8F1FF0F4BD15849012021F011
:10E3A000B9FE384624F0AAFE70E74FF47E63CDE94B
:10E3B00005034023CDE903730FAE96E807008DE80F
:10E3C000070094E80F0025F089F90028E9D012AB86
:10E3D000039396E807008DE8070094E80F0025F006
:10E3E0004AF80646129820F07F44484624F0B2F8D6
:10E3F0003C490246284620F090FE204624F0AAF828
:10E4000039490246284620F088FE304624F0A2F81A
:10E4100038490246284620F080FEC2E73846314699
:10E4200006F0D6FE09EB0A0024F094F82D490246C6
:10E43000F0E7089B08F1010003F83C0C24F08AF88F
:10E440002A490246284620F068FE6FF000425946ED
:10E4500038461FF0A0FB00234FF47E62CDE9053261
:10E460004023CDE903030FAE804696E807008DE810
:10E47000070094E80F0025F031F9002891D012AB85
:10E48000039396E807008DE8070094E80F0024F056
:10E49000F2FF0646129820F07F44484624F05AF8CE
:10E4A00010490246284620F038FE204624F052F853
:10E4B0000D490246284620F030FE304624F04AF846
:10E4C0000C490246284620F028FE404620F09CFADF
:10E4D0000446404624F012FE2046A5E75CB3050042
:10E4E000E0A10500BCA10500F9A10500B6A1050049
:10E4F0007C950500C3A10500FDA1050019A205003A
:10E500002DE9F04F0022A1B00E466E49054622F0DB
:10E5100076F821F02BF9C0B2722808D06A490120A0
:10E5200021F0F8FD0027384621B0BDE8F08F002229
:10E530006649284622F063F821F018F98046002841
:10E5400000F0BD8000226249284622F058F821F0F0
:10E550000DF900225F498146284622F050F821F04B
:10E5600005F900225C498246284622F048F821F04D
:10E57000FDF8002259498346284622F040F801461A
:10E5800009A825F019FA1B22531E09A9C95C09B173
:10E59000134602E01A46002BF6D120AAD3180693A0
:10E5A00003F85CBCF30F059318BF202600273EBB81
:10E5B0007CE04FF0000846E012F8011BFF291CD058
:10E5C0000598013300286CD00A296AD100221C4624
:10E5D000059237B91B20079323F046FF079B074698
:10E5E00030B1224610A9384607931FF0E4FA079B82
:10E5F000059AA1441AB91E1BD9E71C4654E02026EF
:10E60000AAEB0904002C3DDCBBF1FF0FD1D0069B27
:10E610000BF1010B03F85CBC18AB03930DAB93E853
:10E6200007008DE8070009AB0FCB24F024FF189BEF
:10E6300023F07F4A8046504623F08CFF254902464E
:10E64000284620F06AFD404623F084FF1F49024619
:10E65000284620F062FD002023F07CFF1C49024682
:10E66000284620F05AFD584623F074FF1A49024606
:10E67000284620F052FDB8F1000F3FF454AF544645
:10E680004FF00009202E3346A8BF20239C42A8BF8C
:10E690001C46224609EB080110A829F06BFA10AAC3
:10E6A0000023A34288DB3346002C92D1484623F056
:10E6B00051FF07490246284620F02FFD33E7074661
:10E6C00031E700BF5CB30500C8A10500C3A1050088
:10E6D000BCA10500F9A10500B6A105007C950500C7
:10E6E0004FF0FF31FFF70CBF21EAE171FFF708BFE0
:10E6F0002DE9F04F0022A5B03B4921F080FF05AC89
:10E7000001460546204625F03DF9284624F0F6FC52
:10E710001B235E1EA25D0AB11E4602E03346002E98
:10E72000F7D124AB1E444FF001080CAF06F87C8CE7
:10E730000DF1240B03979BE807008DE8070094E890
:10E740000F0024F098FE0546002847D00C9B23F0CC
:10E750007F4303444FF0000913F8013C0C9AFF2B50
:10E7600022F07F4A02D0B8F1FF0F1ED10024AAEB9D
:10E770000406002E14DD412E28BF402632466119C2
:10E7800014A829F0F7F914AA002312F8011BFF2995
:10E7900022D001339E42F8D100221C44002AE6D048
:10E7A00004EB090025B0BDE8F08F08F1010806F878
:10E7B0007C8C03979BE807008DE8070094E80F0026
:10E7C00024F059FED144054658B10C9B23F07F43F9
:10E7D000034413F8013CC1E70122DEE78146044609
:10E7E000DEE70446DCE700BF7C9505002DE9F04F2D
:10E7F0000C46A7B006466749204620F0E5F898B9D0
:10E800006549204620F0E0F850BB6449204620F0DE
:10E81000DBF8054638BB22466149012021F07AFC2D
:10E82000284627B0BDE8F08F4FF0720A5D490020FE
:10E830001DF024FF05460028F2D01C22002130469E
:10E840001FF0A9F90DF11C0801460646404625F0C7
:10E8500099F81B214B1E18F803203AB10B4608E02B
:10E860004FF0770AE2E74FF0610ADFE71946002B25
:10E87000F0D126AAD3184C490593324628460124E4
:10E880000EAE03F87C4C0DF12C0920F046FC0396EB
:10E8900099E807008DE8070098E80F0024F0EBFDE9
:10E8A0000E9BBAF1770F074623F07F4B09D1002862
:10E8B0006ED02846FFF77EFC4FF0000B5F46002627
:10E8C00029E0BAF1610FFAD1002F61D007EB0B03F9
:10E8D00013F8013CFF2B01D0FF2C45D10026ABEBF8
:10E8E0000608B8F1000F16DDB8F1400FA8BF4FF0D1
:10E8F00040084246F11916A829F03CF916AA00234F
:10E9000012F8011BFF2941D001334345F8D1002201
:10E910001E44002AE3D0204623F01CFE2349024671
:10E92000284620F0FAFB304623F014FE2049024628
:10E93000284620F0F2FB384623F00CFE1D49024623
:10E94000284620F0EAFB584623F004FE1A49024606
:10E95000284620F0E2FB504623F0FCFD1749024612
:10E96000284620F0DAFB5BE7059B013403F87C4C7A
:10E97000039699E807008DE8070098E80F0024F057
:10E980007AFD0E9B074623F07F4B9DE70122BFE7F0
:10E990003E46C0E7830006009FAA0500DBC00500D5
:10E9A0009AA10500AAA105007C950500B6A1050065
:10E9B000BCA10500C3A10500F9A105005CB30500D9
:10E9C00010B58CB005AC0146204624F0DBFF0CAB43
:10E9D00013E907008DE8070094E80F0024F03DFEDE
:10E9E0000CB010BDF2F750B924F0C2BC70B50022D3
:10E9F00090B006460846114609F0E6F909AC05460E
:10EA00003146204624F0BEFF0023CDE90533CDE991
:10EA1000035310AB13E907008DE8070094E80F00DB
:10EA200024F05CFE0446284624F068FB204610B023
:10EA300070BD2DE9F041804690B008460C4617465F
:10EA40001E4624F067F810B300221146204609F054
:10EA5000BBF900260546374609AC4146204624F05E
:10EA600091FF0023CDE90353CDE9057610AB13E9FF
:10EA700007008DE8070094E80F0024F02FFE0446FD
:10EA8000284624F03BFB204610B0BDE8F08120462C
:10EA900023F0A2FC0546DFE730B58FB007AC014696
:10EAA0000025204624F06EFFCDE903550EAB13E997
:10EAB00007008DE8070094E80F0024F023FD0446CA
:10EAC00038B1294620F02AF80546204624F016FBE6
:10EAD0002C4620460FB030BD70B58EB007AC164640
:10EAE0000D460146204624F04DFFCDE903560EABFE
:10EAF00013E907008DE8070094E80F0024F002FDF9
:10EB00000EB070BD70B58EB007AC0E460146204603
:10EB100024F038FF0023CDE903330EAB13E90700DF
:10EB20008DE8070094E80F0024F0ECFC054668B17E
:10EB300004F06CFB0446284624F0E0FA1EB121F0F4
:10EB40004FFC24F0DBFA20460EB070BD0446FAE715
:10EB50004FF4D82024F0E2BE13B50C4619F062FA47
:10EB60008DF807000938042805D80DF1070203497C
:10EB7000204621F081FE02B010BD00BF81EB0200F3
:10EB80000B78C1B2184614F023BF00002DE9F04302
:10EB900089B0984605460E46174619F043FAA0F18B
:10EBA0000903DBB2042B04462ED80D280FD1274BC6
:10EBB000DB7863B94FF0FF324FF41651CDE9041200
:10EBC00004A8234A06928DF81C30F6F7D1FD8DF883
:10EBD0000040204C1FB1304620F048FF06466A46F0
:10EBE0002146304621F048FE17B1304624F086FA1F
:10EBF000B8F1000F05D069460D20A04769460A20EC
:10EC0000A04709B0BDE8F0830028FAD102461249B6
:10EC1000284621F0F4FC224681461049284621F07E
:10EC2000EEFC04AD024649460446284614F06EF850
:10EC3000204624F063FA484624F060FA95E80F0075
:10EC40006C4607C42370064CC4E700BF99B500208A
:10EC5000080001005D3C0400F2960500D59905000E
:10EC6000DD31040000231A46FFF790BF01231A4646
:10EC7000FFF78CBF00230122FFF788BF2DE9FF4774
:10EC8000044619F0CFF9002205464049204621F0FC
:10EC9000B6FC002207463E49204621F0B0FCA5F113
:10ECA00009068246002F4CD001463A46684614F0C9
:10ECB0002DF89DF80600FF2802D000210CF0E0FEA0
:10ECC0009DF80700FF2802D000210CF0D9FE9DF826
:10ECD0000400FF2802D000210CF0D2FE9DF80500B0
:10ECE000FF2802D000210CF0CBFEF3B2042B28D970
:10ECF00000222849204621F082FC10B320F036FD86
:10ED00005FFA80F8002140460CF0B8FA002013F0BA
:10ED100091FF8146A8B141461EF089FC804618B19A
:10ED20000146484620F02CFD48461EF0D7FC20B98D
:10ED3000194B1A49586820F0E8FD4946404624F02E
:10ED4000B8FA5146384624F0B4FA1149204620F06A
:10ED5000DCFDF6B20D49204620F0D7FD042E11D877
:10ED60000D2D0AD10E4BDB780BB10CF0BBF8FF2256
:10ED70000021284614F04AFD04E0A5F10C03DBB2A3
:10ED8000012BF4D904B0BDE8F08700BFD599050088
:10ED9000F296050007A10500482E00200CA10500F1
:10EDA00099B50020F0B585B005460F46144619F018
:10EDB00039F9064684B922465249284621F01FFCFB
:10EDC000044622463946684613F0A0FF58B920464B
:10EDD00024F094F905B0F0BDB4F80B3003F50073DE
:10EDE000A4F80B30EDE7009823F0B4FB4649024647
:10EDF000284620F092F97CB122464249284620F06C
:10EE00008CF9A6F10903DBB2042B0AD80D2EE1D14F
:10EE10006846F6F7ADFCDDE73A49284620F075FD77
:10EE2000EFE7002ED6D19DF80500FF2807D001217D
:10EE30000CF026FE01219DF8050019F08FFC9DF8CD
:10EE40000400FF280BD005210CF01AFE602023F0EF
:10EE50002DFC044660B92D49012021F05BF99DF895
:10EE60000630FF2BB6D02A49012021F053F9B1E733
:10EE700002462849284620F050F920461EF016FD8B
:10EE8000002680F8406004460CF024FB009B9DF8AF
:10EE90000A2084F85860C4E914369DF808301344F9
:10EEA0009DF80920B24218BF0133C4E9120184F869
:10EEB000593001219DF804000CF0E0F90446C8B176
:10EEC00023F048FB14490246284620F026F9012089
:10EED00013F0B0FE06460028C1D02A46214620F095
:10EEE0008AF8304624F00AF9013C0C4B0C4A43F8EE
:10EEF0002420B4E79DF804200A49012021F00AF9F2
:10EF0000ADE700BFD5990500F296050082A0050087
:10EF1000DFA00500A8A0050007A1050010B600208D
:10EF2000512C0400B0A0050010B50C4619F07AF879
:10EF3000A0F10903DBB2042B04D82146BDE8104040
:10EF400018F0E6BC02490120BDE8104021F0E2B80B
:10EF500057A005002DE9F74F9846012313600D696E
:10EF600007468A4616460DB10B68ED5C38782E28A8
:10EF700000F0FA805B2836D1012388F8093097F831
:10EF800001B0BBF15E0F02D13368013333604FF043
:10EF9000000907E02E2C19D12E2D08BF49F00109D8
:10EFA000013333603368FC5CF818002C00F0DE801D
:10EFB0005D2CEFD101333360002388F80930BBF1B9
:10EFC0005E0F14BF484689F0010019E0434601AACC
:10EFD0005146FFF7BFFF3368019A49EA00095FFA1B
:10EFE00089F91344DDE75C286CD10223336078781B
:10EFF000642808D1A5F1300009288CBF0020012029
:10F0000003B0BDE8F08F442806D1A5F130000928EF
:10F0100094BF00200120F3E766286ED062286ED0EE
:10F020006E286ED072286ED0732805D1284603B0A2
:10F03000BDE8F04F1DF01EBF532806D128461DF035
:10F0400019FF80F00100C0B2DAE774285DD076289D
:10F050005DD077280ED1A5F13003092B40F28480D2
:10F0600028461DF0FBFE00287ED15F2D14BF002036
:10F070000120C5E757280CD1A5F13003092B12D97F
:10F0800028461DF0EBFE70B9B5F15F0018BF0120F6
:10F09000B6E730283DD0A0F13103082B05D836491A
:10F0A000012021F037F80020AAE778280AD1BB78A0
:10F0B00043B1FB7833B104233360F978B8781DF09D
:10F0C000BCFEC0B298F809302BB33368FA5C2D2A25
:10F0D00021D13B445B785D2B1DD0A8F80A00306835
:10F0E00001303060434601AA51463844FFF732FFF1
:10F0F0003368019A1344336082E70C20E2E708206A
:10F10000E0E70A20DEE70D20DCE70920DAE70B2044
:10F11000D8E70020D6E798F8082062B1A5F14103AE
:10F12000192B98BF2035A0F1410398BFEDB2192BE0
:10F130009CBF2030C0B2B8F90A30B3F5807F11D03F
:10F14000DBB22AB1A3F14102192A9CBF2033DBB202
:10F150004FF480729D42A8F80A20A4D38542A2D819
:10F16000984255E7854281E7012049E7012003499C
:10F1700020F0D0FF204643E7CAA30500E7A305001F
:10F1800082B02DE9F047ACB00C4634A9054681E8C1
:10F190000C001DF015FC30B1002630462CB0BDE847
:10F1A000F04702B070472B780BB17C2B43D158222B
:10F1B00034A90DEB020028F0DDFCDDE93457DDF861
:10F1C000DC9023F037FA2368A2681A440646D21B63
:10F1D000394628461EF0DFFC002104460246304630
:10F1E0001FF009FF204623F089FF0DF16808002475
:10F1F0004C450DDB384623F0ADF9704902463046E8
:10F200001FF08BFF2A466E4930461FF06DFFC4E7A2
:10F2100058F8041BD8F820202846521A1EF0BBFCD0
:10F22000013482460246214630461FF0E4FE504635
:10F2300023F064FFDCE75E2B09D12368A268D34288
:10F24000AAD120F0B7FF0028A6D0013507E0242B73
:10F250001DD1D4E900329A4205F101050CD85022A3
:10F2600036A9684628F086FC34AB0CCB21462846EC
:10F27000FFF786FF064690E74C2237A9684628F03C
:10F2800079FC34AB0ECB284600F026FAF2E7282BA7
:10F290000FD1379B2168A26834A80A44191D082B96
:10F2A00040F8212000EB83014A63CADC0133379325
:10F2B000C7E7292B0AD1379B002BC2DD34AA02EB0A
:10F2C00083032168A2680A441A63BAE734AB15AA1B
:10F2D00021462846FFF73EFE159FEB5DA3F12A026B
:10F2E000012A804605EB07064ED801372F4450B956
:10F2F0002B2B08D14C2237A9684628F03BFC34ABB5
:10F300000ECB3846C0E7214616A81EF0C7F850229B
:10F3100036A9684628F02EFC34AB0CCB16A938462B
:10F32000FFF72EFF0646199823F0E8FED4E90023E4
:10F330009A42BFF432AFB8F1000F3FF42EAF20462F
:10F340001DF012FF34AB15AA21462846FFF702FE36
:10F350002146804616A81EF0A1F8502236A968461C
:10F3600028F008FC34AB0CCB16A93846FFF708FF91
:10F370008146199823F0C2FEB9F1000FD6D030466D
:10F3800023F0BCFE4E46D1E7D4E900239A420BD2CB
:10F3900050B120461DF0E8FE20F00CFF00283FF49D
:10F3A000FBAE159B1D445AE74C2237A9684628F04E
:10F3B000E1FB34AB0ECB304666E700BF09A4050085
:10F3C0000FA405002DE9F047B4B00646084614AF77
:10F3D00020F04CFB002254498046304621F00FF9C2
:10F3E00020F0C4F9002205465049304621F007F9C3
:10F3F000044623F0BCFC48B92146404623F059FF9F
:10F40000002420468037BD46BDE8F08740461FF007
:10F41000FBFAA842F0D320461FF0F6FA00F10803E9
:10F4200023F00703ADEB030D0DF1500A421C5146CA
:10F4300020461FF0A3FB204623F060FE69213046E2
:10F44000FEF786F84FF48072002387F830007A8642
:10F4500041462A46384687F831307B63C7F8288012
:10F460001EF02CFA394607F114001EF017F850224E
:10F4700007F130016846FD6228F07CFB07F128099E
:10F4800099E80C0007F114015046FFF779FE044695
:10F49000386A23F033FE38461DF066FE2CB9D7E9F2
:10F4A00000239A4205F1010514D3F86823F026FEE3
:10F4B000404623F023FED4B9022022F0D5FF0025D8
:10F4C0000446284623F046F81749024630461FF006
:10F4D00024FE96E7394607F114001DF0DFFF5022A5
:10F4E00007F130016846FD6228F044FBC8E7672158
:10F4F0003046FEF72DF8A0B10021204621F0F2FBA6
:10F50000002280460A49204621F079F820F02EF9A1
:10F51000054640461FF078FA0544404623F0EEFDCC
:10F52000CFE70546CDE700BF46A0050039A005009E
:10F5300009A405002DE9F84F04460D4623F017FCF9
:10F5400020B94FF000084046BDE8F88F23F072F86C
:10F5500080460028F5D01DB921461FF003FDF2E7D3
:10F560005149284621F0AEFA00285FD0002022F051
:10F57000F1FF4E49024628461FF0CFFD214628469E
:10F58000FFF720FF0027064626B1304623F079FA20
:10F590008146D0B1304623F0B1FD002022F0DAFFE1
:10F5A0004249024628461FF0B8FD20461FF02CFABB
:10F5B000B842C8DB39466FF0004220461EF0EBFA35
:10F5C000014640461FF0FAFCBDE74946304621F0AF
:10F5D00089FB4A4636498246304621F010F820F031
:10F5E000C5F8814650461FF00FFA8346504623F077
:10F5F00085FDA9EB0702394620461EF0CCFA0146EC
:10F6000040461FF0DBFC0BEB0907304623F076FD8C
:10F61000384622F09FFF2549024628461FF07DFD0F
:10F6200021462846FFF7CEFE0646ADE7284620F0E5
:10F630001DFA814688B11FF0E7F9074620461FF002
:10F64000E3F9002600F1010BABEB070A35465545FF
:10F6500022DC7FB925BB0135F9E70746EEE75D46B9
:10F6600012E0014640461FF07DFC304623F046FD87
:10F67000EE19F0E75545F2D001232A4649462046C7
:10F68000F1F742F80028E6D1AA1B314620461EF0C9
:10F6900082FA06460028E4D1484623F02FFD52E7BF
:10F6A0005545F1D1F8E700BF32A0050046A005009E
:10F6B00009A4050038B5FFF785FE054650B123F0D3
:10F6C000E0F980F00100C4B2284623F017FD04F0F1
:10F6D000010038BD0446F7E784B0F0B59BB021AE19
:10F6E000054686E80E0020F065FD68B90446204610
:10F6F0001BB0BDE8F04004B070475C2C03D16C78BF
:10F70000002CF4D03D4601352C78002CEFD07C2C19
:10F7100005F10107F1D1DDE9211215A81EF0CEF89F
:10F7200023A95022684628F025FA96E80C0015A96E
:10F730003846FFF725FD0446189823F0DFFCD6E78E
:10F7400037B5054601910B4848F208011EF0E3FC6D
:10F75000044660B12A4608491FF0C6FC284601232A
:10F7600001AA214614F0F8FE204623F0C7FC03B09E
:10F7700030BD00BF27FC02003A8E05002DE9F7439B
:10F78000054608460F46904623F006FA38B93A4631
:10F790002549032020F0BEFC03B0BDE8F083B8F19A
:10F7A000000F0BD00022214928461FF043FC0446DD
:10F7B000E8B121F0B1F904461D4E01E01D4E44466A
:10F7C00000223146284620F01AFF814688B93A4681
:10F7D000314628461FF088FCB8F1000FDCD02846DF
:10F7E0002146FFF7ADFF204623F088FCD4E7804692
:10F7F000E2E723F086F938B1394648461FF0B2FBFC
:10F80000484623F07BFCE7E702216846CDE90097F4
:10F8100022F013FF31460746024628461FF064FCDB
:10F82000384623F06BFCEBE7A5960500C99605006A
:10F830009B960500A096050010B500220446FFF730
:10F840009DFF2046BDE81040FDF74ABA38B5154681
:10F8500001220446FFF792FF25B1002229462046E7
:10F86000FFF78CFF2046BDE83840FDF739BA0000AD
:10F870002DE9F74F054623F099FA044640B92A4688
:10F880003449032020F046FC204603B0BDE8F08F49
:10F89000314900201CF0F2FE04460028F4D048F262
:10F8A00008012E481EF037FC8146D8B122462C496B
:10F8B0001FF01AFC22F0BEFE2946824601A81DF068
:10F8C000B5FB00263546019880B9A81B22F042FE00
:10F8D0002449024620461FF020FC52462249204679
:10F8E0001FF01BFC484623F009FCCDE720F05AFD31
:10F8F0008046FDF723F930B348F260011B481EF043
:10F900000AFC0746284622F025FE002102468346CF
:10F9100038461FF082FE584623F0F0FB224610497D
:10F9200038461FF0E1FB39464A464046FFF78EFF56
:10F93000394623F0BEFC404623F0E0FB01A8013528
:10F940001DF063FBBFE74246294650461FF053FBBC
:10F950000136F0E747990500FA9F05000DFA02000D
:10F960003A8E0500EF9F0500F59F050071F9020032
:10F970002DE9F0410F46904613490022054620F03C
:10F980003EFE1FF0F3FE002204461049284620F0F8
:10F9900036FE0646B0B142463946013C1FF02BFB0D
:10F9A000204622F0D7FD0849024628461FF0B5FB45
:10F9B0001CB931462846FFF7C3FE3046BDE8F0418A
:10F9C00023F09CBBBDE8F081EF9F0500F59F05008B
:10F9D00037B5054601910B4848F208011EF09BFB24
:10F9E000044660B12A4608491FF07EFB28460123E1
:10F9F00001AA214614F0B0FD204623F07FFB03B09E
:10FA000030BD00BF21FC02003A8E050038B500224F
:10FA10000D460949044620F0F2FD58B123F06EFB73
:10FA2000204605491FF071FF29462046BDE83840B1
:10FA3000FFF7CEBF38BD00BFF59F05002DE9F043AD
:10FA400085B006460191414914461FF05EFF4049CA
:10FA500030461FF05AFF00223E49304620F0CFFDCD
:10FA60003C49054630461FF050FF204623F049F838
:10FA7000074660B3214603A81DF0D8FA0024039876
:10FA800078B920F0ADFC804658B301462846FFF710
:10FA90009FFF2A462146404623F0FEFB05B0BDE805
:10FAA000F08320F07FFC01AB0122314681461CF03F
:10FAB00097F8804617B923F021FBA046484623F06B
:10FAC0001DFB03A81DF0A1FA00274446D7E7002C30
:10FAD000D7D0204601AB012231461CF081F8044604
:10FAE000CFE74DB32046FDF729F850B348F208019F
:10FAF00019481EF010FB48F20801064617481EF090
:10FB00000AFB0746A6B198B12A46154930461FF0B0
:10FB1000EBFA2A46124938461FF0E6FA012231462E
:10FB20002046FFF72BFE424639462046FFF726FEC9
:10FB30003946304623F0BDFB2946204623F0B9FB69
:10FB4000ACE721462846FFF7FBFDF5E79B9605004D
:10FB5000A096050011F6050041F70200D1F9020058
:10FB60003A8E0500294B2DE9F047B2F10009284EE5
:10FB700008BF1E460D4600223146804620F03FFD5C
:10FB8000044670BB02462349DFF888A0404620F0B7
:10FB900036FD04464CB9B9F1000F25D12A461E495D
:10FBA0000120BDE8F04720F0B5BA002231462046DA
:10FBB00020F025FD0746024648B129462046FFF7BA
:10FBC0003DFF21463846BDE8F04723F072BB514661
:10FBD000204620F014FD0746204623F08FFA3C46CD
:10FBE000D8E7B9F1000F05D02A460C4940461FF06E
:10FBF0007BFA4CB1404622462946FFF71FFF2046BC
:10FC0000BDE8F04723F07ABABDE8F087A09605007A
:10FC10009B96050011F60500D2960500C9960500D1
:10FC20000022FFF79FBF0122FFF79CBF70B505467A
:10FC30000E4622F06FFF58B9284622F022FF0446F4
:10FC400030B92A460E49032020F064FA204670BDE0
:10FC5000304622F05FFF18B10A49012020F05AFA1D
:10FC600022F0FEFC04460028F0D0284622F052FF85
:10FC70000028EBD02A46044920461FF035FAE5E774
:10FC8000609A0500939A0500D99B0500F7B518F016
:10FC900038FA054618F056FA18B90024204603B081
:10FCA000F0BD22F0DDFC04460028F6D005EB45054A
:10FCB000224B5E195B5D40338DF8043001A80023B0
:10FCC0008DF8053023F081FA1D49024620461FF0C9
:10FCD00024FA707822F03EFC1A49024620461FF0B2
:10FCE0001CFAB57885B122F0BBFC074660B122F062
:10FCF000A1FC064690B905F01F0022F02BFC12492A
:10FD0000024620461FF009FA22F0AAFC024600280B
:10FD1000C4D00E4920461FF000FABFE7AB0606D557
:10FD2000012022F017FC014630461FF047F9324609
:10FD3000074938461FF0F1F9DDE700BFBC7D05003B
:10FD40005C960500AA9D0500B39D0500BB9D0500BE
:10FD5000AE9D05002DE9F74F0BF0BCFB8946074629
:10FD60001EF098FA83460BF0B5FB80468A4622F0D7
:10FD700077FC0446002800F0A680564B5649586888
:10FD8000002220F03CFC0546002800F0A0801EF078
:10FD90005FFD0646284623F0B1F9002501230D2119
:10FDA0004E485A1E01FB0202B2F80B0080060FD02B
:10FDB00010460193009222F01DFF0135019B0D2199
:10FDC00030B1009A12680C32B2FBF1F213441544C0
:10FDD000013340F6C4129342E2D9B018AB1B401B6A
:10FDE000009322F0B7FB3E49024620461FF095F9EA
:10FDF000009B184622F0AEFB3A49024620461FF00F
:10FE00008CF940F6C41022F0A5FB37490246204683
:10FE10001FF083F9304622F09DFB2F490246204611
:10FE20001FF07BF9584622F095FB304902462046E8
:10FE30001FF073F9B8EB07006AEB090127F058F9D6
:10FE400000222B4B27F082F92A4B002227F07EF963
:10FE500041EC100B22F06CFB2749024620461FF0B4
:10FE60005CF90D2022F076FB2449024620461FF063
:10FE700054F9234822F06EFB2249024620461FF027
:10FE80004CF9002022F066FB1F49024620461FF075
:10FE900044F91E4822F05EFB1D49024620461FF031
:10FEA0003CF94FF4D82022F055FB1A49024620466F
:10FEB0001FF033F94FF4002022F04CFB16490246A4
:10FEC00020461FF02AF9204603B0BDE8F08F064611
:10FED00063E700BF482E0020779F0500682E0020B2
:10FEE0007F9F0500849F05008A9F0500909F050065
:10FEF00000408F400000B03E939F05009A9F050090
:10FF0000C8C20020A49F0500B49F0500A4060600F7
:10FF1000C09F0500D19F0500E29F050010B522F0AB
:10FF20009FFB0446294823F050F929490246204600
:10FF30001FF0F3F8274823F048F9274902462046E6
:10FF40001FF0EBF8254823F040F9254902462046EA
:10FF50001FF0E3F84FF4002022F0FCFA214902469A
:10FF600020461FF0DAF84FF4204022F0F3FA1E4941
:10FF7000024620461FF0D1F84FF4803022F0EAFA12
:10FF80001A49024620461FF0C8F804F08BFB1849B6
:10FF9000024620461FF0C1F803F01AFD154902463B
:10FFA00020461FF0BAF8144823F00FF9134902460F
:10FFB00020461FF0B2F8124822F0CCFA114902464E
:10FFC00020461FF0AAF8204610BD00BFDE9E0500A7
:10FFD000E69E0500EE9E0500F79E0500029F0500C7
:10FFE0000B9F0500119F0500179F050038BA0500FB
:10FFF0001F9F0500269F05002E9F0500699F050095
:020000023000CC
:10000000A82D0020719F050038B50849054600203D
:100010001CF034FB044638B1284622F024FB044986
:10002000024620461FF079F8204638BD809D050025
:1000300045A305002DE9F8430D46032107460BF0C3
:100040001FFD002401264FF08008A14615F1FF3561
:1000500002D22046BDE8F88388F311880021384693
:100060000BF01EFA0320F1F763FC012138460BF078
:1000700017FA0A20F1F75CFC38460BF0FDF900B1E5
:10008000344389F311883520F1F752FC7600DDE71F
:1000900010B5032104460BF0F3FC002120460BF0C1
:1000A000FFF94FF4FA70F1F743FC012120460BF001
:1000B000F7F95020F1F73CFC20460BF0DDF904463F
:1000C0004FF4D270F1F734FC84F00100C0B210BDDF
:1000D00008B50022034920F092FABDE8084018F064
:1000E00027B800BF45A305002DE9F04F8BB00C46A3
:1000F000FFF7EEFF064618F025F828B94FF0000884
:1001000040460BB0BDE8F08F22F094FA80460028FC
:10011000F4D0631EFF2B28BFF0242246E317CDE95D
:1001200000234FF000093046FFF7B2FF0028E7D068
:10013000DDE9002308213046FDF7B8FC0124002545
:10014000AA46274601213046FFF774FF01215FFAD6
:1001500080FB3046FFF76EFFBBF1010FC0B22BD121
:1001600001283AD1402FCBDD9DF80C30002BC7D0B1
:1001700005AC0DF10C090025A34619F8017B3809DF
:100180001CF030FC207007F00F001CF02BFC013538
:10019000082D607004F10204EFD1002358468DF859
:1001A000243023F012F8014640461EF007FFD146E6
:1001B000BAF1000FA4D0B6E70AAB2B44834513F87D
:1001C0001C3C2DD14F4524DA1C4214BF4FF0010BCB
:1001D0004FF0000BBBF1000F21D00AAB2B444FF0C6
:1001E000010B13F81C3C23430AAA2A44012102F8FC
:1001F0001C3C30465A4600236400FDF757FC14F0BF
:10020000FF0404BF01350124072D07F1010799DD23
:10021000A8E70CBF4FF0010B4FF0000BDAE7BA462E
:1002200023EA0403E0E770B58AB00C46FFF750FFFD
:10023000064617F087FF68B3204622F0BFFC18B3CC
:1002400020461EF00FFD0146054601201DF07EF9F7
:10025000044650B10146002268461DF056FB15F1D8
:10026000FF3505D268461CF07CFE20460AB070BD02
:1002700008213046FFF7DEFEC1B268461DF091F856
:1002800068461CF097FFEAE708213046FFF7D2FEE8
:1002900022F060F90446E8E737B50D461446FFF74B
:1002A00017FF8DF8070017F04DFF80B10DF1070221
:1002B0000C49284620F0E0FA9DF807004CB10121D6
:1002C0000BF0EEF801219DF807000BF0D9FB03B00D
:1002D00030BD04210BF0D4FB01219DF807000BF089
:1002E000DFF8F4E73BDB020010B5FFF7F1FE044650
:1002F00017F028FF38B12046CC2200230821BDE8A2
:100300001040FDF7D3BB10BD2DE9F04186B00C467F
:10031000FFF7DEFE054617F015FF40B1204622F03C
:1003200026FD38B92246264903201FF0F3FE06B009
:10033000BDE8F08120461EF067FB1028F2D1284668
:10034000FFF7A6FE2146002201A81DF0B7FA0024FF
:1003500027462646A04601A81DF06DF88DF800003E
:1003600001A81DF068F800231A468DF8010010213D
:1003700068468DF802801CF088FDA4F12002C4F1CB
:100380002003A14000FA02F220FA03F31143A04037
:1003900008341943402C47EA000746EA0106DAD13F
:1003A000049822F0ABFE2846552200230821FDF7D1
:1003B0007DFB3A46334621462846FDF777FBB6E7F4
:1003C000889D050010B5FFF783FE044617F0BAFEBE
:1003D00020B12046BDE81040FFF75ABE10BD10B155
:1003E00001211EF001BF70472DE9F74305460F4676
:1003F000914622F0D1FB044640B92A4657490320D2
:100400001FF088FE204603B0BDE8F083284622F0A6
:1004100041FB60B3A98828681DF07DFE04460028D2
:10042000F0D0294668461CF001FE009D7DB3B5F86A
:100430000B3003F50073A5F80B3028461FF0B2FF10
:100440008046284622F0DBFCD8B1B8F1000F2AD054
:10045000012128461EF0C8FE064630B1014620465E
:100460001EF09DFC304622F049FE01260AE0284697
:1004700022F088FB002814BF0820072021F0F4FF99
:10048000CCE706464146284622F013FF6EB9B9F183
:10049000000F0ED1009D002D45D13A46304920462F
:1004A0001EF022FEAEE74646ECE768461CF0ADFDC6
:1004B000BBE7494601A81CF0B9FD01980028E9D026
:1004C0001FF070FF009D064665B1B5F80B3003F5CF
:1004D0000073A5F80B30284622F091FC40B928465D
:1004E00022F00CFE3246002120461FF096F813E061
:1004F0000122002128461FF00FF8314680461DF0EA
:1005000005F9414620461EF04AFC2846414622F0A5
:10051000D0FE68461CF079FD304622F0EFFD01A8C0
:100520001CF073FDC9E7B5F80B30012203F5007329
:10053000A5F80B30114628461EF0EEFF064630B1F6
:10054000014620461EF02BFC304622F0D7FD2846FF
:1005500022F0D4FD68461CF058FD9BE7A7970500E4
:100560003A8E05002DE9F04F8FB0814602AF10465C
:100570008A46164622F01AFC0446002856D0304619
:100580001EF064FAB0F5807F044680460AD9024620
:100590002B4901201FF0BEFD002420463437BD4604
:1005A000BDE8F08F8300DA1D22F00702ADEB020DEB
:1005B00002AD2A462B440021934219D10122314633
:1005C000381D1DF0B2FD381D1CF0FDFC98B9381D1A
:1005D0001CF0CDFC00231946CDE900855246484663
:1005E0001AF018FF29460446404622F038FED4E7A8
:1005F00042F8041BE0E7381D1DF04EFD064622F0D0
:1006000057FC60B130461EF02DFBB0F1000B06DB4D
:100610005C4504DD381D1FF08AFF45F82B0030468D
:1006200022F06CFD381D1EF093FBCCE72EB1324654
:10063000044901201FF06EFDAFE7B0463546C9E71B
:10064000239705006C9705002DE9F34704460D46F6
:1006500022F0A2FA30B9444903201FF05BFD02B03A
:10066000BDE8F087284622F097FA0028F3D020460C
:1006700022F010FA0646284622F00CFA86420AD0EA
:10068000284622F007FAB4F80B30002842D043F095
:100690004003A4F80B30204622F074FA06462846A0
:1006A00022F070FA86420BD0284622F06BFAB4F89A
:1006B0000B3023F03F0380B343F00803A4F80B3062
:1006C00000222A49DFF8A490DFF8A4A020461EF0FB
:1006D000B1FC00222649074620461EF0ABFC064628
:1006E00020461FF02DF9294601A81CF09FFC019D12
:1006F000B5B91FB1394620461EF051FB384622F0ED
:10070000FDFC1EB1314620461EF049FB304622F06A
:10071000F5FCA4E723F04003BBE743F00703CDE774
:10072000B5F80B3003F5007301A8A5F80B301CF0E9
:100730006CFC494628461EF047F988B951462846C0
:100740001EF042F960B9012128461EF04DFD804699
:1007500030B1014620461EF022FB404622F0CEFC7E
:10076000284622F0CBFCC2E7DE970500FC97050087
:100770007DF305002DE9F74305460F46144622F0A8
:10078000B7FB30B9354903201FF0C4FC03B0BDE806
:10079000F083384622F0EBFA08B93149F3E72046F6
:1007A00022F0FAF928B9204622F0E1FA08B92D49D9
:1007B000E9E739462C481FF035FC80460028E5D093
:1007C0000146012228461EF03CFE0646404622F025
:1007D00095FC30461FF0E6FD804620BB21463046A2
:1007E0001CF094FF3146404622F063FD1F49384615
:1007F0001EF0EAF80028C9D000221D4928461FF043
:10080000FEFE019022F0B3FA48B11A4928460123AE
:1008100001AA13F0D9FE164928461FF076F8019870
:1008200022F06CFCB2E722F06CF920B12146404680
:100830001EF098FBD6E721F0FDFE414681461EF0F2
:1008400091FB214648461EF08DFB494630461CF080
:100850005DFF484622F052FCC4E700BFE39B050061
:100860001A9C0500519C0500A99C0500FA950500FD
:1008700027A20500AF9C0500F8B5064608461446B9
:100880001F4622F0A2FC3946054620461DF043FCD7
:100890002946044602463046FFF76CFF29462046AB
:1008A000BDE8F84022F005BD73B505460C4622F0C0
:1008B0001FFB20B9214903201FF02CFC1AE0204621
:1008C00022F055FAC0B121461D481FF0ABFB064689
:1008D00080B10146012228461EF0B3FD0446304691
:1008E00022F00CFC34B1284621461EF049FF204678
:1008F00022F004FC02B070BDF4B9294601A81CF036
:1009000095FB104E019C002CF4D0B4F80B3003F58D
:10091000007301A8A4F80B301CF077FB01223146CC
:1009200020461EF049F818B1214628461EF028FF3F
:10093000204622F0E3FBE5E70349BCE7E39B050023
:10094000A99C0500B79C0500BB9C050038B5054671
:10095000084622F03AFC044640B101462846FFF71B
:10096000A3FF2046BDE8384022F0C8BB38BD0000D8
:10097000F8B507460C46164622F0BAFA28B92149BE
:100980000320BDE8F8401FF0C5BB204622F0EFF978
:10099000A8B321461C481FF045FB044688B3014616
:1009A000012238461EF04DFD0546204622F0A6FBEA
:1009B00028461FF0F7FC044640B186420BD1294679
:1009C00038461EF0DDFE204622F098FB2846BDE8A2
:1009D000F84022F093BB22F094F80028F3D031467F
:1009E0000122204621F046FB06460028EBD00146B6
:1009F00020461EF0C5FE304622F080FBE3E70349A7
:100A0000BEE7F8BDE39B0500A99C0500109D05000D
:100A10002DE9F04786B000AF81460C461546E84602
:100A200022F066FA40B9264903201FF073FB1837FD
:100A3000C546BD46BDE8F087204622F098F908B9C2
:100A40002049F1E7214620481FF0ECFA82460028B1
:100A5000EDD02946381D1CF0E9FA002407F10805FD
:100A6000786830B1042C21D12246184903201FF0A8
:100A700051FB786822F042FB0022514648461EF0A6
:100A8000E0FC20F049F80646504622F037FB2EB134
:100A900023462A463146484613F05EFD304622F092
:100AA0002DFB2946204622F0DAFBC0E71FF07AFC36
:100AB00045F82400381D1CF0A8FA0134D0E700BF27
:100AC000E39B0500669B0500A99C05009F9B050014
:100AD000F7B5014601A81CF0A9FA1A4F00260198A3
:100AE000C8B11FF05FFC044648B321F0CAFF0546B9
:100AF00028BB204622F00EF898B92246394603203A
:100B00001FF008FB0125204622F0F8FA01A81CF08E
:100B10007CFA002DE3D0019822F0F0FA304603B0C1
:100B2000F0BD3EB9B4F80B3003F50073A4F80B30F8
:100B30002646E8E7214630461FF03DFDE3E7002565
:100B4000E1E700BF469A050070B505460E4622F063
:100B500023F8A8B10122104928461EF06BFA04467A
:100B600021F069FF90B922460C4903201FF0D2FA08
:100B7000204622F0C3FA2846BDE8704021F02CBC84
:100B8000284621F0C7FF0028E4D1E8E73146204697
:100B90001CF0BCFDECE700BFD99B0500539D050090
:100BA0002DE9F84304460F46164621F0B3FF0546EB
:100BB00040B92949224601201FF0ACFA2C462046B4
:100BC000BDE8F883304621F0A5FF054610B932464E
:100BD0002249F0E7384621F073FB00222049814684
:100BE00030461FF00CFD002207461E4930461FF01C
:100BF00006FD8046B7B9A8B900221B4930461FF050
:100C0000FEFC05462A46494620461EF04CFC294675
:100C1000484622F04EFBB4F80B3003F50073A4F8FD
:100C20000B30CCE7062021F01FFC054660B11FB158
:100C30003A460B491EF058FAB8F1000F04D042466C
:100C4000084928461EF050FA4146384622F031FB4A
:100C5000002DD7D1D0E700BF0E9B0500379B0500C4
:100C6000A2B805000EB605006EA2050073B50446D5
:100C70000D4621F04FFF064640B91A492246012091
:100C80001FF048FA3446204602B070BD284621F0D5
:100C900041FF064610B92A461349F0E7294601A844
:100CA0001CF0C4F9019D35B9B4F80B3003F500739D
:100CB000A4F80B30E7E7B5F80B3003F50073A5F89F
:100CC0000B3028461FF06EFB29460646024620469A
:100CD000FFF766FF3246294622F0DEFA01A81CF033
:100CE00094F9DFE7B99A0500E39A050070B5044668
:100CF00088B0084621F0E4FA0646204622F0F8F8CB
:100D0000054640B10022314620461EF09AFB10B144
:100D100022F0F4F904E0204621F0FCFE30B1002579
:100D2000304622F0EBF9284608B070BD204611F09D
:100D3000DDFB05460028F2D02022694630461DF032
:100D40001DFF28466A46214611F026FD051C18BFE6
:100D50000125DDE7F8B507460C46FFF7C7FF10B9D8
:100D600000242046F8BD204621F0AAFA01220446BC
:100D70000146384616F038F90546204622F0BEF9FD
:100D8000002DEDD021F06CFC0446284614B922F069
:100D9000B5F9E6E721F061FE064638461CF0EAFBAD
:100DA0000746012021F0CEFB2349024620461EF0D3
:100DB000B4F9002F37D02846B84780F00100C0B200
:100DC00000F0010021F0BEFB1C49024620461EF047
:100DD000A4F986F00100C0B221F0B4FB1849024624
:100DE00020461EF09AF928461EF049FC064621F0DE
:100DF000E3FDD0B10022134930461FF000FC114939
:100E0000024620461EF089F900220F4930461FF0A5
:100E1000F6FB0D49024620461EF07FF9304622F0CF
:100E20006DF92846B3E70120CAE728461FF0BAFA51
:100E300006490246EFE700BFB89B0500C19B0500CD
:100E4000CC9B0500A2B805000EB605006EA20500F9
:100E500010B5142994B0A8BF14210C461FF094FFBC
:100E600024EAE4740A2351EC100B009302AA4623EF
:100E700001941BF0E1FD02A822F0A7F914B010BD07
:100E800030B5044695B008460D4621F0E3FF48B35F
:100E9000204621F093FE28B328461DF0E3FE831E72
:100EA000222B05461ED8204621F0D4FF60B12046F3
:100EB0001DF0D8FE2B46012202A91BF09AFD02A8C4
:100EC00022F083F915B030BD20461FF05DFF4FF0D2
:100ED000FF33CDE9005302AA462351EC100B1BF05F
